:100000000C94740A0C94950A0C94950A0C94F40FB1
:100010000C942E100C94950A0C94950A0C94950A45
:100020000C94950A0C94950A0C94950A0C94950AD4
:100030000C94950A0C94950A0C94950A0C945E13F2
:100040000C94950A0C94950A0C94950A0C94950AB4
:100050000C94950A0C941F640C94950A0C94950AC0
:100060000C94950A0C949A640C94950A0C94950A35
:100070000C94950A0C94950A0C94950A0C94950A84
:100080000C9435780C94950A0C94950A0C94950A66
:100090000C94C9640C94950A0C94950A0C94950AD6
:1000A0000C94950A0C94950A0C94950A0C94950A54
:1000B0000C94950A0C94950A0C94950A0C94950A44
:1000C0000C94950A0C94950A0C94950A0C94950A34
:1000D0000C94950A0C94950A0C94950A0C94950A24
:1000E0000C94950A0C945A6B0C94646B0C94506BA2
:1000F0000C94106B0C94906B0C94866B0C947A6B34
:100100000C946E6B0C94950A0C94950A0C94950AB9
:100110000C94950A0C94950A0C94950A0C94950AE3
:100120000C94950A0C94950A0C94950A0C94950AD3
:100130000C94950A657E847E027FF17F1180318068
:100140003980E67F084AD73B3BCE016E84BCBFFDB9
:10015000C12F3D6C74319ABD56833DDA3D00C77F97
:1001600011BED9E4BB4C3E916BAAAABE0000008030
:100170003F07634236B79BD8A71A39685618AEBAFC
:10018000AB558C1D3CB7CC5763BD6DEDFD753EF690
:10019000177231BF000000803F08000000BE9224AB
:1001A00049123EABAAAA2ABECDCCCC4C3E000000E0
:1001B00080BEABAAAAAA3E00000000BF00000080DB
:1001C0003F0000000000084178D3BB4387D1133DB6
:1001D000190E3CC3BD4282AD2B3E68EC8276BED97F
:1001E0008FE1A93E4C80EFFFBE01C4FF7F3F0000BE
:1001F000000000000C947A660C9407780C94C2847A
:100200000C94B9810C944D810C94E67F0C94F47499
:100210000C94F4670C9410780C9434730C944E374F
:100220000C9437730C9420730C94E3720C947B4BF6
:100230000C947D650C9487720C9413690C942A734A
:100240000C94DA760C94D7760C942F730C94AC68DB
:100250000C9429150C94204C0C9441670C94041DAB
:100260000C9415160C9438670C94D56C0C94847E01
:100270000C94AB6B0C94EE710C94027F0C94666939
:100280000C9425730C9431800C942A650C94228173
:100290000C94F1590C94FA710C94FA100C94678533
:1002A0000C94D2760C9439800C94657E0C947281F7
:1002B0000C9476770C94FE810C946F660C9467888E
:1002C0000C94B0720C945F0E0C9499860C94A965F2
:1002D0000C947E4C0C949B770C94F17F0C94790ECB
:1002E0000C94966A0C9411806E616E00696E6600C3
:1002F00025630025730A005854414C5F5452494D00
:100300003D25640025730A0025730A005465737443
:1003100020362025730A0054657374203520257318
:100320000A005465737420342025730A00546573E1
:100330007420332025730A005465737420322025FD
:10034000730A005465737420312025730A006368B2
:10035000616E3D25640A0074787077723D25640AE9
:10036000003530306B0A003235306B0A00313135E0
:100370006B0A0035366B0A0033386B0A0025730AA6
:1003800000765F6C6F773D252D332E32660A00258F
:10039000730A0073656E743D252D75206475703D7C
:1003A000252D752069676E6F7265643D252D75205A
:1003B00074746C5F7A65726F3D252D750A00253760
:1003C0002E33662025372E33660025352E326620E3
:1003D000004572726F72203020566F6C74004E6F41
:1003E0007420737570706F727465640A0045727260
:1003F0006F72203020566F6C74004572726F7220DD
:100400003020566F6C740062756C6B5F64656C6154
:10041000793D252D750062756C6B3D252D75005657
:10042000616C7565206E6F7420616C6C6F776564AC
:100430000062756C6B3A206D61783D257520737490
:100440006172743D25752C20656E643D25752C20E8
:10045000696E5F7573653D25750A007062323D25D2
:10046000730A00256C7500416C6C6F7765642073AE
:100470007065656420312F31302F3130302F3430AA
:1004800030206B6269742F730025630074746C3DB7
:10049000252D64200074746C3D252D6420004E656C
:1004A000772074746C3D252D6420002563004D5326
:1004B0003536313120503D252D372E326620252D01
:1004C000372E32666D0A00424D5030383520256C8B
:1004D000642050612020252D372E32666D00256363
:1004E00000545F484541545F4944583D252D352E01
:1004F00032662000545F4445573D252D352E326627
:10050000200041483D252D352E32662000545F5392
:10051000485432583D252D352E3266200052485F12
:1005200053485432583D252D352E32662000545FF5
:1005300052483D252D342E3166200052483D252D50
:10054000342E3166200025630025630025630025D5
:1005500063002563007265706F72745F616C6C3D3F
:10056000007265706F72743D00256300256300257D
:100570006300256300204F534343414C3D256420D5
:100580000020467573653A2065653D253032782038
:1005900068663D25303278206C663D253032782003
:1005A0006C623D25303278004D43553D2530366C28
:1005B000780025630074785F6C656E3D252D6C7541
:1005C0002C765F6C6F773D252D6C752C73687432BB
:1005D000783D252D6C752C62756C6B3D252D6C75E9
:1005E000002563004F4B0A00256300256300256347
:1005F0000025630025630025630025630025630053
:1006000064656275675F616C6C3D00646562756707
:100610003D0064656275673D0025730A0064656589
:10062000700A006E6F6E650A00707772733D00701D
:1006300062323D25730A007062313D25730A0069FC
:100640006E74725F7365635F70313D252D372E3395
:10065000660A00696E74725F70313D252D6C640A04
:1006600000696E74725F7365635F70303D252D376E
:100670002E33660A00696E74725F70303D252D6CF2
:10068000640A00765F6D63753D252D352E32660A4E
:1006900000745F6D63753D252D352E32660A00703E
:1006A0007077723D25730A0064656275673D00725C
:1006B000636D643D25730A0025730A006175746FCC
:1006C0000A006C6F675F6D6F64653D007573625FF4
:1006D0007077723D25730A0072656C61793D2573F0
:1006E0000A0074746C3D252D640A0052494D455F23
:1006F000616464723D252D642E252D640A006E65AB
:10070000696768626F725F7461626C655F73697A52
:10071000653D25640A00765F6C6F773D252D332E8D
:1007200032660A00747870773D25640A0063686158
:100730006E3D25640A0069643D006932635F62753D
:10074000733D006932635F73706565643D252D6C90
:10075000750A007478743D25730A005379737465C3
:100760006D2053756D6D6172790A002530366C7895
:100770000041744D65676132353652465232004150
:10078000744D656761313238524652320041744DC2
:100790006567613634524652320041744D65676177
:1007A00031323852464131004D43553D006D617341
:1007B0006B3D002C00696E74657276616C3D252D71
:1007C000750023252D642C00745F686561745F6972
:1007D000647800745F64657700616800705F6D73B2
:1007E000353631310072685F736874327800745F37
:1007F0007368743278007061007000616434006165
:10080000643300616432006164310061330061323D
:1008100000613100765F696E007268006572720077
:10082000757074696D650070315F6C737400703140
:100830005F740070310070305F6C73740070305FF3
:100840007400703000765F6D637500745F6D637562
:100850000074310074006964006536340074787483
:10086000002D002B006175746F006E6F6E65006265
:10087000756C6B00706F7765725F736176655F6C26
:10088000656472790072656C61795F6C656479008A
:10089000636F6D7061737300616363656C00707288
:1008A000657300705F707772006165730070315F0F
:1008B0006C6564790070305F6C65647200657665A4
:1008C0006E74006C6564006F7700706B74007478F0
:1008D0005F6C6564790072785F6C656472006F703C
:1008E0006572006E6F6E65002530327800765F614C
:1008F00064343D252D382E3666002000765F616415
:10090000333D252D382E3666002000765F61643237
:100910003D252D382E3666002000765F6164313D1E
:10092000252D382E3666002000765F6C6967687466
:100930003D252D382E3666002000765F61323D253C
:100940002D372E3366002000765F61313D252D372F
:100950002E3366002000765F696E3D252D352E32E0
:100960006600204E657665722D757365642073741C
:1009700061636B203E2025642062797465730A00F0
:10098000757074696D653D252D642D646179732DD5
:10099000253032643A253032643A253032642D688D
:1009A0006F7572730A0074657374205B6F66667C82
:1009B000317C327C337C347C355D2020202020202B
:1009C00020202D2074657374206D6F6465730A0D8B
:1009D000007478205B706B74207061796C6F616457
:1009E0005D2020202020202020202020202D20736A
:1009F000656E6420726164696F20706B74206B6532
:100A000079626F6172640A0D00776474205B6F6EA7
:100A10007C6F66667C746573745D202020202020C6
:100A200020202020202D207761746368646F670A7E
:100A30000D00765F6C6F77205B765F6C6F775D2063
:100A400020202020202020202020202020202D2099
:100A50006C6F77657374207265706F727420766F37
:100A60006C746167650A0D00757067722020202024
:100A70002020202020202020202020202020202076
:100A8000202020202D207265626F6F7420766961AE
:100A900020626F6F746C6F616465720A0D0075611E
:100AA0007274205B33386B7C35366B7C3131356B3F
:100AB0007C3235306B7C3530306B5D202D2073659A
:100AC00074207465726D2F75617274207370656522
:100AD000640A0D00626F6F742020202020202020E7
:100AE0002020202020202020202020202020202006
:100AF0002D207265626F6F740A0D0070777273201B
:100B00005B646565707C6E6F6E655D2020202020C3
:100B1000202020202020202D206D637520736C65FF
:100B20006570206D6F64650A0D00726573742065D1
:100B30006570726F6D202020202020202020202032
:100B40002020202020202D20726573746F72652074
:100B5000656570726F6D0A0D0070707772205B6F43
:100B60006E7C6F66665D20202020202020202020C3
:100B700020202020202D2070726F6772616D6D61C2
:100B8000626C65207077720A0D0070623220205B03
:100B90006F6E7C6F66665D20202020202020202044
:100BA0002020202020202D2070726F6772616D6DD3
:100BB00061626C652070696E2062320A0D0070629D
:100BC0003120205B6F6E7C6F66665D2020202020C8
:100BD000202020202020202020202D2062756C6BDA
:100BE000204750494F2070696E0A0D0074787420B8
:100BF0005B737472696E675D2020202020202020A6
:100C000020202020202020202D2053657420726574
:100C1000706F7274207465787420737472696E6773
:100C20000A0D0074787077205B31352D305D2020FF
:100C30002020202020202020202020202020202DA7
:100C4000205458205077722E204869676865737465
:100C5000203020283364426D290A0D0074746C2002
:100C60005B302D31355D20202020202020202020C9
:100C700020202020202020202D2074696D652D74D7
:100C80006F2D6C69766520666F72207061636B658D
:100C900074730A0D00737320202020202020202050
:100CA0002020202020202020202020202020202044
:100CB000202D2073797374656D2073756D6D61726D
:100CC000790A0D007273202020202020202020206F
:100CD0002020202020202020202020202020202014
:100CE0002D20726164696F2073746174730A0D0042
:100CF0007269205B236E5D205B696E745D2020202D
:100D00002020202020202020202020202D2072653F
:100D1000706F727420696E74657276616C0A0D0072
:100D200072636D64205B6F6E7C6F66665D20202051
:100D30002020202020202020202020202D20616C19
:100D40006C6F7720636D642066726F6D206E6574C2
:100D50006F726B0A0D007265205B236E5D205B2B4A
:100D60007C2D5D205B6D61736B7C6175746F2C6D88
:100D700061736B5D202D206D6F7465207265706FDF
:100D80007274207365742F6D6F646966790A0D0043
:100D90006F772020202020202020202020202020AD
:100DA0002020202020202020202020202D206F6E99
:100DB000652D776972652073656E736F72730A0DA6
:100DC000006C6F67205B6175746F7C6F6E7C6F6603
:100DD000665D20202020202020202020202D206D36
:100DE0006F7465732064617461206F6E2055534287
:100DF0000A0D006E65205B666C7573685D202020AF
:100E00002020202020202020202020202020202DD5
:100E1000206E65696768626F72207461626C650A32
:100E20000D0065727220202020202020202020200C
:100E300020202020202020202020202020202D20A5
:100E40006572726F722073746174730A0D006D6342
:100E5000752020202020202020202020202020203D
:100E6000202020202020202020202D206D63752090
:100E7000696E666F0A0D00693263205B70726F6283
:100E8000657C737065656420236E5D2020202020C2
:100E90002020202D206932632070726F62652062ED
:100EA00075737C73657420627573207370656564F7
:100EB0000A0D006964205B72657365745D202020F3
:100EC0002020202020202020202020202020202D15
:100ED0002069642068616E646C696E670A0D006841
:100EE000756D202020202020202020202020202060
:100EF00020202020202020202020202D2068756DFB
:100F000069646974792073656E736F720A0D00727B
:100F1000656C6179205B6F6E7C6F66667C73746153
:100F200074735D20202020202020202D2072656CED
:100F30006179206E6574776F726B207265706F7265
:100F400074730A0D006465205B6D61736B5D202016
:100F50002020202020202020202020202020202091
:100F6000202D2064656275670A0D006368616E203C
:100F70005B31312D32365D202020202020202020A2
:100F8000202020202020202D206368616E20313118
:100F90002D32362028322E3430352D323438302060
:100FA0004D687A290A0D0063616C69205B5B765F8E
:100FB000696E7C61317C61325D20766F6C747C720D
:100FC000657365747C6E6F6E655D202D2063616C4A
:100FD0006962726174650A0D0062756C6B205B5BFF
:100FE00073686F777C666C7573685D205B7365747E
:100FF0002074687273682064656C61795D5D20207F
:101000002D2062756C6B696E67207061636B65740F
:1010100073200A0D006164632020202020202020FE
:1010200020202020202020202020202020202020C0
:10103000202D2073686F7720765F696E2C206131D8
:101040002C20613220766F6C74616765730A0D0025
:10105000752020202020202020202020202020203B
:101060002020202020202020202020202D207570CE
:1010700074696D650A0D0076202020202020202034
:101080002020202020202020202020202020202060
:101090002020202D2076657273696F6E0A0D00681E
:1010A0002020202020202020202020202020202040
:1010B00020202020202020202020202D2068656C4A
:1010C000700A0D00256300756E6B6E6F776E20637E
:1010D0006D640A00484D43353838330025730025C8
:1010E0007300202573002025362E3266200025301F
:1010F00032780074656D705F65787465726E3D2539
:101100002D362E326600202573002025362E3266BD
:10111000204F6E2D426F617264002530327800746A
:10112000656D705F626F6172643D252D362E32668B
:10113000000A0042756C6B2072656D3A2073746111
:1011400072743D25752C20656E643D25752C2069D3
:101150006E5F7573653D25750A0042756C6B206185
:1011600064643A2073746172743D25752C20656E39
:10117000643D25752C20696E5F7573653D25750A84
:101180000042756C6B207468726573683A207469EC
:101190006D65723D25750A00503A20256C6420501B
:1011A000612020252D372E3266206D0A00493243FA
:1011B0003A20004E657665722D75736564207374F0
:1011C00061636B203E2025642062797465730A0098
:1011D0004A54414720726573657474210A0057614F
:1011E000746368646F67207265736574210A0042D6
:1011F000726F776E6F7574207265736574210A0063
:1012000045787465726E616C207265736574210A2D
:1012100000506F7765722D6F6E2072657365742153
:101220002E0A004F6E6C696E650A00526F75746904
:101230006E6720456E61626C65640A0052504C20F6
:10124000456E61626C65640A0025732025732C204D
:101250006368616E6E656C202575202C206368655F
:10126000636B207261746520257520487A2074783C
:1012700020706F7765722025750A000A2A2A2A2AAB
:101280002A2A2A426F6F74696E672025732A2A2AD8
:101290002A2A2A2A0A004A54414720726573657433
:1012A000210A005761746368646F67207265736513
:1012B00074210A0042726F776E6F757420726573C5
:1012C0006574210A0045787465726E616C207265E0
:1012D000736574210A00506F7765722D6F6E2072EE
:1012E000657365742E0A00726E6720697373756585
:1012F000732025640A00454550524F4D20697320E4
:10130000636F72727570742C20726577726974697C
:101310006E6720776974682064656661756C7473A4
:101320002E0A006C6F63616C686F73740041544DDA
:101330004547413235367266723200020000FFFEC8
:10134000000001452025642E256420636C6F636BCB
:1013500020256C752063707520256C75206C706D70
:1013600020256C752069727120256C7520676C656D
:101370006420256C7520796C656420256C7520725D
:101380006C656420256C7520747820256C75206C44
:10139000697374656E20256C752073656E736F724A
:1013A0007320256C752073657269616C20256C75DE
:1013B0000A0000407A10F35A00A0724E180900107B
:1013C000A5D4E80000E87648170000E40B540200BA
:1013D00000CA9A3B000000E1F505000080969800E5
:1013E000000040420F000000A0860100000010270E
:1013F00000000000E803000000006400000000009E
:101400000A00000000000100000000002C76D888CF
:10141000DC674F0823DFC1DFAE59E1B1B796E5E3E2
:10142000E453C63AE651997696E8E6C28426EB89FB
:101430008C9B62ED407C6FFCEFBC9C9F40F2BAA598
:101440006FA5F490055A2AF75C936B6CF9676DC130
:101450001BFCE0E40D47FEF520E6B500D0ED902E34
:101460000300943577050080841E080000204E0A92
:10147000000000C80C333333330F986E12831141D0
:10148000EF8D2114893BE65516CFFEE6DB18D1849B
:101490004B381BF77C1D901DA4BBE42420328472C2
:1014A0005E228100C9F124ECA1E53D274E414E4961
:1014B0004E495459494E46CDCCCC3D0AD7233C1712
:1014C000B7D13877CC2B329595E6241FB14F0A005F
:1014D0000020410000C84200401C4620BCBE4CCA4F
:1014E0001B0E5AAEC59D740011241FBECFEFD1E86C
:1014F000DEBFCDBF00E00CBF1AE0A0E0B2E0E8E341
:10150000FAE201E00BBF02C007900D92A033B107D1
:10151000D9F729E3A0E3BAE001C01D92A03FB207CA
:10152000E1F70E94AF620C941A950C9400002F9280
:101530003F924F925F926F927F928F929F92AF9263
:10154000BF92CF92DF92EF92FF920F931F93CF93B0
:10155000DF93CDB7DEB763970FB6F894DEBF0FBE4B
:10156000CDBF7C011B016A01FC01178216828381B9
:1015700081FF66C3BE016F5F7F4F4B01F70193810F
:10158000F10193FD859193FF81911F01882309F457
:1015900053C3853239F493FD859193FF81911F01E7
:1015A000853239F4B70190E00E94F491560165014B
:1015B000E5CF10E0512C20E02032A0F48B3269F00E
:1015C00030F4803259F0833269F420612CC08D32BE
:1015D00039F0803339F4216026C02260246023C0B2
:1015E000286021C027FD27C030ED380F3A3078F44D
:1015F00026FF06C0FAE01F9F300D1124132F13C0E1
:101600006AE0569E300D1124532E20620CC08E329B
:1016100021F426FD11C3206406C08C3611F4206825
:1016200002C0883641F4F10193FD859193FF8191C9
:101630001F018111C1CF9BEB980F933018F42061EB
:10164000805E06C09BE9980F933008F0AAC12F7EF8
:1016500026FF16E02F73722E853621F4F22FF064E8
:101660007F2E08C0863621F4622F6068762E02C075
:101670001111115077FE07C01C3348F444244394E1
:10168000410E27E00BC0183030F4212F06C027E0B0
:101690004CE3442E03C027E017E0412C560174E0D0
:1016A000A70EB11CF6016081718182819381042DA6
:1016B000A4010E946C906C01098100FF02C003FF2D
:1016C00006C071FC07C072FC08C0612C08C03DE276
:1016D000632E05C02BE2622E02C090E2692E802F9D
:1016E0008C7099F1662011F084E001C083E08515CB
:1016F00010F0512C0BC0581A73FC08C0B70180E2DF
:1017000090E00E94F4915A94C9F7F3CF662029F033
:10171000B701862D90E00E94F49103FD03C00CEE0A
:1017200012E002C008EE12E0F72DF0717F2EF801F2
:101730008491882309F476C271108052B70190E039
:101740000E94F4910F5F1F4FF2CF77FE0FC04C0C39
:1017500004FF04C08A81813309F44A94141474F597
:10176000F8E0F41578F588E0482E2CC076FC2AC005
:10177000812F90E08C159D059CF06CEFC6166FEFE5
:10178000D60674F0772D7068772E0AC0E2E0F0E09C
:10179000EC0FFD1FE10FF11D8081803319F4115012
:1017A0001111F4CF77FE0EC044244394410E812FD3
:1017B00090E0C816D9062CF41C1904C044244394A4
:1017C00001C010E077FE07C01C141D043CF4960114
:1017D0002F5F3F4F05C025E030E002C021E030E040
:1017E000662011F02F5F3F4F112331F0412F50E061
:1017F0004F5F5F4F240F351F452D50E024173507ED
:1018000014F4521A01C0512C872D897049F45520C7
:1018100039F0B70180E290E00E94F4915A94F7CF3A
:10182000662029F0B701862D90E00E94F49173FCA8
:1018300009C0552039F0B70180E390E00E94F4918F
:101840005A94F7CF77FE5FC09C2D8D2DD7FE02C036
:1018500090E080E0692E782E40E050E0C6018419C7
:1018600091099D878C87960126193709280D391D06
:10187000812F90E0EE27FF27E81BF90BFF87EE870B
:10188000FFEF6F167F0669F4B7018EE290E02B8BB5
:101890003A8B488B598B0E94F491598948893A892F
:1018A0002B89C614D70454F06C857D8566157705A1
:1018B0002CF4F901E40FF51F818101C080E371E090
:1018C000671A71084F5F5F4FEE85FF856E167F06C2
:1018D0006CF0B70190E02B8B3A8B488B598B0E94B0
:1018E000F4912B893A8948895989CACF6C147D04AF
:1018F00039F49A81963318F4953311F404FF81E397
:10190000B70190E04BC08A81813309F00F7EB701A7
:1019100090E00E94F491111105C074FE18C085E496
:1019200090E017C0B7018EE290E00E94F49182E04F
:1019300066246394680EF401E80FF11D8081B701FD
:1019400090E00E94F491115041F3862DF1CF85E68D
:1019500090E0B7010E94F491D7FC05C0C114D104F6
:1019600039F404FF05C0D194C194D1088DE201C0BF
:101970008BE2B70190E00E94F49180E36AE0C61622
:10198000D1042CF08F5FFAE0CF1AD108F7CFB7015E
:1019900090E00E94F491B701C601C0960E94F491B4
:1019A00041C1833631F0833779F0833509F058C06F
:1019B00021C0560172E0A70EB11CF6018081898317
:1019C00001E010E0640114C05601F2E0AF0EB11C5A
:1019D000F601C080D18026FF03C0612F70E002C0F5
:1019E0006FEF7FEFC6012B8B0E94A0918C012B899A
:1019F0002F7715C05601F2E0AF0EB11CF601C08082
:101A0000D18026FF03C0612F70E002C06FEF7FEF2F
:101A1000C6012B8B0E9455918C012B892068722E58
:101A200023FD1AC0852D90E008171907A8F4B70107
:101A300080E290E00E94F4915A94F4CFF60177FC92
:101A4000859177FE81916F01B70190E00E94F4913A
:101A500051105A94015011090115110579F7E2C08E
:101A6000843611F0893651F5560127FF09C0F4E09C
:101A7000AF0EB11CF60160817181828193810AC031
:101A8000F2E0AF0EB11CF60160817181882777FD0D
:101A90008095982F022F0F7697FF08C0909580951C
:101AA000709561957F4F8F4F9F4F00682AE030E01F
:101AB000A4010E94F592C82EC8183EC0022F853797
:101AC00021F40F7E2AE030E01DC0097F8F3691F0AF
:101AD00018F4883559F0B0C0803719F0883711F004
:101AE000ABC0006104FF09C0046007C024FF08C048
:101AF000066006C028E030E005C020E130E002C00A
:101B000020E132E0560107FF09C0F4E0AF0EB11C3E
:101B1000F601608171818281938108C0F2E0AF0E8D
:101B2000B11CF6016081718180E090E0A4010E9407
:101B3000F592C82EC8180F7706FF0BC0202F2E7FF6
:101B4000C11650F404FF0AC002FD08C0202F2E7EEB
:101B500005C0DC2C202F03C0DC2C01C0D12E24FFBB
:101B60000DC0FE01EC0DF11D8081803311F4297E42
:101B700009C022FF06C0D394D39404C0822F867874
:101B800009F0D39423FD13C020FF06C01C2DD514EB
:101B900018F4150D1D19D52CD51468F4B70180E281
:101BA00090E02B8B0E94F491D3942B89F5CFD51420
:101BB00010F45D1801C0512C24FF12C0B70180E35E
:101BC00090E02B8B0E94F4912B8922FF17C021FFFC
:101BD00003C088E590E002C088E790E0B7010CC040
:101BE000822F867859F021FD02C080E201C08BE28D
:101BF00027FD8DE2B70190E00E94F491C11638F400
:101C0000B70180E390E00E94F4911150F7CFCA949D
:101C1000F401EC0DF11D8081B70190E00E94F49178
:101C2000C110F5CF552009F4C2CCB70180E290E095
:101C30000E94F4915A94F6CFF7018681978102C0F1
:101C40008FEF9FEF63960FB6F894DEBF0FBECDBF48
:101C5000DF91CF911F910F91FF90EF90DF90CF9088
:101C6000BF90AF909F908F907F906F905F904F90BC
:101C70003F902F9008958115910511F00197F1F78C
:101C8000089589E296E09F938F930E943892809105
:101C9000660290916702A0916802B09169020F906C
:101CA0000F9093FF03C083E296E002C08DE196E0BF
:101CB0009F938F930E9438920F900F900895E09118
:101CC000E21CEF73F0E0ED5CF24E80838091E21C49
:101CD0008F5F8093E21C8091833588608093833589
:101CE0004CE452E061E1CA010E94146F80E090E090
:101CF0000895CF93DF93EC014091891350918A139B
:101D000060918B1370918C1346FF1DC08E811F92C2
:101D10008F938D811F928F938C811F928F938B81D4
:101D20001F928F938A811F928F9389EE92E09F93E7
:101D30008F930E9426928DB79EB70C960FB6F8949B
:101D40009EBF0FBE8DBFBE018BE79AE00E940B7055
:101D5000BE0188E092E0DF91CF910C9498701092D0
:101D6000991D10929A1D1092981D0895CF92DF929E
:101D7000EF92FF920F931F93CF93DF93EC01FB0140
:101D80008091981D843108F0B7C080919A1D64E15C
:101D90000E94298790939A1DC090B530D090B6309C
:101DA000E090B730F090B830092F10E06DE8969FC2
:101DB000900111242856324ED9011396CD92DD920E
:101DC000ED92FC9216974115510569F0DA018C915C
:101DD000D901AA57BF4F8C93DA0111968C91D90182
:101DE000A957BF4F8C932097A1F029813DE8309FE0
:101DF000C001319F900D11248856924EDC01A657E8
:101E0000BF4F2C93119688818F708C9388818F702F
:101E10008C933097B9F186819DE8909F9001919FB6
:101E2000300D11242856324ED901A757BF4F8C933D
:101E3000858111978C93A90144575F4F83859485C1
:101E4000A585B685C92EDA2EEB2EFF24DA01CD92B8
:101E5000DC927901BEE8EB0EF11C238534854585C3
:101E60005685A4E6B0E00E94C287672F782F892F9D
:101E7000992724E630E040E050E00E945D87F701BA
:101E8000718360838DE8809FD001819FB00D112404
:101E9000A156B24EFE0132968FE701900D928A95BF
:101EA000E1F720919A1D2F5F20939A1D3091981D84
:101EB0003F5F3093981D8091891390918A13A09170
:101EC0008B13B0918C13A0FF2DC01F923F931F92D4
:101ED0002F938091991D1F928F938AE591E19F9393
:101EE0008F930E9438928DB79EB708960FB6F894DC
:101EF0009EBF0FBE8DBF16C08091C5309091C63079
:101F0000A091C730B091C8300196A11DB11D80933A
:101F1000C5309093C630A093C730B093C83080E0EE
:101F200090E002C081E090E0DF91CF911F910F918E
:101F3000FF90EF90DF90CF9008952091981D22237D
:101F400069F18091991D8F5F21502093981D64E164
:101F50000E942987392F9093991D80918913909120
:101F60008A13A0918B13B0918C13A0FF1AC01F92FB
:101F70002F9380919A1D1F928F931F923F9383E31B
:101F800091E19F938F930E9438928DB79EB70896E8
:101F90000FB6F8949EBF0FBE8DBF03C080E090E0E7
:101FA000089581E090E008958823B9F052985A98F6
:101FB0001DBA80916900806280936900EA9A539803
:101FC0005B98EB9A809169008068809369008091AA
:101FD00068008160809368000895109269005A9AA1
:101FE000EA985B9AEB9808951F920F920FB60F92A2
:101FF00011248F939F93AF93BF938091680080FFCC
:1020000024C080915E3590915F35A0916035B0918C
:1020100061350196A11DB11D80935E3590935F35AA
:10202000A0936035B09361358091891390918A13A4
:10203000A0918B13B0918C1387FF07C0749882E036
:1020400090E09093920280939102BF91AF919F9103
:102050008F910F900FBE0F901F9018951F920F92A7
:102060000FB60F9211248F939F93AF93BF938091DC
:10207000680080FF24C08091623590916335A09103
:102080006435B09165350196A11DB11D809362350F
:1020900090936335A0936435B0936535809189132F
:1020A00090918A13A0918B13B0918C1390FF07C06D
:1020B000739882E090E09093920280939102BF9196
:1020C000AF919F918F910F900FBE0F901F90189519
:1020D00080937C0080917B00877F80937B00809140
:1020E0007C00806C80937C0085E080937A008091F6
:1020F0007A00806880937A0080917B0087FFFCCF14
:1021000080917B0085FFFCCF80917A008064809372
:102110007A0080917A0086FDFCCF109279001092AF
:10212000780084E090E060E070E020917A00206424
:1021300020937A0020917A0026FDFCCF2091780030
:1021400030917900620F731F0197009771F7109219
:102150007C0080917A008F7780937A0076956795DE
:102160007695679580E090E00E94028B089580E06C
:102170000E9468102091890230918A0240918B025E
:1021800050918C020E94E68C21EE3AE744E95EE32E
:102190000E949B8908950F931F93CF93DF93CFE104
:1021A000D0E00BE51EE0C093510187EC90E00E9467
:1021B0003B0E8091510185FD0DC0C031D10521F04C
:1021C0002CF00B54110904C004EC19E0025311095E
:1021D0002197E9CFB80180E090E00E94028B20E0D7
:1021E00030E04AE754E40E94658ADF91CF911F9165
:1021F0000F910895CF93DF93EC0188819981009727
:1022000099F0863D914121F01982188283E011C036
:10221000623171F40E94CB106093B1307093B23090
:102220008093B3309093B43086ED91E199838883A5
:1022300081E0DF91CF91089580917B008860809349
:102240007B0089EC80937C0085E080937A0080910C
:102250007A00806880937A0080917B0087FFFCCFB2
:1022600080917B0085FFFCCF80917A008064809311
:102270007A0080917A0086FDFCCF80917A0080649C
:1022800080937A0080917A0086FDFCCF609178007F
:102290007091790080917A008F7780937A0080E046
:1022A00090E00E94028B27ED33EA40E95FE30E9451
:1022B000E68C26E636E648E853E40E949A890895BB
:1022C000BF92CF92DF92EF92FF920F931F93CF9323
:1022D000DF93CDB7DEB729970FB6F894DEBF0FBEF8
:1022E000CDBF6C01109283138FEF898703EF1CE140
:1022F000B12C7E0189E0E80EF11C89858823E9F183
:10230000E8E0BE16E1F1BE016F5F7F4FC7010E949A
:10231000B15D89858F3F11F08E3F19F4809383134F
:102320002CC0CE010196C114D10471F40E94CA5D83
:1023300080938035FE013196A8E7B5E381918D93B6
:10234000EE15FF05D9F71DC00E94CA5DF801808314
:10235000FE01319620E030E0A801485051098191FA
:10236000DA01A20FB31F8C932F5F3F4F2830310546
:10237000B1F7B394075F1F4FC0CF8B2D03C088E028
:1023800001C081E029960FB6F894DEBF0FBECDBF25
:10239000DF91CF911F910F91FF90EF90DF90CF9041
:1023A000BF90089581E391E19F938F930E943892AB
:1023B0000F900F9008952F923F924F925F926F92DD
:1023C0007F928F929F92AF92BF92CF92DF92EF92C5
:1023D000FF920F931F93CF93DF93EC014B01009774
:1023E00011F427E004C08130910549F426E04AE267
:1023F00050E06BE270E089E290E00E94915CCE01D7
:102400000E9460119E012C573C4E5901D9018C93BA
:10241000CD2B69F0A3EFCA2EACE1DA2ECBEEDCE1D6
:10242000E12CF12CB2EE2B2EB0E13B2EA6C088E7BA
:1024300095E30E945D5EBC01882777FD8095982F0B
:102440000E94048B6B017C01892869F020E030E058
:1024500048EC52E40E94658A9F938F937F936F9319
:102460008FE191E1ACC0C8E7D5E30AE111E18991C0
:102470001F928F931F930F930E9438920F900F908B
:102480000F900F90B5E3C038DB0789F720E030E00C
:1024900048EC52E4C701B6010E94658A9F938F936E
:1024A0007F936F938AE091E19F938F930E9438927C
:1024B0000F900F900F900F900F900F90809180359C
:1024C000882319F088E193E002C08CE893E09F93A1
:1024D0008F9386E091E19F938F930E9438920F90A3
:1024E0000F900F900F9075C000E010E0FE01E00F1C
:1024F000F11F80811F928F93AEEEB0E1BF93AF9337
:102500000E9438920F5F1F4F0F900F900F900F9007
:102510000830110559F720E030E048EC52E4C301DF
:10252000B2010E94658A9F938F937F936F93A6EE6B
:10253000B0E1BF93AF930E9438920F900F900F902D
:102540000F900F900F90D6018C91882309F455C0FD
:1025500088E193E09F938F933F922F920E9438924D
:102560000E94D211BFEFEB1AFB0AE9E0CE0ED11C9C
:1025700029960F900F900F900F90D5018C9190E0BD
:10258000E816F906ECF5CE010E945D5EBC018827D5
:1025900077FD8095982F0E94048B2B013C018114BC
:1025A000910409F4A1CF20E030E048EC52E40E940D
:1025B000658A9F938F937F936F9383EF90E19F93AF
:1025C0008F930E9438920F900F900F900F900F9062
:1025D0000F90DF91CF911F910F91FF90EF90DF90BF
:1025E000CF90BF90AF909F908F907F906F905F90B3
:1025F0004F903F902F900C94D2118CE893E0AACF8B
:10260000DF91CF911F910F91FF90EF90DF90CF90CE
:10261000BF90AF909F908F907F906F905F904F9002
:102620003F902F900895CF93DF931F921F92CDB7C5
:10263000DEB780917935898380917F358A83CE0199
:1026400001960E944B730F900F90DF91CF910895E8
:10265000CF93DF93EC01209178353091793540911B
:102660007A3550917B3560917C3570917D358091C4
:102670007E3590917F35AFEF0E948E89E1F427E09F
:102680004AE250E06BE270E089E290E00E94915CE7
:1026900080E090E00E946011CC57DC4E888349E0D6
:1026A00050E06EE070E088E795E30E947193DF915F
:1026B000CF910C941313DF91CF9108951F920F9235
:1026C0000FB60F9211240BB60F92FF920F931F9328
:1026D0002F933F934F935F936F937F938F939F932A
:1026E000AF93BF93CF93DF93EF93FF9380918335A5
:1026F0008260809383358091660286FD2B9A80915B
:10270000660287FD2B9A8091910290919202181691
:10271000190614F4749A739A8091891390918A130C
:10272000A0918B13B0918C1385FF02C0749873989D
:10273000809106029091070201979093070280937F
:102740000602892B09F04BC180913E0A90913F0A05
:10275000019690933F0A80933E0A8091B530909104
:10276000B630A091B730B091B8300196A11DB11D1F
:102770008093B5309093B630A093B730B093B83013
:1027800080E190E0909307028093060280916602B8
:1027900080FD02C01D9B05C0109288131092871304
:1027A00006C081E090E09093881380938713809116
:1027B000891390918A13A0918B13B0918C1397FF7A
:1027C00008C08091871390918813892B49F0749ADF
:1027D0007398C2E9DCE10AEC10E3FF24F3941FC014
:1027E000739A7498F6CF80913E0A90913F0A0196B1
:1027F0000E943587892BC9F0688579856115710537
:1028000091F5688579856115710509F03FC02A96B3
:102810000B5F1F4FFCE1CA3BDF0709F44DC0688521
:1028200079856115710541F3DECF4A81417020E061
:1028300030E050E060E070E080E090E0A0E00E94D6
:102840008E89D1F277988091891390918A13A09103
:102850008B13B0918C1392FFCFCF74981092920289
:1028600010929102C9CF80913E0A90913F0A019641
:102870000E943587892B29F6F80114821382A8015A
:1028800062E184E292E00E94146FBBCF80913E0A25
:1028900090913F0A0E943587892B09F0B8CFF80143
:1028A000F082D283C18314821382A80162E182E4A0
:1028B00092E00E94146FABCF60916C0270916D0238
:1028C00061157105A1F180913E0A90913F0A0E9425
:1028D0003587892B61F580915E3590915F35A091A8
:1028E0006035B09161354091A7285091A82860913A
:1028F000A9287091AA28841B950BA60BB70B80936F
:10290000BA1C9093BB1CA093BC1CB093BD1C8091BF
:102910005E3590915F35A0916035B09161358093BF
:10292000A7289093A828A093A928B093AA286091DB
:102930006A0270916B0261157105A1F180913E0AE6
:1029400090913F0A0E943587892B61F5809162350D
:1029500090916335A0916435B09165354091AB2875
:102960005091AC286091AD287091AE28841B950BD6
:10297000A60BB70B8093BE1C9093BF1CA093C01CEA
:10298000B093C11C8091623590916335A0916435FC
:10299000B09165358093AB289093AC28A093AD2877
:1029A000B093AE288091660286FD2B9880916602D6
:1029B00090916702A0916802B091690291FF0FC0E7
:1029C0000E942F688A3119F0C1E0C80F01C0CBE026
:1029D0000E946F668C2F0E9447680E94386740E013
:1029E00050E060E085EB92E00E94146FFF91EF9160
:1029F000DF91CF91BF91AF919F918F917F916F9117
:102A00005F914F913F912F911F910F91FF900F90E8
:102A10000BBE0F900FBE0F901F9018958091E21C77
:102A20009091C930891B08950E940E15882371F07A
:102A3000E091C930EF73F0E0ED5CF24E808190E000
:102A40002091C9302F5F2093C93008958FEF9FEFF9
:102A50000895CF93DF93EC0110926F0A10926E0AE3
:102A6000888199810097B1F0843E934021F01982CA
:102A7000188283E0B6C0613109F0B2C00E9414151B
:102A8000992790936A0A8093690A8D3009F443C0AC
:102A90008F3F49F40E940E158111F0CF84EE93E030
:102AA000998388839DC08231910509F45AC08F377C
:102AB000910509F052C08091670A9091680A181632
:102AC00019060CF56091EA397091EB3988E090E0D5
:102AD0000E94F4916091EA397091EB3980E290E0C4
:102AE0000E94F4916091EA397091EB3988E090E0AE
:102AF0000E94F4918091670A9091680A01979093DF
:102B0000680A8093670A8091670A9091680A8F37F4
:102B1000910509F0BFCF1092C9301092E21C80914C
:102B2000670A9091680AFC01E252FF4C1082909370
:102B30006F0A80936E0A1092680A1092670A809159
:102B4000813590918235009709F4A4CF40E050E0A0
:102B5000609181130E94146F9DCF8830910571F5AB
:102B6000AACF6091EA397091EB398DE090E00E9434
:102B7000F4911092660A1092650A8091650A90910C
:102B8000660A2091670A3091680A821793070CF051
:102B9000BACFFC01E252FF4C80816091EA3970911A
:102BA000EB3990E00E94F4918091650A9091660A59
:102BB00001969093660A8093650ADFCF6091EA39A7
:102BC0007091EB390E94F4918091670A9091680AA4
:102BD0002091690AFC01E252FF4C208301968FCFBD
:102BE00081E0DF91CF9108958091871390918813B0
:102BF000892BD1F08091660290916702A0916802C2
:102C0000B091690293FD10C00E946F6683B7817F07
:102C1000866083BFF89483B7816083BF789488957A
:102C200083B78E7F83BF78940895CF93DF93EC01B1
:102C300088819981009749F08930924121F0198269
:102C4000188283E014C0653889F40E946E650E9482
:102C5000F41540E050E065E88091CB149091CC14DD
:102C60000E94146F89E092E19983888381E0DF916B
:102C7000CF910895CF93DF931F921F92CDB7DEB708
:102C8000892B81F05F934F938FED90E19F938F930A
:102C900069837A830E9438920F900F900F900F9063
:102CA0007A8169817F936F938CED90E19F938F93ED
:102CB0000E9438920F900F900F900F900F900F90EE
:102CC000DF91CF910895FF920F931F93CF93DF93DE
:102CD0000E946E6580EB0E94EA5E81111CC00E941A
:102CE0004E5F8091AF2C9091B02C81609093B02C6E
:102CF0008093AF2C81E293E09F938F938CED90E1D2
:102D00009F938F930E9438920F900F900F900F9087
:102D1000C1E0D0E002C0C0E0D0E0FEB08F2D8470F2
:102D2000F82E729A0E946E658EE40E94EA5E81110E
:102D300016C00E944E5F8091AF2C9091B02C8260A3
:102D40009093B02C8093AF2C8E010F5F1F4F43E107
:102D500059E069E273E0CE010E943A16E801F110F1
:102D600001C072980E946E658EEE0E94EA5E81112B
:102D700016C00E944E5F8091AF2C9091B02C846061
:102D80009093B02C8093AF2C8E010F5F1F4F43E1C7
:102D900059E061E373E0CE010E943A16E8010E9417
:102DA0006E6586EA0E94EA5E811116C00E944E5F3F
:102DB0008091AF2C9091B02C88609093B02C809330
:102DC000AF2C8E010F5F1F4F43E159E068E373E0C2
:102DD000CE010E943A16E8010E946E658CE30E94C3
:102DE000EA5E81111EC00E944E5F8091AF2C9091CF
:102DF000B02C80619093B02C8093AF2C8E010F5F2C
:102E00001F4F43E159E060E473E0CE010E943A169F
:102E100084ED90E19F938F930E9438920F900F90D2
:102E2000E8010E946E6582ED0E94EA5E811116C083
:102E30000E944E5F8091AF2C9091B02C8062909355
:102E4000B02C8093AF2C8E010F5F1F4F43E159E0F0
:102E500068E473E0CE010E943A16E8010E946E65B4
:102E600080E80E94EA5E811116C00E944E5F809148
:102E7000AF2C9091B02C91609093B02C8093AF2C9C
:102E80008E010F5F1F4F43E159E061E573E0CE0112
:102E90000E943A16E8010E946E6580ED0E94EA5E8B
:102EA000811116C00E944E5F8091AF2C9091B02C82
:102EB00080689093B02C8093AF2C8E010F5F1F4FD2
:102EC00043E159E067E573E0CE010E943A16E8015C
:102ED0000E946E658CEE0E94EA5E811116C00E940F
:102EE0004E5F8091AF2C9091B02C92609093B02C5B
:102EF0008093AF2C8E010F5F1F4F43E159E06FE5C8
:102F000073E0CE010E943A16E80107E010E00E944B
:102F10006E658CE70E94EA5E811113C00E944E5FCD
:102F20008091AF2C9091B02C80649093B02C8093C2
:102F3000AF2C43E159E066E673E0CE010E943A16F9
:102F400005C0015011090115110509F70E944E5FD6
:102F5000DF91CF911F910F91FF900C94D211CF93DD
:102F6000DF931F921F92CDB7DEB74A8369830E9419
:102F7000255F6981862F0E94565F4A81842F0E94B7
:102F8000565F0F900F90DF91CF910C944E5FAF92F0
:102F9000BF92DF92EF92FF920F931F93CF93DF9335
:102FA00000D0CDB7DEB7182FD22E4A835B8369835A
:102FB0000E94255F6981862F0E94565F812F816064
:102FC0000E944C5F4A81A42E5B81B52E00E010E088
:102FD000ED2CF12C81E0E81AF1080D1580F40E15A6
:102FE0001F0519F40E94715F02C00E94675FF5011E
:102FF00080830F5F1F4FFFEFAF1ABF0AEECF0F9016
:103000000F900F90DF91CF911F910F91FF90EF9054
:10301000DF90BF90AF900C944E5FAF92BF92CF9273
:10302000DF92EF92FF920F931F93CF93DF93CDB771
:10303000DEB760970FB6F894DEBF0FBECDBFB82ED7
:10304000A42E6623E9F18E010F5F1F4F80E1F80186
:1030500011928A95E9F728E0A80168E980EB0E94BF
:10306000C717BB2041F02FE633E03F932F930E9418
:1030700026920F900F906E01F8E0CF0ED11C96E7CC
:10308000E92E93E0F92EF80181918F011F928F9321
:10309000FF92EF920E9426920F900F900F900F9048
:1030A0000C151D0581F788851F928F932BEC33E05B
:1030B0003F932F930E9426920F900F900F900F90A6
:1030C000AA20E9F18E010F5F1F4F80E1F8011192F4
:1030D0008A95E9F720E1A80160E880EB0E94C71714
:1030E000BB2041F08BE793E09F938F930E94269241
:1030F0000F900F906E01F0E1CF0ED11C86E7E82E05
:1031000083E0F82EF80181918F011F928F93FF9237
:10311000EF920E9426920F900F900F900F900C1537
:103120001D0581F788891F928F938BEC93E09F9305
:103130008F930E9426920F900F900F900F906096A1
:103140000FB6F894DEBF0FBECDBFDF91CF911F91B8
:103150000F91FF90EF90DF90CF90BF90AF900895C8
:10316000CF93DF931F921F92CDB7DEB71A821982D9
:1031700022E0AE014F5F5F4F6AEA8EEE0E94C717F2
:10318000898190E0982F88272A81822B9093741D43
:103190008093731D22E0AE014F5F5F4F6CEA8EEEAD
:1031A0000E94C717898190E0982F88272A81822B57
:1031B0009093761D8093751D22E0AE014F5F5F4FA7
:1031C0006EEA8EEE0E94C717898190E0982F8827BB
:1031D0002A81822B9093781D8093771D22E0AE0187
:1031E0004F5F5F4F60EB8EEE0E94C717898190E0C2
:1031F000982F88272A81822B9093861D8093851D86
:1032000022E0AE014F5F5F4F62EB8EEE0E94C71768
:10321000898190E0982F88272A81822B9093881D9E
:103220008093871D22E0AE014F5F5F4F64EB8EEE0F
:103230000E94C717898190E0982F88272A81822BC6
:1032400090938A1D8093891D22E0AE014F5F5F4FEE
:1032500066EB8EEE0E94C717898190E0982F882731
:103260002A81822B90937A1D8093791D22E0AE01F2
:103270004F5F5F4F68EB8EEE0E94C717898190E029
:10328000982F88272A81822B90937C1D80937B1D09
:1032900022E0AE014F5F5F4F6AEB8EEE0E94C717D0
:1032A000898190E0982F88272A81822B9093801D16
:1032B00080937F1D22E0AE014F5F5F4F6CEB8EEE7F
:1032C0000E94C717898190E0982F88272A81822B36
:1032D0009093821D8093811D22E0AE014F5F5F4F6E
:1032E0006EEB8EEE0E94C717898190E0982F882799
:1032F0002A81822B9093841D8093831D0F900F90C1
:10330000DF91CF9108952F923F924F925F926F92EB
:103310007F928F929F92AF92BF92CF92DF92EF9265
:10332000FF920F931F93CF93DF93CDB7DEB76A97CA
:103330000FB6F894DEBF0FBECDBF182F488F298F70
:1033400019821A821B828091971D811107C06A8F92
:103350000E94B01881E08093971D6A8D662309F45E
:103360006CC04EE264EF8EEE0E94AF1769E07AE126
:1033700080E090E00E94C85E22E0AE014F5F5F4FA8
:1033800066EF8EEE0E94C7172981822F90E0A0E0A1
:10339000B0E02227382F492F5A2F8A81282B80917D
:1033A000891D90918A1D281B390B41095109A09153
:1033B000871DB091881D0E94C2876B017C018FE040
:1033C000F594E794D794C7948A95D1F76091811DBD
:1033D0007091821D882777FD8095982F2BE0660FCE
:1033E000771F881F991F2A95D1F72091831D30914F
:1033F000841D442737FD4095542F2C0D3D1D4E1D37
:103400005F1D0E947F87C20ED31ED0927E1DC09288
:103410007D1D88E0C80ED11C34E0D594C7943A9540
:10342000E1F7EE24D7FCE094FE2CC0928B1DD092E5
:103430008C1DE0928D1DF0928E1D012F0295000FC4
:10344000000F007C0C5CA12FB0E0BD8BAC8BA3E027
:10345000B0E0012E02C0AA0FBB1F0A94E2F725E3D9
:1034600035E00E94BB87DC01CB010296A11DB11D96
:103470008C879D87AE87BF8780E593ECA0E0B0E0A6
:1034800004C0B595A795979587951A95D2F7888B1F
:10349000998BAA8BBB8B10E0188619861A861B861F
:1034A000A8E02A2E312CAC89BD892A1A3B0A988DB6
:1034B000191709F436C1402F64EF8EEE0E94AF1742
:1034C0006C857D858E859F850E94C85E23E0AE0158
:1034D0004F5F5F4F66EF8EEE0E94C717E0917D1D34
:1034E000F0917E1DE05AFF409F01DF010E94A487FA
:1034F0006B017C018091751D9091761D9F8B8E8B49
:10350000A090731DB090741D2091771D3091781D8F
:103510000E94A4872B013C01ADE0759467945794F9
:103520004794AA95D1F7A091791DB0917A1DA70172
:1035300096018CE055954795379527958A95D1F753
:103540000E94CD87BB2797FDB095AB2F480E591E23
:103550006A1E7B1E92E0490E511C611C711C32E0F8
:1035600075946794579447943A95D1F7A0E85A0E0A
:10357000611C711CA091851DB091861DA301920153
:103580000E94C287DC01CB014FE0B695A7959795C5
:1035900087954A95D1F78C839D83AE83BF8329811C
:1035A0008A8190E0A0E0B0E04424582E692E7A2E63
:1035B000622A8B81482A022C04C075946794579420
:1035C00047940A94D2F74501AA2497FCA094BA2CF8
:1035D00062E0880C991CAA1CBB1C6A95D1F7A091CB
:1035E0007B1DB0917C1DA70196010E94CD876B01C8
:1035F0007C0177E1F594E794D794C7947A95D1F755
:103600002E893F89DF010E94A487EBE0959587957D
:1036100077956795EA95D1F7C60ED71EE81EF91E75
:103620008C0C9D1CAE1CBF1C0C8804C0880C991C03
:10363000AA1CBB1C0A94D2F792E0890E911CA11C13
:10364000B11CF2E0B594A79497948794FA95D1F7BA
:10365000481859086A087B08A3019201688979898A
:103660008A899B890E94198797FD0DC0660F771F75
:10367000881F991F2C813D814E815F810E945D874B
:1036800049015A010CC02C813D814E815F810E940D
:103690005D8749015A01880C991CAA1CBB1C9927FB
:1036A000B7FC9A958B2D7A2D692D9B01AC010E9458
:1036B00019879B01AC01AEEDBBE00E94C2876C0193
:1036C000FF24D7FCF094EF2CA3E4B3EEA501940102
:1036D0000E94D087BB2797FDB095AB2FC80ED91E8F
:1036E000EA1EFB1EAFECCA0EAEE0DA1EE11CF11CB6
:1036F00064E0F594E794D794C7946A95D1F7C80C21
:10370000D91CEA1CFB1C88859985AA85BB858C0D74
:103710009D1DAE1DBF1D88879987AA87BB871F5F28
:10372000C6CE112391F0212F30E040E050E06885B3
:1037300079858A859B850E945D8720938F1D3093B4
:10374000901D4093911D5093921DA98DAA2389F13C
:1037500060918F1D7091901D8091911D9091921D8F
:10376000611571058105910521F10E94048B20E806
:1037700036EE45EC57E40E94658A21E03EED42E4D6
:103780005EE30E94498D9B01AC0160E070E080E83F
:103790009FE30E949A892BE43AE34DEB57E30E94A2
:1037A000658A6093931D7093941D8093951D9093EB
:1037B000961D6A960FB6F894DEBF0FBECDBFDF919F
:1037C000CF911F910F91FF90EF90DF90CF90BF901E
:1037D000AF909F908F907F906F905F904F903F90B1
:1037E0002F9008950F931F93CF93DF9300D000D0B5
:1037F000CDB7DEB78E010F5F1F4F86E0F801119243
:103800008A95E9F78091891C811113C040E061E33A
:1038100086EA0E94AF174AE06CE286EA0E94AF1780
:1038200081E08093891C6CE77EE380E090E00E9459
:10383000C85E48E06DE286EA0E94AF176CE77EE35F
:1038400080E090E00E94C85E26E0A80162E386EA7C
:103850000E94C71747E06DE286EA0E94AF178A818F
:1038600090E0982F88272981822B9093841C809345
:10387000831C2C8130E0322F22274B81242B309364
:10388000861C2093851C4E8150E0542F44276D8167
:10389000462B5093881C4093871C5F934F933F9314
:1038A0002F939F938F938FE793E09F938F930E9423
:1038B00026920FB6F894DEBF0FBECDBF26960FB688
:1038C000F894DEBF0FBECDBFDF91CF911F910F9156
:1038D0000895CF92DF92EF92FF920F931F93CF93B1
:1038E000DF93CDB7DEB72A970FB6F894DEBF0FBED1
:1038F000CDBF8E010F5F1F4F86E0F80111928A95B0
:10390000E9F741E062E08CE30E94AF1748E560E030
:103910008CE30E94AF1762E174E380E090E00E94C4
:10392000C85E26E0A80163E08CE30E94C71743E06D
:1039300062E08CE30E94AF17098110E0102F00278E
:103940008A81082B1093641C0093631CEB80F12C7C
:10395000FE2CEE248C81E82AF092661CE092651C15
:10396000CD80D12CDC2CCC248E81C82AD092681C2E
:10397000C092671CB801882777FD8095982F0E9418
:10398000048B9B01AC01B701882777FD8095982FA8
:103990002F83388749875A870E94048B2F81388567
:1039A00049855A850E940E8A20EE3EE245E652E4A1
:1039B0000E94E68C20E030E044E353E40E949B89BF
:1039C0009F938F937F936F93DF92CF92FF92EF92AB
:1039D0001F930F938DE893E09F938F930E942692FD
:1039E0000FB6F894DEBF0FBECDBF2A960FB6F8947F
:1039F000DEBF0FBECDBFDF91CF911F910F91FF9022
:103A0000EF90DF90CF900895CF93DF93EC01888102
:103A10009981009759F1823F914121F019821882D2
:103A200083E071C08CE49AE00E94A56D892B51F16E
:103A30008091891390918A13A0918B13B0918C136C
:103A400093FD22C04091891350918A1360918B138A
:103A500070918C1354FD49C04091891350918A1381
:103A600060918B1370918C1355FD46C040E850E077
:103A700060E070E08CE49AE00E94876D82EF91E153
:103A80009983888381E03FC08091AF2C82FFDACF99
:103A900021E048E061E083E00E9483198091961D57
:103AA0008F938091951D8F938091941D8F9380911A
:103AB000931D8F938091921D8F938091911D8F9371
:103AC0008091901D8F9380918F1D8F9388E991E154
:103AD0009F938F930E9438928DB79EB70A960FB628
:103AE000F8949EBF0FBE8DBFADCF8091AF2C83FFEA
:103AF000B3CF0E94F21BB0CF8091AF2C84FFB6CF22
:103B00000E94691CB3CFDF91CF910895CF93C82F46
:103B10008CEE0E944C5F8C2F0E94565F65E375E02F
:103B200080E090E00E94C85E8DEE0E944C5F0E9493
:103B3000675FC82F0E94715F2C2F30E0322F222741
:103B4000A901482BCA01CF910895CF93DF93C82FC5
:103B50008CEE0E944C5F8C2F0E94565F62E174E3F2
:103B600080E090E00E94C85E8CEE0E944C5F80E096
:103B70000E94565F65E375E080E090E00E94C85EB9
:103B80008DEE0E944C5F0E94675FC82F0E94675FA6
:103B9000D82F0E94715F4D2F50E060E070E0762FCB
:103BA000652F542F44276C2B482BCB01BA01DF9192
:103BB000CF9108952F923F924F925F926F927F9292
:103BC0008F929F92AF92BF92CF92DF92EF92FF922D
:103BD0000F931F93CF93DF93CDB7DEB7CD54D109A9
:103BE0000FB6F894DEBF0FBECDBF80910402909156
:103BF0000502892BD1F110920502109204028CEE7D
:103C00000E944C5F8EE10E94565F6BE17EE480E093
:103C100090E00E94C85E82EA0E94861D90933D0A51
:103C200080933C0A84EA0E94861D90933B0A80930D
:103C30003A0A86EA0E94861D9093390A8093380AD0
:103C400088EA0E94861D9093370A8093360A8AEA92
:103C50000E94861D9093350A8093340A8CEA0E9454
:103C6000861D9093330A8093320A88E40E94A51D32
:103C70006FAB78AF89AF9AAF88E50E94A51D4B0165
:103C80005C018091340A9091350A20E030E040E0F8
:103C900050E0BA0126962FAF269727963FAF279779
:103CA00028964FAF289729965FAF29972A966FAF2E
:103CB0002A972B967FAF2B979C0140E050E060E065
:103CC00070E080E090E008E00E9430890E94E9887E
:103CD0003901B42FA52FF62FE72F8C019401A501F0
:103CE00060E070E080E090E05301CB2EDA2EEF2E02
:103CF000FE2E0E94678929833A832A011B014C0109
:103D0000B101C401315041095F4F6F4F7F4F8F4F59
:103D10009F4FA1E0B0E02596BFAFAEAF259721152C
:103D20003F4F4F4F5140610571058105910509F0E5
:103D300020F425961FAE1EAE259725966EAC7FAC5F
:103D400025978091320A9091330A5C01C12CD12CC5
:103D5000E12CF12C00E010E029813A81A201B101AF
:103D6000C4010E94D587D22EE32EF42E052F162FE4
:103D7000B72FF82FE92FA0E00E948E8984F42150FC
:103D8000310940485F4F6F4F7F4F8F4F9F4FD22E6B
:103D9000E32EF42E052F162FB72FF82FE92F2D2DF8
:103DA0003E2D4F2D502F612F7B2F8F2F9E2F07E100
:103DB0000E9449892B8F3C8F4D8F5E8F6F8F78A328
:103DC00089A39AA32053384F4F4F5F4F6F4F7F4FB8
:103DD0008F4F9F4F2B8B3C8B4D8B5E8B6F8B788FD8
:103DE000898F9A8F2056304F4F4F5F4F6F4F7F4FC5
:103DF0008F4F9F4F243D30434105510561057105AB
:103E00008105910541F038F025966EAC7FAC259781
:103E1000FFEF6F1A7F0A80913A0A90913B0A9C014A
:103E200040E050E060E070E080E090E000E10E945F
:103E300030892B833C834D835E836A8779878F83A8
:103E400098874091360A5091370AA980BA8062015A
:103E5000710184019A0140E050E060E070E080E090
:103E600090E00E94D587D22EE32EF42E052F162F38
:103E7000B72FF82FE92FA0E00E948E895CF4AFE7FE
:103E80000E947089D22EE32EF42E052F162FB72F05
:103E9000F82FE92F2D2D3E2D4F2D502F612F7B2FE9
:103EA0008F2F9E2F07E00E94498959016A017B01EB
:103EB0008C012B813C814D815E816A8579858F8162
:103EC00098850E9467892B833C834D835E836F8333
:103ED00078878F87988B2E5F3F4F434051096E4FF5
:103EE0007F4F8F4F9F4F22303105494F5F4F6440C6
:103EF00071058105910521F018F01FEF611A710A13
:103F000080913C0A90913D0ABC0180E090E020E065
:103F100030E840E050E00E942E8829873A874B879E
:103F20005C876A8B798B8D879E874091380A509188
:103F3000390AA980BA806201710184019A0140E0C6
:103F400050E060E070E080E090E00E94D587D22EE3
:103F5000E32EF42E052F162FB72FF82FE92FA0E010
:103F60000E948E8984F421503F4F4F4F5F4F6F4F17
:103F70007F4F8F4F9F4FD22EE32EF42E052F162FFB
:103F8000B72FF82FE92F2D2D3E2D4F2D502F612FBC
:103F90007B2F8F2F9E2F08E00E94498959016A01CB
:103FA0007B018C0129853A854B855C856A897989F5
:103FB0008D859E850E94678929873A874B875C8714
:103FC0006D877E87898B9A8B2F5F3F4F41405109C8
:103FD0006109710981099109213030484C4F5F47CF
:103FE000614071058105910521F018F0BFEF6B1A52
:103FF0007B0A2B893C894D895E896F89788D898DF3
:104000009A8D2F3C374041055105610571058105A9
:10401000910511F00CF0A5C1A980BA80620171016F
:1040200084019501A201B101C4010E94D587A12C90
:10403000B12CC12C10E8D12EE12CF12C00E010E0C5
:104040000E945B882BAF3CAF4DAF5EAF6FAF219648
:104050007FAF219722968FAF229723969FAF23970A
:10406000AB8CBC8CCD8CDE8CEF8CF8A009A11AA196
:104070009501A601B701C8010E94D58759016A01BF
:104080007B01E82F192F02E00E9430890E2F0E9439
:10409000678969017A01162F272EF82FE92F322E12
:1040A0008D2C942EAF2CB62E072F582EB92FA0E0B2
:1040B0000E948E895CF4A1E00E947089322E832ECA
:1040C000942EA52EB62E072F582EB92F232D382D1E
:1040D000492D5A2D6B2D702F852D9B2F01E00E94AD
:1040E00049892E962FAF2E972D963FAF2D9749A732
:1040F0005AA76BA77CA78DA79EA7522E432E4BA332
:104100005CA36DA37EA38FA398A7B22D9601A701F0
:10411000612F722D8F2F9E2FA0E00E948E894CF46C
:10412000A3E00E94708969017A01162FB72FF82F3A
:10413000E92F9601A701612F7B2F8F2F9E2F02E081
:104140000E9449892FA738AB49AB5AAB6BAB7CAB0C
:104150008DAB9EAB19014A01B62FA72F24968FAFC6
:104160002497F92F2B893C894D895E896F89788D39
:10417000898D9A8D24323A4F4F4F5F4F6F4F7F4F4B
:104180008F4F9F4F0CF08CC02B8D3C8D4D8D5E8DD5
:104190006F8D78A189A19AA12455324F4F4F5F4F5F
:1041A0006F4F7F4F8F4F9F4F59016A017B018C01E9
:1041B0000E94D58719014A01B62FA72FFC0103E001
:1041C0000E94308951016401EB2EFA2E8F010E946A
:1041D0007C8959016A017B018C012E962FAD2E97A7
:1041E0002D963FAD2D9749A55AA56BA57CA58DA50C
:1041F0009EA50E946789522E432E4BA35CA36DA3FC
:104200007EA38FA398A79101A4016B2F7A2FCF01D2
:1042100002E00E94308951016401EB2EFA2E8F01D9
:104220000E947C8902E00E9430890E2F0E947C89C6
:10423000F22E032F142FD52EE62EB72FF82FE92FAD
:10424000A0E00E948E895CF4A1E00E947089F22EA9
:10425000032F142FD52EE62EB72FF82FE92F2F2D51
:10426000302F412F5D2D6E2D7B2F8F2F9E2F01E044
:104270000E94498959016A017B018C012FA538A947
:1042800049A95AA96BA97CA98DA99EA90E946789F1
:1042900019014A01B62FA72F24968FAF2497F92F23
:1042A0002B813C814D815E816F8178858F859889D6
:1042B000A52CB42CCBA0DCA0EDA0FEA00FA118A5CE
:1042C0000E947C892B833C834D835E836F83788738
:1042D0008F87988B29853A854B855C856D857E8592
:1042E00089899A8951016401EB2EFA2E24960FAD2B
:1042F00024971F2F0E947C8929873A874B875C87E8
:104300006D877E87898B9A8B2B893C894D895E8945
:104310006F89788D898D9A8DABACBCACCDACDEACA1
:10432000EFAC2196FFAC219722960FAD22972396F2
:104330001FAD23970E947C892056304F4F4F5F4F0F
:104340006F4F7F4F8F4F9F4F243D304341055105A5
:10435000610571058105910521F018F02FEF621AB2
:10436000720A6FA978AD89AD9AADAB01BC0180E04E
:1043700090E0DC0124964FAF249725965FAF2597F8
:1043800026966FAF269727967FAF279728968FAFF1
:10439000289729969FAF29972A96AFAF2A972B96F1
:1043A000BFAF2B97A984BA84CB84DC84ED84FE84D0
:1043B00009891A899A01AB0160E070E080E090E021
:1043C0000E94D587F22E032F142FD52EE62EB72F5D
:1043D000F82FE92FA0E00E948E8984F42150310942
:1043E000404E5F4F6F4F7F4F8F4F9F4FF22E032FE7
:1043F000142FD52EE62EB72FF82FE92F2F2D302F83
:10440000412F5D2D6E2D7B2F8F2F9E2F05E10E945A
:104410004989AB80BC80CD80DE80EF80F8840F8539
:1044200018890E947C89F22E032F142FD52EE62E98
:10443000B72FF82FE92FA0E00E948E8984F4215035
:1044400030484F4F5F4F6F4F7F4F8F4F9F4FF22E30
:10445000032F142FD52EE62EB72FF82FE92F2F2D4F
:10446000302F412F5D2D6E2D7B2F8F2F9E2F0FE034
:104470000E94498969017A018B018A839983290104
:104480001A014B015C01285E334041095109610961
:10449000710981099109283D304D4140510561055F
:1044A00071058105910521F018F0BFEF6B1A7B0AA9
:1044B0000E944E5F672859F09601A701B8018A81D2
:1044C00099810E94E98829011A014B015C0192013E
:1044D000A101B401C5010E94FE8A20E030E048EC51
:1044E00052E40E94658AC35BDF4F0FB6F894DEBFCB
:1044F0000FBECDBFDF91CF911F910F91FF90EF9035
:10450000DF90CF90BF90AF909F908F907F906F90F3
:104510005F904F903F902F9008954F925F926F92CF
:104520007F928F929F92AF92BF92CF92DF92EF9243
:10453000FF922B013C0169017A0123EC35EF4CE835
:1045400051E4C701B6010E94E68C4B015C0128EBE7
:104550003EE143E753E4C701B6010E949B899B01FA
:10456000AC01C501B4010E94658A0E94D28A4B0148
:104570005C0120E030E048EC52E4C301B2010E944B
:10458000658A21E835E943EC50E40E94E68CA501F8
:1045900094010E94E68C4B015C0123E333E948E877
:1045A00053E4C701B6010E949B899B01AC01C50180
:1045B000B4010E94658A23E333EB48E553E40E948B
:1045C000E68CFF90EF90DF90CF90BF90AF909F90E0
:1045D0008F907F906F905F904F9008954F925F9271
:1045E0006F927F928F929F92AF92BF92CF92DF9203
:1045F000EF92FF9269017A010E94688C20E030E01E
:1046000040E050E40E949A8922E93CE54EED5EE3E9
:104610000E94658A4B015C0123EC35EF4CE851E4C4
:10462000C701B6010E94E68C2B013C0128EB3EE15C
:1046300043E753E4C701B6010E949B899B01AC018B
:10464000C301B2010E94658A9B01AC01C501B4019E
:104650000E949B896B017C0128EB3EE143E753E418
:104660000E94E68C4B015C01A701960163EC75EF9B
:104670008CE891E40E949A899B01AC01C501B401C8
:104680000E94658AFF90EF90DF90CF90BF90AF902F
:104690009F908F907F906F905F904F9008954F9272
:1046A0005F926F927F928F929F92AF92BF92CF92C2
:1046B000DF92EF92FF922B013C0169017A0123EC1A
:1046C00035EF4CE851E4C701B6010E94E68C4B017E
:1046D0005C0128EB3EE143E753E4C701B6010E94C9
:1046E0009B899B01AC01C501B4010E94658A0E94AF
:1046F000D28A4B015C0120E030E048EC52E4C30177
:10470000B2010E94658AA50194010E94E68C20E016
:1047100030E040E251E40E949A8924EE38E34EE012
:104720005FE30E94E68C9B01AC01C701B6010E94C9
:104730009B89FF90EF90DF90CF90BF90AF909F90BC
:104740008F907F906F905F904F90089580E80E94C7
:104750004C5F81110DC08EEF0E94565F811108C021
:104760006BE17EE480E090E00E94C85E0C944E5FB6
:104770000E944E5F8091C1309091C230A091C330B1
:10478000B091C4300196A11DB11D8093C1309093AA
:10479000C230A093C330B093C4300895FC01DC0153
:1047A00082E020E041E39D91292798E0322F330FEA
:1047B00027FF03C0232F242701C0232F9150B1F7D7
:1047C000815089F781E090E03281231711F080E079
:1047D00090E00895DF92EF92FF920F931F93CF9393
:1047E000DF930E94A62380E80E944C5F81116DC078
:1047F0008AEF0E94565F811168C08FE00E94565F69
:10480000811163C065E375E080E090E00E94C85EBE
:1048100081E80E944C5F811158C00E94675FC82FD9
:104820000E94675F0E94675FD82F0E94675F0E94A7
:10483000675F182F0E94675F0E94715F082F80E8F2
:104840000E944C5F811141C08CEF0E94565F811124
:104850003CC089EC0E94565F811137C065E375E06A
:1048600080E090E00E94C85E81E80E944C5F0E9458
:10487000675FE82E0E94675FD82E0E94675F0E94E4
:10488000675FF82E0E94715F1F92DF921F92EF9276
:104890001F920F931F921F931F92DF931F92CF932C
:1048A0001F928F931F92FF9282EA93E09F938F93C0
:1048B0000E9426920E944E5F8DB79EB742960FB619
:1048C000F8949EBF0FBE8DBF17C00E944E5F8091AF
:1048D000C1309091C230A091C330B091C4300196E4
:1048E000A11DB11D8093C1309093C230A093C330FD
:1048F000B093C4300E94A62320E030E040E050E0B6
:1049000060E070E080E090E0DF91CF911F910F9127
:10491000FF90EF90DF900895EF92FF920F931F9317
:10492000CF93DF9300D0CDB7DEB78C0180E80E9433
:104930004C5F811154C00115110551F085EE0E94A4
:10494000565F81114CC061E077E980E090E009C0DA
:1049500083EE0E94565F811142C069E97AEB81E0E3
:1049600090E00E94C85E81E80E944C5F811137C0D0
:104970000E94675FF82E89830E94675FE82E8A8312
:104980000E94715F8B830E944E5FCE0101960E9450
:10499000CE23892B21F16E2D70E07F296C7F80E082
:1049A00090E0012B69F00E94028B20E030E04AEF9A
:1049B0005AE30E94E68C20E030E040EC50E40CC06A
:1049C0000E94028B22E538EB4FE25BE30E94E68C0B
:1049D00026E636E64BE352E40E949A891BC00E9409
:1049E0004E5F8091C1309091C230A091C330B091A0
:1049F000C4300196A11DB11D8093C1309093C23087
:104A0000A093C330B093C4300E94A62360EF7FEF21
:104A100089E794E40F900F900F90DF91CF911F9151
:104A20000F91FF90EF9008950F931F93CF93DF9313
:104A3000729A8091660283FF08C08EE40E94EA5E4B
:104A4000811167C0C0E5D0E00AC0C0E5D0E087EEC4
:104A500093E00E943B0E21972097C9F7EECF87EE97
:104A600093E00E943B0E21972097C9F78FE40E94A4
:104A7000EA5E0E94675F082F0F730E94675F182F1E
:104A80000E94675FD82F0E94715FC82F0E944E5FFF
:104A90008091660283FF7298602F70E0762F662700
:104AA000610F711D80E090E00E94028B20E134E0F4
:104AB00048EC5BE30E94E68C6093A3287093A428E3
:104AC0008093A5289093A6286D2F70E0762F6627F7
:104AD0006C0F711D769567957695679580E090E0EF
:104AE0000E94028B24EA3CEF44E25CE30E94E68CE5
:104AF00020E030E040E252E40E949A8960938435DD
:104B000070938535809386359093873580E090E06B
:104B100002C081E090E0DF91CF911F910F91089545
:104B20007298729A8EE40E94EA5E80EA0E94565F52
:104B300080E00E94565F80E00E94565F8FE40E94F2
:104B4000EA5E0E94675F8EE40E94EA5E80E80E944F
:104B5000565F80E00E94565F80E00E94565F0E9490
:104B60004E5F80E090E0089587EC90E19F938F93F3
:104B70000E943892809180020F900F90882361F0FC
:104B80001F928F9384EC90E19F938F930E943892B1
:104B90000F900F900F900F9008958FE990E19F93E1
:104BA0008F930E94389287E790E19F938F930E94A2
:104BB000389280E590E19F938F930E94389285E12F
:104BC00090E19F938F930E94389289ED9FE09F938D
:104BD0008F930E94389287EA9FE09F938F930E9461
:104BE00038928BE69FE09F938F930E94389285E4E2
:104BF0009FE09F938F930E9438928FE09FE09F9356
:104C00008F930E9438928091AF2C9091B02C82703B
:104C100091702DB73EB72E5E3F4F0FB6F8943EBF52
:104C20000FBE2DBF892B41F08FED9EE09F938F9398
:104C30000E9438920F900F9083EB9EE09F938F938A
:104C40000E94389287E79EE09F938F930E9438924C
:104C50008EE49EE09F938F930E94389282E29EE0C2
:104C60009F938F930E94389283EF9DE09F938F9341
:104C70000E94389281EC9DE09F938F930E9438921E
:104C800080E99DE09F938F930E94389286E59DE096
:104C90009F938F930E94389280E29DE09F938F9321
:104CA0000E94389280EF9CE09F938F930E943892ED
:104CB00084EC9CE09F938F930E94389285E99CE05E
:104CC0009F938F930E9438928CE59CE09F938F93E3
:104CD0000E94389283E29CE09F938F930E943892C7
:104CE0008CEE9BE09F938F930E9438928EEB9BE01B
:104CF0009F938F930E9438928DB79EB780960FB680
:104D0000F8949EBF0FBE8DBF8AE89BE09F938F9360
:104D10000E94389289E59BE09F938F930E9438927E
:104D20008AE29BE09F938F930E9438928BEF9AE0E8
:104D30009F938F930E94389284ED9AE09F938F9374
:104D40000E9438928EE99AE09F938F930E94389246
:104D500088E69AE09F938F930E94389282E39AE0CC
:104D60009F938F930E94389289E09AE09F938F934C
:104D70000E94389281ED99E09F938F930E94389220
:104D800086EA99E09F938F930E9438922DB73EB7A1
:104D90002A5E3F4F0FB6F8943EBF0FBE2DBF089559
:104DA00081ED93E00C945C924F925F926F927F92B0
:104DB0008F929F92AF92BF92CF92DF92EF92FF922B
:104DC000CF93DF93CDB7DEB728970FB6F894DEBF49
:104DD0000FBECDBF8091B5309091B630A091B73065
:104DE000B091B83089839A83AB83BC834090B5304F
:104DF0005090B6306090B7307090B8308091B53038
:104E00009091B630A091B730B091B8308D839E8329
:104E1000AF83B8876091B5307091B6308091B7306C
:104E20009091B8302CE3822E912CA12CB12CA501AD
:104E300094010E945D877F936F9330E1C32E3EE023
:104E4000D32EE12CF12C6D817E818F819885A70175
:104E500096010E945D87A50194010E945D873F93A2
:104E60002F9340E8842E41E5942EAA24A394B12CDC
:104E7000C301B201A50194010E945D87A7019601BB
:104E80000E945D873F932F9369817A818B819C81FA
:104E9000A50194010E945D873F932F9380E899E0DC
:104EA0009F938F930E9438920FB6F894DEBF0FBE87
:104EB000CDBF28960FB6F894DEBF0FBECDBFDF91F1
:104EC000CF91FF90EF90DF90CF90BF90AF909F90E9
:104ED0008F907F906F905F904F900895E0EFF9E38F
:104EE000808191818234924479F0E05FF943FF93AD
:104EF000EF9382E699E09F938F930E9438920F90F0
:104F00000F900F900F9008953A96E53F81E8F807CB
:104F100038F30895CF93DF93EC018C9A0E94B71079
:104F20009F938F937F936F9386E599E09F938F93E1
:104F30000E9438920F900F900F900F900F900F904B
:104F4000209719F00E94D21108C084E599E09F9340
:104F50008F930E9438920F900F9081E00E9468100A
:104F600020918502309186024091870250918802FB
:104F70000E94E68C9F938F937F936F9388E499E0D0
:104F80009F938F930E9438920F900F900F900F90E5
:104F90000F900F90209719F00E94D21108C086E45C
:104FA00099E09F938F930E9438920F900F9082E028
:104FB0000E94681020918102309182024091830208
:104FC000509184020E94E68C9F938F937F936F93FE
:104FD0008AE399E09F938F930E9438920F900F90ED
:104FE0000F900F900F900F90209719F00E94D21100
:104FF00008C088E399E09F938F930E9438920F90A6
:105000000F9083E00E9468109F938F937F936F931C
:1050100089E299E09F938F930E9438928C980F9029
:105020000F900F900F900F900F90209719F00E9403
:10503000D21108C087E299E09F938F930E94389223
:105040000F900F908091AF2C87FF83C021E042E149
:1050500061E080ED0E94AE609F938F937F936F938A
:105060008AE199E09F938F930E9438920F900F905E
:105070000F900F900F900F90209719F00E94D2116F
:1050800008C088E199E09F938F930E9438920F9017
:105090000F9021E042E162E080ED0E94AE609F93BC
:1050A0008F937F936F938BE099E09F938F930E94F0
:1050B00038920F900F900F900F900F900F902097B5
:1050C00019F00E94D21108C089E099E09F938F9354
:1050D0000E9438920F900F9021E042E163E080ED52
:1050E0000E94AE609F938F937F936F938CEF98E0B5
:1050F0009F938F930E9438920F900F900F900F9074
:105100000F900F90CD2B19F00E94D21108C08AEF9A
:1051100098E09F938F930E9438920F900F9021E018
:1051200042E164E080ED0E94AE609F938F937F9395
:105130006F938DEE98E09F938F930E9438920F901B
:105140000F900F900F900F900F90DF91CF910C94D4
:10515000D211CD2BD1F3DF91CF9108950F931F93EF
:10516000CF93DF93882389F049E050E06FEF70E040
:1051700088E795E30E947A9149E050E06EE070E0A4
:1051800088E795E30E94719313C0C8E7D5E308EE62
:1051900018E089911F928F931F930F930E9438926A
:1051A0000F900F900F900F9085E3C038D80789F7C4
:1051B000DF91CF911F910F910C94D211882311F0A0
:1051C000299A089529980895882311F02A9A089514
:1051D0002A980895CF93DF9360917E0270917F02A9
:1051E00080E090E00E946091EC016EE074E00E942B
:1051F0008191892B99F48091660290916702A09128
:105200006802B0916902A46080936602909367027D
:10521000A0936802B09369022A9A1BC061E174E00E
:10522000CE010E948191892BF1F4809166029091C8
:105230006702A0916802B0916902AB7F8093660219
:1052400090936702A0936802B093690280E00E9485
:10525000E42844E050E06EE170E086E692E0DF9101
:10526000CF910C9471932A9B03C08EE094E002C00E
:1052700081E194E09F938F938BE594E09F938F93CC
:105280000E9438920F900F900F900F90DF91CF9166
:105290000895CF92DF92EF92FF92CF93DF936B014D
:1052A0007C0160FF11C085E194E09F938F938CEDAA
:1052B00090E19F938F930E9438920F900F900F90E0
:1052C0000F9081E090E002C080E090E0C1FE09C054
:1052D000EC01219643E159E06AE174E00E943A163C
:1052E000CE01C2FE09C0EC01219643E159E062E221
:1052F00074E00E943A16CE01C3FE09C0EC0121966B
:1053000043E159E06AE274E00E943A16CE01C4FE1D
:1053100009C0EC01219643E159E06EE875E00E9476
:105320003A16CE01C5FE09C0EC01219643E159E0D1
:105330006EE274E00E943A16CE01C6FE09C0EC018E
:10534000219643E159E062E374E00E943A16CE01EF
:10535000C7FE09C0EC01219643E159E068E374E01F
:105360000E943A16CE01D0FE09C0EC01219643E11D
:1053700059E060E474E00E943A16CE01D1FE09C003
:10538000EC01219643E159E068E474E00E943A168A
:10539000CE01D2FE09C0EC01219643E159E06CE454
:1053A00074E00E943A16CE012091AF2C3091B02CBF
:1053B00024703270232B59F0D3FE09C0EC012196E2
:1053C00043E159E062E574E00E943A16CE01209173
:1053D000AF2C23FF0BC0D4FE09C0EC01219643E1A2
:1053E00059E067E574E00E943A16CE012091AF2C97
:1053F00024FF0BC0D5FE09C0EC01219643E159E022
:105400006DE574E00E943A16CE01D6FE09C0EC01AB
:10541000219643E159E065E674E00E943A16CE0118
:10542000D7FE09C0EC01219643E159E060E774E042
:105430000E943A16CE01E0FE0CC043E159E061E85B
:1054400074E0DF91CF91FF90EF90DF90CF900C94BC
:105450003A16CD28CE28CF2841F483EE98E09F93CA
:105460008F930E9438920F900F90DF91CF91FF9011
:10547000EF90DF90CF900895CF92DF92EF92FF925E
:10548000CF93DF93EC01C12CD12C7601209709F446
:10549000A3C06EED78E0CE010E944C91892B11F4EF
:1054A0006894C0F866ED78E0CE010E944C91892B9B
:1054B00011F46894C1F86EEC78E0CE010E944C9132
:1054C000892B11F46894C2F86AEC78E0CE010E944E
:1054D0004C91892B11F46894C3F867EC78E0CE0105
:1054E0000E944C91892B11F46894C4F863EC78E025
:1054F000CE010E944C91892B11F46894C5F86DEB94
:1055000078E0CE010E944C91892B11F46894C6F882
:1055100065EB78E0CE010E944C91892B11F46894E0
:10552000C7F86DEA78E0CE010E944C91892B11F406
:105530006894D0F869EA78E0CE010E944C91892BFA
:1055400011F46894D1F863EA78E0CE010E944C919E
:10555000892B11F46894D2F86EE978E0CE010E94AC
:105560004C91892B11F46894D3F868E978E0CE0166
:105570000E944C91892B11F46894D4F860E978E08A
:10558000CE010E944C91892B11F46894D5F865E8FE
:1055900078E0CE010E944C91892B11F46894D6F8E2
:1055A00064E778E0CE010E944C91892B11F4689455
:1055B000D7F86FE678E0CE010E944C91892B11F468
:1055C0006894E0F860917E0270917F0280E090E044
:1055D0000E946091EC015ACFC701B601DF91CF91D3
:1055E000FF90EF90DF90CF900895AF92BF92CF924F
:1055F000DF92EF92FF920F931F93CF93DF93F22EE0
:10560000032F142FE52ED62EA72EB82EC92E2170CB
:1056100030E040E050E060E070E080E090E0A0E04A
:105620000E948E8989F0E6E8F4E0FF93EF93ECEDB9
:10563000F0E1FF93EF930E9438920F900F900F903C
:105640000F90E1E0F0E002C0E0E0F0E08091AF2CEC
:1056500080FF17C02F2D247030E040E050E060E064
:1056600070E080E090E0A0E00E948E8951F0EF01B0
:10567000219643E159E06AE874E0CF010E943A16AE
:10568000FE012F2D227030E040E050E060E070E03D
:1056900080E090E0A0E00E948E8951F0EF01219619
:1056A00043E159E06EE874E0CF010E943A16FE0132
:1056B0002F2D287030E040E050E060E070E080E0A6
:1056C00090E0A0E00E948E8951F0EF01219643E125
:1056D00059E066EA74E0CF010E943A16FE012F2DD0
:1056E000207130E040E050E060E070E080E090E069
:1056F000A0E00E948E8951F0EF01219643E159E02C
:1057000061E974E0CF010E943A16FE012F2D20724C
:1057100030E040E050E060E070E080E090E0A0E049
:105720000E948E8951F0EF01219643E159E064E92E
:1057300074E0CF010E943A16FE012F2D207430E054
:1057400040E050E060E070E080E090E0A0E00E9487
:105750008E8951F0EF01219643E159E06AE974E046
:10576000CF010E943A16FE012F2D207830E040E054
:1057700050E060E070E080E090E0A0E00E948E8960
:1057800051F0EF01219643E159E060EA74E0CF0166
:105790000E943A16FE0120E0302F317040E050E0C8
:1057A00060E070E080E090E0A0E00E948E8951F01F
:1057B000EF01219643E159E063EA74E0CF010E94D2
:1057C0003A16FE0120E0302F327040E050E060E0F9
:1057D00070E080E090E0A0E00E948E8951F0EF013F
:1057E000219643E159E068EA74E0CF010E943A163D
:1057F000FE0120E0302F347040E050E060E070E0C7
:1058000080E090E0A0E00E948E8951F0EF012196A7
:1058100043E159E06FEA74E0CF010E943A16FE01BD
:1058200020E0302F387040E050E060E070E080E031
:1058300090E0A0E00E948E8951F0EF01219643E1B3
:1058400059E062EB74E0CF010E943A16FE0120E0BD
:10585000302F307140E050E060E070E080E090E098
:10586000A0E00E948E8951F0EF01219643E159E0BA
:1058700067EB74E0CF010E943A16FE0120E0302F62
:10588000307240E050E060E070E080E090E0A0E046
:105890000E948E8951F0EF01219643E159E06EEBB1
:1058A00074E0CF010E943A16FE0120E030E040E0B3
:1058B00050E06D2D647070E080E090E0A0E00E9408
:1058C0008E8951F0EF01219643E159E065EC74E0D7
:1058D000CF010E943A16FE018091AF2C81FF17C0C4
:1058E00020E0302F307440E050E060E070E080E075
:1058F00090E0A0E00E948E8951F0EF01219643E1F3
:1059000059E069EC74E0CF010E943A16FE018091E3
:10591000AF2C9091B02C90FF17C020E030E040E019
:105920005E2D507160E070E080E090E0A0E00E94A9
:105930008E8951F0EF01219643E159E06CEC74E05F
:10594000CF010E943A16FE018091AF2C9091B02CAD
:1059500090FF17C020E030E040E05E2D507260E024
:1059600070E080E090E0A0E00E948E8951F0EF01AD
:10597000219643E159E06FEC74E0CF010E943A16A2
:10598000FE018091AF2C9091B02C90FF17C020E0C9
:1059900030E040E05E2D507460E070E080E090E028
:1059A000A0E00E948E8951F0EF01219643E159E079
:1059B00065ED74E0CF010E943A16FE0120E0302F21
:1059C000307840E050E060E070E080E090E0A0E0FF
:1059D0000E948E8951F0EF01219643E159E060EE7B
:1059E00074E0CF010E943A16FE0120E030E0412F22
:1059F000417050E060E070E080E090E0A0E00E9444
:105A00008E8951F0EF01219643E159E065EE74E093
:105A1000CF010E943A16FE0120E030E0412F427093
:105A200050E060E070E080E090E0A0E00E948E89AD
:105A300051F0EF01219643E159E068EE74E0CF01A7
:105A40000E943A16FE0120E030E0412F447050E001
:105A500060E070E080E090E0A0E00E948E8951F06C
:105A6000EF01219643E159E06BEE74E0CF010E9413
:105A70003A16FE018091AF2C87FF17C020E030E07E
:105A8000412F487050E060E070E080E090E0A0E0DE
:105A90000E948E8951F0EF01219643E159E06EEEAC
:105AA00074E0CF010E943A16FE018091AF2C87FF6F
:105AB00017C020E030E0412F407150E060E070E01E
:105AC00080E090E0A0E00E948E8951F0EF012196E5
:105AD00043E159E062EF74E0CF010E943A16FE0103
:105AE0008091AF2C87FF17C020E030E0412F40723B
:105AF00050E060E070E080E090E0A0E00E948E89DD
:105B000051F0EF01219643E159E066EF74E0CF01D7
:105B10000E943A16FE018091AF2C87FF17C020E04B
:105B200030E0412F407450E060E070E080E090E0B1
:105B3000A0E00E948E8951F0EF01219643E159E0E7
:105B40006AEF74E0CF010E943A16FE018091AF2CFB
:105B500082FF17C020E030E0412F407850E060E045
:105B600070E080E090E0A0E00E948E8951F0EF01AB
:105B7000219643E159E061E276E0CF010E943A16B6
:105B8000FE018091AF2C82FF17C020E030E040E0A2
:105B90005E2D517060E070E080E090E0A0E00E9437
:105BA0008E8951F0EF01219643E159E06EEF74E0E8
:105BB000CF010E943A16FE018091AF2C9091B02C3B
:105BC00090FF17C020E030E040E05E2D527060E0B2
:105BD00070E080E090E0A0E00E948E8951F0EF013B
:105BE000219643E159E061E075E0CF010E943A1649
:105BF000FE018091AF2C9091B02C90FF17C020E057
:105C000030E040E05E2D547060E070E080E090E0B5
:105C1000A0E00E948E8951F0EF01219643E159E006
:105C200069E075E0CF010E943A16FE018091AF2C29
:105C30009091B02C91FF1EC020E030E040E05E2D3E
:105C4000587060E070E080E090E0A0E00E948E89F3
:105C500089F043E159E062E175E0CF01DF91CF9136
:105C60001F910F91FF90EF90DF90CF90BF90AF907A
:105C70000C943A162F2D302F412F5E2D6D2D7A2D3D
:105C80008B2D9C2DA0E00E948E8941F48AE698E03D
:105C90009F938F930E9438920F900F90DF91CF9136
:105CA0001F910F91FF90EF90DF90CF90BF90AF903A
:105CB00008958F929F92BF92DF92EF920F931F935E
:105CC000CF93DF93EC014B01FB01108265E678E096
:105CD0000E944C91892B61F58091AF2C7DE4D72EE9
:105CE000E0E8EE2E82FD02C004E001C004E810E00E
:105CF000B12C81FF02C060ECE62E26E04AE250E0C3
:105D00006BE270E089E290E00E94915C81E090E0BB
:105D10000E946011882311F05DE5D52E8091AF2C93
:105D20009091B02C90FD16E091FF07C0186005C05F
:105D3000D12CE12C00E010E0B12C63E678E0CE013C
:105D40000E944C91892B61F481E0F4018083609181
:105D50007E0270917F0280E090E00E946091EC01F1
:105D600061E678E0CE010E944C91892B61F48FEFBF
:105D7000F401808360917E0270917F0280E090E068
:105D80000E946091EC01209709F424C16DE578E050
:105D9000CE010E944C91892B19F4FD2DF160DF2E6C
:105DA00069E578E0CE010E944C91892B19F48D2D84
:105DB0008460D82E66E578E0CE010E944C91892B54
:105DC00019F4ED2DE260DE2E64E578E0CE010E944C
:105DD0004C91892B19F4FD2DF860DF2E61E578E0F8
:105DE000CE010E944C91892B19F48D2D8061D82E03
:105DF0006BE478E0CE010E944C91892B19F4ED2DD3
:105E0000E062DE2E65E478E0CE010E944C91892BA1
:105E100019F4FD2DF064DF2E62E478E0CE010E94DB
:105E20004C91892B19F48D2D8068D82E6DE378E084
:105E3000CE010E944C91892B19F4EE2DE160EE2EDB
:105E400066E378E0CE010E944C91892B19F4FE2D77
:105E5000F260EF2E63E378E0CE010E944C91892B33
:105E600019F48E2D8460E82E6EE278E0CE010E9457
:105E70004C91892B19F4EE2DE860EE2E67E278E064
:105E8000CE010E944C91892B19F4FE2DF061EF2E6A
:105E900060E278E0CE010E944C91892B19F48E2D9E
:105EA0008062E82E6CE178E0CE010E944C91892B53
:105EB00019F4EB2DE460BE2E69E178E0CE010E947A
:105EC0004C91892B19F4FE2DF064EF2E64E178E0FB
:105ED000CE010E944C91892B19F48E2D8068E82EFA
:105EE00061E178E0CE010E944C91892B09F40160B8
:105EF0006EE078E0CE010E944C91892B09F402609B
:105F00006BE078E0CE010E944C91892B09F404608B
:105F100067E078E0CE010E944C91892B09F408607B
:105F200063E078E0CE010E944C91892B09F4006176
:105F30006FEF77E0CE010E944C91892B09F400624B
:105F40006BEF77E0CE010E944C91892B09F400643D
:105F500069EF77E0CE010E944C91892B09F400682B
:105F600066EF77E0CE010E944C91892B09F4116015
:105F70006EEE77E0CE010E944C91892B09F41260FD
:105F800065EE77E0CE010E944C91892B09F41460F4
:105F90006CED77E0CE010E944C91892B09F41860DA
:105FA00069ED77E0CE010E944C91892B09F41061D4
:105FB00063ED77E0CE010E944C91892B09F41062C9
:105FC00068EC77E0CE010E944C91892B09F0D2CE8B
:105FD0001064D0CE2D2D3E2DA8016B2D70E080E0F9
:105FE00090E0DF91CF911F910F91EF90DF90BF90E4
:105FF0009F908F9008955F926F927F928F929F9261
:10600000AF92BF92CF92DF92EF92FF920F931F93C6
:10601000CF93DF93782EC2E9DCE100E010E0F2ECF0
:10602000EF2EF7E0FF2E8170582E872D8270682E9C
:10603000ADEACA2EA7E0DA2EB5EBAB2EB7E0BB2E49
:1060400083EB882E87E0982E772051F01F930F93D3
:10605000FF92EF920E9438920F900F900F900F9046
:106060005520A1F089858F9388858F93BF92AF9239
:106070000E9438920F900F900F900F906620C1F001
:106080009F928F920E9438920F900F90662081F01D
:10609000DF92CF920E943892288139814A815B81B8
:1060A0006C817D818E819F810E94F52A0F900F90D7
:1060B0000E94D2110F5F1F4F2A960430110521F65E
:1060C000DF91CF911F910F91FF90EF90DF90CF90D4
:1060D000BF90AF909F908F907F906F905F9008954A
:1060E00088EA97E09F938F930E94389280919F282F
:1060F0009091A028A091A128B091A2280F900F9074
:10610000813027EA92072EE1A207B10519F48AE946
:1061100097E01DC0823026EA92072EE1A207B10562
:1061200019F48DE897E013C0823027EA92072EE138
:10613000A207B10519F48FE797E009C0823028EA79
:1061400092072EE1A207B10549F481E797E09F93FA
:106150008F930E9438920F900F900895BF93AF9342
:106160009F938F938BE697E09F938F930E94389233
:106170000F900F900F900F900F900F9008958BE558
:1061800097E09F938F930E9438920E94D0260E949E
:1061900070300E94D21189E79CE19F938F9383E531
:1061A00097E09F938F930E94389260916002709164
:1061B0006102809162029091630228EE33E040E038
:1061C00050E00E945D875F934F933F932F9383E44A
:1061D00097E09F938F930E9438928AE397E09F9372
:1061E0008F930E9438920E9463168091AF2C2DB736
:1061F0003EB7225F3F4F0FB6F8943EBF0FBE2DBF94
:1062000080FF05C041E061E081E00E940D1886E357
:1062100097E09F938F930E94389280E00E94AE286F
:106220000E94D426809165021F928F938DE297E0A1
:106230009F938F930E943892809186131F928F9321
:1062400084E297E09F938F930E943892809190020E
:106250008F9380918F028F9380918E028F93809184
:106260008D028F9386E197E09F938F930E943892DF
:106270001F9280E48F938EEF96E09F938F930E94FE
:106280003892809197371F928F93809196371F9203
:106290008F938BEE96E09F938F930E94389280911C
:1062A00064021F928F9382EE96E09F938F930E94D9
:1062B00038928091660290916702A0916802B09135
:1062C00069022DB73EB7225E3F4F0FB6F8943EBF2E
:1062D0000FBE2DBF96FF03C08EE094E002C081E1A7
:1062E00094E09F938F9388ED96E09F938F930E9405
:1062F000389283E00E94FB2F0F900F900F900F9029
:106300001D9B03C08EE094E002C081E194E09F9366
:106310008F938CEC96E09F938F930E94389282EC3F
:1063200096E09F938F930E943892809166020F901F
:106330000F900F900F900F900F9081FF09C08CEB82
:1063400096E09F938F930E9438920F900F9013C006
:1063500080FF03C08EE094E002C081E194E09F934F
:106360008F9388EB96E09F938F930E9438920F90C3
:106370000F900F900F908091660290916702A0910C
:106380006802B091690297FF03C08EE094E002C0FA
:1063900081E194E09F938F938FEA96E09F938F9390
:1063A0000E94389288EA96E09F938F930E943892D9
:1063B0006091891370918A1380918B1390918C1343
:1063C0000E9449290E94D2110F900F900F900F90B8
:1063D0000F900F90779903C08EE094E002C081E1A6
:1063E00094E09F938F938FE996E09F938F930E9401
:1063F00038920E94410E0E941C119F938F937F93AD
:106400006F9381E996E09F938F930E9438920E9448
:10641000CB109F938F937F936F9383E896E09F9326
:106420008F930E94389281E090E00E948A278091A9
:106430005E3590915F35A0916035B0916135BF9325
:10644000AF939F938F9385E796E09F938F930E94DE
:106450003892809173358F93809172358F938091AC
:1064600071358F93809170358F9381E696E09F937D
:106470008F930E9438928091623590916335A091FC
:106480006435B0916535BF93AF939F938F9383E548
:1064900096E09F938F930E9438928DB79EB7829615
:1064A0000FB6F8949EBF0FBE8DBF809177358F9346
:1064B000809176358F93809175358F938091743567
:1064C0008F938FE396E09F938F930E94389261E0C1
:1064D00070E080E090E00E94DB1161E070E081E01C
:1064E00090E00E94DB110F900F900F900F900F9093
:1064F0000F90299B03C08EE094E002C081E194E0FC
:106500009F938F9387E396E09F938F930E94389297
:106510000F900F900F900F902A9B03C08EE094E095
:1065200002C081E194E09F938F938FE296E09F9366
:106530008F930E9438920F900F900F900F900895B4
:10654000F894E0E0F0E081E2809357008491E2E08B
:10655000F0E041E2409357004491E4E0F0E091E242
:1065600090935700E49190E0A0E0B0E0DC0199271F
:10657000882750E060E070E0762F652F542F442785
:10658000840F951FA61FB71F8E0F911DA11DB11D52
:1065900080939F289093A028A093A128B093A2282D
:1065A00078940895CF93DF93CDB7DEB761970FB698
:1065B000F894DEBF0FBECDBF48E250E062E270E06B
:1065C00082E99CE10E9453932091921C3091931C8C
:1065D0004091941C5091951C6091961C7091971C51
:1065E0008091981C9091991CAFEF0E948E8909F0C0
:1065F0005DC08DE48093921C80E88093931C84E0BE
:106600008093941C1092951C1092961C1092971CCB
:106610001092981C1092991C8CE390E090939B1C14
:1066200080939A1C10929C1C10929D1C10929E1C90
:1066300010929F1C1092A01C1092A11C1092A21CE0
:106640001092A31C1092A51C1092A41C1092A61CC0
:106650001092A71C1092A81C1092A91C1092AA1CA0
:106660001092AB1C1092AC1C1092AD1C1092AF1C7F
:106670001092AE1C1092B01C1092B11C1092B21C61
:106680001092B31C1092B41C1092B51C1092B61C40
:106690001092B71C1092B91C1092B81C48E250E03E
:1066A00062E270E082E99CE10E94719344E050E074
:1066B0006EE170E0CE010B960E9453938B859C8512
:1066C000AD85BE858F3F2FEF9207A207B207A9F4D1
:1066D0008AE090E4A0E0B0E08093660290936702C5
:1066E000A0936802B093690244E050E06EE170E06C
:1066F00086E692E00E94719308C0809366029093B0
:106700006702A0936802B09369028091660290913B
:106710006702A0916802B0916902A2FF02C02A9AA2
:1067200003C080E00E94E42844E050E06AE570E0A5
:10673000CE010B960E9453938B859C85AD85BE85BB
:106740008F3F2FEF9207A207B20789F410928913A7
:1067500010928A1310928B1310928C1344E050E025
:106760006AE570E089E893E10E94719308C0809324
:10677000891390938A13A0938B13B0938C1349E0E1
:1067800050E06EE070E088E795E30E9453930E942A
:10679000131344E050E06EE470E0CE010B960E94CB
:1067A00053938B859C85AD85BE8544E050E06EE4B7
:1067B00070E08F3F9F4FAF4FBF4F29F485E892E0C5
:1067C0000E94719304C085E892E00E94539344E0D4
:1067D00050E06AE470E0CE010B960E9453938B85E3
:1067E0009C85AD85BE8544E050E06AE470E08F3F53
:1067F0009F4FAF4FBF4F29F481E892E00E94719301
:1068000004C081E892E00E94539344E050E062E5C6
:1068100070E0CE010B960E9453938B859C85AD85CD
:10682000BE8544E050E062E570E08F3F9F4FAF4F80
:10683000BF4F29F489E892E00E94719304C089E86F
:1068400092E00E94539341E050E06DE170E0CE0190
:1068500041960E945393898941E050E06DE170E0D8
:106860008F3F29F486E893E10E94719304C086E883
:1068700093E10E94539341E050E06CE170E0CE015F
:1068800041960E945393898941E050E06CE170E0A9
:106890008F3F29F485E692E00E94719304C085E65B
:1068A00092E00E94539341E050E06BE170E0CE0132
:1068B00041960E945393898941E050E06BE170E07A
:1068C0008F3F29F484E692E00E94719304C084E62D
:1068D00092E00E9453934AE050E064E070E0CE0101
:1068E00001960E94539389814AE050E064E070E091
:1068F0008F3F29F489E79CE10E94719304C089E7E6
:106900009CE10E94539344E050E066E570E0CE01C4
:106910000B960E9453938B859C85AD85BE8544E084
:1069200050E066E570E08F3F9F4FAF4FBF4F29F4B7
:106930008DE892E00E94719304C08DE892E00E947D
:10694000539344E050E067E170E0CE010B960E9463
:1069500053938B859C85AD85BE8544E050E067E10F
:1069600070E08F3F9F4FAF4FBF4F29F480E692E01A
:106970000E94719304C080E692E00E94539342E02B
:1069800050E062E070E0CE010F960E9453938F8535
:10699000988942E050E062E070E08F3F910529F471
:1069A0008FE793E10E94719304C08FE793E10E9407
:1069B000539342E050E060E070E0CE010F960E94F9
:1069C00053938F85988942E050E060E070E08F3FFC
:1069D000910529F48DE793E10E94719304C08DE73E
:1069E00093E10E94539361960FB6F894DEBF0FBEF9
:1069F000CDBFDF91CF910895CF92DF92EF92FF92BA
:106A000060917E0270917F0280E090E00E94609130
:106A10006BE175E00E948191892B09F03BC18DE407
:106A20008093921C80E88093931C84E08093941C54
:106A30001092951C1092961C1092971C1092981C04
:106A40001092991C8CE390E090939B1C80939A1C6D
:106A500010929C1C10929D1C10929E1C10929F1CC8
:106A60001092A01C1092A11C1092A21C1092A31CA8
:106A70001092A51C1092A41C1092A61C1092A71C88
:106A80001092A81C1092A91C1092AA1C1092AB1C68
:106A90001092AC1C1092AD1C1092AF1C1092AE1C48
:106AA0001092B01C1092B11C1092B21C1092B31C28
:106AB0001092B41C1092B51C1092B61C1092B71C08
:106AC0001092B91C1092B81C48E250E062E270E0EB
:106AD00082E99CE10E9471938AE090E4A0E0B0E03A
:106AE0008093660290936702A0936802B093690254
:106AF00044E050E06EE170E086E692E00E9471931F
:106B00001092891310928A1310928B1310928C1387
:106B100044E050E06AE570E089E893E10E947193F7
:106B200042E2C42EDD24DA944CECE42E4BE3F42E46
:106B3000C0928502D0928602E0928702F09288028B
:106B400044E050E06EE470E085E892E00E947193CA
:106B5000C0928102D0928202E0928302F09284027B
:106B600044E050E06AE470E081E892E00E947193B2
:106B700087ED94E3AFEEBCE38093890290938A02A1
:106B8000A0938B02B0938C0244E050E062E570E089
:106B900089E892E00E9471938AE999E9A9E1B0E459
:106BA00080938D0290938E02A0938F02B0939002F7
:106BB00044E050E066E570E08DE892E00E94719359
:106BC0001092861380E00E94586941E050E06DE128
:106BD00070E086E893E10E9471938AE180936502F8
:106BE0000E94326841E050E06CE170E085E692E09E
:106BF0000E9471938FE08093640241E050E06BE16A
:106C000070E084E692E00E9471938AE0E9E7FCE19B
:106C1000DF011D928A95E9F74AE050E064E070E0F8
:106C2000CF010E94719380EA96E8A1E0B0E08093E2
:106C3000600290936102A0936202B093630244E009
:106C400050E067E170E080E692E00E94719310925C
:106C5000801310927F1342E050E062E070E08FE713
:106C600093E10E94719310927E1310927D1342E083
:106C700050E060E070E08DE793E10E94719381E065
:106C80000E94AE2880E090E0FF90EF90DF90CF90E0
:106C90000C942813FF90EF90DF90CF9008950E94FE
:106CA00056656C9A6B9A6A9A6F9A729A749A739AEA
:106CB000779A809880B3897F80BB8398849887E097
:106CC00080937E00549A0E94A0320E94D23281E0CA
:106CD0000E94D40F80E090E00E942813609160022F
:106CE0007091610280916202909163020E94D55E70
:106CF0000E94CB106093B1307093B2308093B33068
:106D00009093B4308091660286FD239A219A229A4C
:106D1000239A0E94AF0E1D9B05C0109288131092FB
:106D20008713089581E090E09093881380938713F0
:106D300008950F931F93CF93DF939DE8899FE00100
:106D40001124C556D24E4091891350918A136091F7
:106D50008B1370918C1341FD08C08091660280FDF9
:106D600004C081FF89C01D9B87C0CE0104969F93FC
:106D70008F9382E295E09F938F930E942692FE016B
:106D8000ED57FF4F80810F900F900F900F9008816B
:106D900019812A813B81882309F440C04091B53094
:106DA0005091B6306091B7307091B830401B510BA4
:106DB000620B730B7F936F935F934F933896918120
:106DC0009F9390819F93329791819F9390819F93FE
:106DD000339790811F929F93319790811F929F9339
:106DE000339690811F929F93319790811F929F932A
:106DF000CC57DF4F98811F929F931F928F9388E209
:106E000095E09F938F930E9426928DB79EB74696EA
:106E10000FB6F8949EBF0FBE8DBF1CC08091B530D9
:106E20009091B630A091B730B091B830801B910BE3
:106E3000A20BB30BBF93AF939F938F938FE695E015
:106E40009F938F930E9426920F900F900F900F9018
:106E50000F900F900E94D21180918002882361F0E0
:106E60001F928F9380EF92E09F938F930E943892AE
:106E70000F900F900F900F90DF91CF911F910F9176
:106E800008958091981D882341F08091991D90E08C
:106E90000E9499360E949D0FF4CF0895CF93DF93FF
:106EA000EC01888199818D3C2EE09207F1F018F475
:106EB000892BC1F04BC0853D2EE0920709F44CC0F0
:106EC000893D9E4009F042C080E49AE00E94A56D91
:106ED000892B09F43FC080E49AE00E94916D80E024
:106EE0000E94DE288DEC9EE02EC0623199F5299A31
:106EF00040917D1350917E135695542F44275795FA
:106F0000479560E070E080E49AE00E94876D4091D0
:106F1000891350918A1360918B1370918C1360FFC9
:106F200010C080917E138F9380917D138F9381E8A1
:106F300091E19F938F930E9438920F900F900F9042
:106F40000F9085ED9EE09983888304C01982188292
:106F500083E019C081E017C080E49AE00E94A56D2B
:106F6000892BC1F380E49AE00E94916D0E94413721
:106F700040E250E060E070E080E49AE00E94876DBB
:106F800089ED9EE0E0CFDF91CF9108952F923F925F
:106F90004F925F926F927F928F929F92AF92BF9229
:106FA000CF92DF92EF92FF920F931F93CF93DF93D5
:106FB000CDB7DEB72B970FB6F894DEBF0FBECDBFAF
:106FC0009B878A874A01FC0180819181892B11F07E
:106FD0000C945D4B60917E0270917F02CA010E9409
:106FE000609160E870E0C4010E94A091009759F49C
:106FF0006091EA397091EB398AE090E00E94F49157
:1070000081E00C94624B8130910561F4F401B08011
:107010001B2D110F110B012F412E512E612E712EA0
:10702000A12EBCC082309105B9F4F401808199276A
:1070300087FD9095982F88272181820F911D27FD2C
:107040009A95B82E192F092F000F000B402E502EA5
:10705000602E702EA02EA2C083309105B1F5F401F0
:107060002081922F990F990B392F492F592F692F72
:10707000792F892F00E10E94308919012A013B01F3
:10708000B82FA92F2181922F990F990B392F492FB2
:10709000592F692F792F892F08E00E9430895901D3
:1070A0006A017B018C019101A201B3018B2F9A2F00
:1070B0000E946789A2801A2D110F110BB12EC12ECB
:1070C000D12EE12EF12E012F55C004970CF45DC096
:1070D000F4012081922F990F990B392F492F592FA5
:1070E000692F792F892F08E10E94308919012A011F
:1070F0003B01B82FA92F2181922F990F990B392F7E
:10710000492F592F692F792F892F00E10E9430894B
:1071100059016A017B018C019101A201B3018B2FFE
:107120009A2F0E946789A3801A2D110F110BB12E7F
:10713000C12ED12EE12EF12E012F0E946789190157
:107140002A013B01B82FA92F2281922F990F990B69
:10715000392F492F592F692F792F892F08E00E9445
:10716000308959016A017B018C019101A201B301AF
:107170008B2F9A2F0E946789B22E132F042F452E32
:10718000562E672E782EA92E09C0FAE0BF2E10E0E9
:1071900000E0412C512C612C712CA12C0E94D211A9
:1071A0002B2D312F402F542D652D762D872D9A2D87
:1071B0002537F3E63F07FDE64F07510561057105E9
:1071C0008105910511F40C9448462537E3E63E0706
:1071D000EDE64E075105610571058105910511F038
:1071E00008F0BFC12337F2E73F07410551056105AC
:1071F00071058105910511F40C94DB482337E2E712
:107200003E0741055105610571058105910511F0A4
:1072100008F0BEC02536F4E63F074105510561057B
:1072200071058105910509F43AC72536E4E63E0764
:1072300041055105610571058105910511F008F0C1
:1072400042C0A6E70E948E8911F40C94D1420E949C
:107250008E8909F068F4A8E60E948E8909F470C747
:10726000A5E70E948E8911F40C94BB420C945B4BF1
:107270002B2D312F402F542D652D762D872D9A2DB6
:107280002436F1E63F074105510561057105810589
:10729000910511F40C9403492537E2E63E074105B8
:1072A0005105610571058105910509F499C42A33D9
:1072B000364241055105610571058105910509F4C5
:1072C0004EC30C945B4B2B2D312F402F542D652D2D
:1072D000762D872D9A2D2737EFE63E07410551057C
:1072E000610571058105910511F40C94AE462737AF
:1072F000FFE63F07410551056105710581059105CF
:1073000009F0C8F42436E9E63E0741055105610558
:1073100071058105910511F40C94944225363E4681
:1073200041055105610571058105910511F40C9424
:10733000E2460C945B4B2B2D312F402F542D652DA5
:10734000762D872D9A2D2536E2E73E07410551051A
:10735000610571058105910511F40C94AC4729363E
:10736000F2E73F074105510561057105810591056A
:1073700011F40C948A4823333147410551056105C6
:1073800071058105910511F00C945B4B0C94034938
:107390002B2D312F402F542D652D762D872D9A2D95
:1073A0002236F5E63F07F4E64F0751056105710502
:1073B0008105910509F473C62236E5E63E07E4E649
:1073C0004E075105610571058105910511F008F021
:1073D0005DC02133F4E63F07F1E64F075105610533
:1073E00071058105910509F4CEC22133E4E63E071B
:1073F000E1E64E075105610571058105910509F02A
:10740000C0F42337F3E73F074105510561057105D6
:107410008105910511F40C94EF4828373447410554
:107420005105610571058105910509F498C20C9417
:107430005B4B2B2D312F402F542D652D762D872D15
:107440009A2D2837F4E63F07F1E64F07510561050D
:1074500071058105910509F492C22C36E5E73E07D6
:10746000E2E64E075105610571058105910509F4B4
:10747000B7C3233634464146510561057105810580
:10748000910511F00C945B4B0C9403492B2D312F7B
:10749000402F542D652D762D872D9A2D2D36E5E71D
:1074A0003E07E8E64E075105610571058105910526
:1074B00011F40C9419492D36F5E73F07F8E64F070C
:1074C0005105610571058105910509F0E0F4223748
:1074D000E2E73E07E5E64E075105610571058105C6
:1074E000910511F40C94F94523363D464846510563
:1074F000610571058105910511F00C945B4B0E94AB
:10750000691C0C945D4B2B2D312F402F542D652D74
:10751000762D872D9A2D2436E3E63E07ECE64E07BE
:107520005105610571058105910511F40C945C45C7
:107530002736FFE63F07FCE64F0751056105710559
:107540008105910511F40C945F4523363243494679
:107550005105610571058105910511F00C945B4B96
:1075600032C22B2D312F402F542D652D762D872D96
:107570009A2D2037FCE63F07F5E64F07F8E65F0750
:10758000610571058105910509F4DAC52037ECE63E
:107590003E07E5E64E07E8E65E07610571058105F1
:1075A000910511F008F0E8C02437F8E73F07F4E749
:1075B0004F075105610571058105910511F40C9482
:1075C0003D432437E8E73E07E4E74E0751056105F0
:1075D00071058105910511F008F062C02033F1E3D7
:1075E0003F07F1E74F0751056105710581059105D9
:1075F00011F40C94F9452033E1E33E07E1E74E072F
:107600005105610571058105910509F0D8F4213313
:10761000F2E63F07F0E74F07510561057105810567
:10762000910509F4A8C2223332464047510561054D
:1076300071058105910511F00C945B4B0E94EA28BD
:107640000C945D4B2B2D312F402F542D652D762D15
:10765000872D9A2D2037F5E63F07F2E74F075105B2
:10766000610571058105910511F40C94AC472C3628
:10767000E4E73E074E075105610571058105910557
:1076800011F40C94844A213331434147510561057B
:1076900071058105910511F00C945B4B0C944846E3
:1076A0002B2D312F402F542D652D762D872D9A2D82
:1076B0002B36ECE63E07E5E74E07E2E65E0761059E
:1076C00071058105910509F48BC22B36FCE63F0755
:1076D000F5E74F07F2E65F07610571058105910542
:1076E00009F0E0F42437E4E63E07E7E74E075105EA
:1076F000610571058105910511F40C94D24A243776
:107700003F464F465246610571058105910511F0CE
:107710000C945B4B0C9400000C945D4B2B2D312F83
:10772000402F542D652D762D872D9A2D2E36E1E68E
:107730003E07E8E64E07E3E65E0761057105810551
:10774000910509F46EC72633F9E63F07F5E74F07C1
:10775000F5E65F07610571058105910509F4F4C43B
:1077600029363C4641465346610571058105910520
:1077700011F00C945B4BD1C22B2D312F402F542D87
:10778000652D762D872D9A2D2437F3E73F07F5E6F3
:107790004F07F2E75F07610571058105910511F457
:1077A0000C945C472437E3E73E07E5E64E07E2E743
:1077B0005E07610571058105910511F008F064C04F
:1077C0002337F5E63F07F2E74F07F0E75F0761056C
:1077D00071058105910511F40C94C9492337E5E63B
:1077E0003E07E2E74E07E0E75E07610571058105A8
:1077F000910509F0D0F42136FDE63F07F5E74F0784
:10780000F8E65F07610571058105910511F40C9497
:10781000CC462237374740475047610571058105FF
:10782000910509F4ACC10C945B4B2B2D312F402FEB
:10783000542D652D762D872D9A2D2436FDE63F0794
:10784000F3E64F07F2E75F076105710581059105D2
:1078500009F485C52136ECE63E07E5E64E07E2E78A
:107860005E07610571058105910509F48AC4233716
:10787000324747475047610571058105910511F071
:107880000C945B4B0C945F472B2D312F402F542DC4
:10789000652D762D872D9A2D2437E2E73E07E1E608
:1078A0004E07E5E75E07610571058105910509F45D
:1078B000B1C52437F2E73F07F1E64F07F5E75F0769
:1078C000610571058105910509F0C8F42437E3E7E6
:1078D0003E07E5E64E07E4E75E07610571058105B1
:1078E000910509F4F5C627373047484754476105E5
:1078F00071058105910509F46AC60C945B4B2B2D2B
:10790000312F402F542D652D762D872D9A2D2F3612
:10791000ECE63E07EFE54E07E6E75E076105710519
:107920008105910509F4C6C42C36F1E63F07F4E75A
:107930004F07F8E75F07610571058105910511F4AF
:107940000C94514A22373746404755476105710527
:107950008105910511F00C945B4B0C94374583E045
:1079600080936635109268351092673546E655E388
:1079700062E182E492E00E94146F0C945D4B0E94DD
:10798000F21B0C945D4B21E042E161E080ED0E942E
:10799000AE6021E042E161E080ED0E94AE6021E056
:1079A00042E161E080ED0E94AE6021E042E161E0F1
:1079B00080ED0E94AE6021E042E161E080ED0E9436
:1079C000AE600C945D4B60917E0270917F0280E00E
:1079D00090E00E9460916BE775E00E948191892B95
:1079E00009F0C5C060917E0270917F0280E090E056
:1079F0000E9460915C01009709F497C064E673E00F
:107A00000E948191892BE1F488EE93E0A0E0B0E040
:107A10008093600290936102A0936202B09363022C
:107A200068EE73E080E090E00E94D55E44E050E0B4
:107A300067E170E080E692E00E9471930C945D4BE8
:107A400061E875E0C5010E948191892BE1F480E134
:107A500097E2A0E0B0E08093600290936102A0936F
:107A60006202B093630260E177E280E090E00E94FE
:107A7000D55E44E050E067E170E080E692E00E946D
:107A800071930C945D4B64E875E0C5010E9481918F
:107A9000892BE1F480EA96E8A1E0B0E080936002EF
:107AA00090936102A0936202B093630260EA76E869
:107AB00081E090E00E94D55E44E050E067E170E034
:107AC00080E692E00E9471930C945D4B68E875E04B
:107AD000C5010E948191892BE1F480E89AE1A6E03A
:107AE000B0E08093600290936102A0936202B09331
:107AF000630260E87AE186E090E00E94D55E44E0AF
:107B000050E067E170E080E692E00E9471930C948F
:107B10005D4B87E694E09F938F930E9438920E947A
:107B2000D2110F900F900C945D4B60916002709198
:107B30006102809162029091630228EE33E040E09E
:107B400050E00E945D875F934F933F932F9383E6AE
:107B500094E09F938F930E9438920E94D2110F90CD
:107B60000F900F900F900F900F900C945D4B0E9410
:107B700063160C945D4B0E94EA280C945D4B609157
:107B80007E0270917F0280E090E00E9460918C0103
:107B90006EE074E00E948191892B19F477980C941F
:107BA0005D4B61E174E0C8010E948191892B19F459
:107BB000779A0C945D4B779903C08EE094E002C0F5
:107BC00081E194E09F938F9389E196E09F938F9357
:107BD0000E9438920F900F900F900F900C945D4B75
:107BE00060917E0270917F0280E090E00E9460913F
:107BF0008C016CE875E00E948191892BD1F4809111
:107C0000981D1F928F9380919A1D1F928F93809140
:107C1000991D1F928F931F9284E18F9381E394E0CB
:107C20009F938F930E9438920FB6F894DEBF0FBED9
:107C3000CDBF61E975E0C8010E948191892B19F4DB
:107C40000E94413766C069E975E0C8010E948191D0
:107C5000892BF1F560917E0270917F0280E090E0C7
:107C60000E946091009709F454C00E944E908531A3
:107C7000910528F59093801380937F1342E050E0A4
:107C800062E070E08FE793E10E94719360917E0261
:107C900070917F0280E090E00E9460910097C9F1AE
:107CA0000E944E9090937E1380937D1342E050E0AB
:107CB00060E070E08DE793E10E9471932AC08FE14C
:107CC00094E09F938F930E9438920F900F9021C061
:107CD000809180138F9380917F138F9386E194E03E
:107CE0009F938F930E9438920E94D21180917E13AD
:107CF0008F9380917D138F9387E094E09F938F9370
:107D00000E9438920E94D2110FB6F894DEBF0FBEC7
:107D1000CDBF0E94D2110C945D4B60917E02709198
:107D20007F0280E090E00E9460918C0165EE74E03B
:107D30000E948191892B09F077C060917E02709139
:107D40007F0280E090E00E9460918C01009711F426
:107D50000C945D4B67E975E00E948191892BB1F429
:107D600082E29FEFACECBBE38093850290938602A6
:107D7000A0938702B093880244E050E06EE470E084
:107D800085E892E00E9471930C945D4B6DE975E07B
:107D9000C8010E948191892BB1F482E29FEFACEC83
:107DA000BAE38093850290938602A0938702B093F2
:107DB000880244E050E06EE470E085E892E00E94C2
:107DC00071930C945D4BC8010E944A902B013C01B9
:107DD00020E030E0A9010E94618A8823D9F081E087
:107DE0000E9468109B01AC01C301B2010E94658A28
:107DF0006093850270938602809387029093880235
:107E000044E050E06EE470E085E892E00E947193F7
:107E10000C945D4B8AEF93E09F938F930E9438926E
:107E20000F900F900C945D4B68EE74E0C8010E94B7
:107E30008191892B09F077C060917E0270917F0259
:107E400080E090E00E9460918C01009711F40C9406
:107E50005D4B67E975E00E948191892BB1F482E264
:107E60009FEFACECBBE38093810290938202A093DE
:107E70008302B093840244E050E06AE470E081E859
:107E800092E00E9471930C945D4B6DE975E0C8011E
:107E90000E948191892BB1F482E29FEFACECBAE3AE
:107EA0008093810290938202A0938302B093840214
:107EB00044E050E06AE470E081E892E00E9471934F
:107EC0000C945D4BC8010E944A902B013C0120E0BC
:107ED00030E0A9010E94618A8823D9F082E00E94E3
:107EE00068109B01AC01C301B2010E94658A6093D6
:107EF000810270938202809383029093840244E013
:107F000050E06AE470E081E892E00E9471930C9482
:107F10005D4B8DEE93E09F938F930E9438920F906C
:107F20000F900C945D4B60EE74E0C8010E9481914B
:107F3000892B09F073C060917E0270917F0280E00E
:107F400090E00E9460918C01009711F40C945D4BBD
:107F500067E975E00E948191892BB1F487ED94E384
:107F6000AFEEBCE38093890290938A02A0938B02C8
:107F7000B0938C0244E050E062E570E089E892E062
:107F80000E9471930C945D4B6DE975E0C8010E94ED
:107F90008191892B51F48EED93E09F938F930E94F2
:107FA00038920F900F900C945D4BC8010E944A903C
:107FB0002B013C0120E030E0A9010E94618A882366
:107FC00019F180E00E9468104B015C0121EE3AE754
:107FD00044E95EE3C301B2010E949A89A5019401BC
:107FE0000E94658A6093890270938A0280938B0253
:107FF00090938C0244E050E062E570E089E892E002
:108000000E9471930C945D4B81ED93E09F938F934D
:108010000E9438920F900F900C945D4B0E94B71005
:108020009F938F937F936F938AEC93E09F938F93AB
:108030000E94389282E00E94681020918102309163
:10804000820240918302509184020E94E68C162F96
:10805000072FF82EE92E81E00E946810EF92FF9220
:108060000F931F93209185023091860240918702E1
:10807000509188020E94E68C9F938F937F936F9319
:108080008EEB93E09F938F930E9438920E94D211BF
:108090000FB6F894DEBF0FBECDBF0C945D4B609160
:1080A0007E0270917F0280E090E00E9460910097D4
:1080B00011F10E943C2A8090891390908A13A0901D
:1080C0008B13B0908C13681579058A059B0539F1DF
:1080D0006093891370938A1380938B1390938C13FE
:1080E00044E050E06AE570E089E893E10E94719312
:1080F00082E196E002C08BE096E09F938F930E940E
:1081000038926091891370918A1380918B139091AA
:108110008C130E9449290E94D2110F900F9080E089
:1081200096E09F938F930E9438926FEF7FEFCB0181
:108130000E9449290E94D2110F900F900C945D4B20
:108140000E94CD250C945D4BF4018481843329F485
:1081500040E061E080E00E940D1880918002882359
:1081600011F40C945D4B1F928F938DEF95E09F93CC
:108170008F930E9438920F900F900F900F900C9455
:108180005D4BF4018481893709F080C060917E02E3
:1081900070917F0280E090E00E9460918C016EE01F
:1081A00074E00E948191892B51F480916602909134
:1081B0006702A0916802B0916902906410C061E109
:1081C00074E0C8010E948191892BD1F480916602EC
:1081D00090916702A0916802B09169029F7B8093A1
:1081E000660290936702A0936802B093690244E02C
:1081F00050E06EE170E086E692E00E94719346C026
:1082000062EA75E0C8010E948191892B21F5809175
:10821000911C8F938091901C8F9380918F1C8F93D2
:1082200080918E1C8F9380918D1C8F9380918C1CDC
:108230008F9380918B1C8F9380918A1C8F9383E9FD
:1082400093E09F938F930E9438920FB6F894DEBF0D
:108250000FBECDBF1BC08091660290916702A091B6
:108260006802B091690296FF03C08EE094E002C0FC
:1082700081E194E09F938F938FE893E09F938F9396
:108280000E9438920F900F900F900F908091800273
:10829000882311F40C945D4B1F928F938AEF95E025
:1082A0009F938F930E9438920F900F900F900F9092
:1082B0000C945D4BF40184818737E9F560917E026F
:1082C00070917F0280E090E00E9460910097D9F069
:1082D0000E944A902B013C0120E030E0A9010E945D
:1082E000618A882381F040928D0250928E026092C2
:1082F0008F027092900244E050E066E570E08DE8F5
:1083000092E00E947193809190028F9380918F02EE
:108310008F9380918E028F9380918D028F9381E84D
:1083200093E09F938F930E9438920F900F900F903D
:108330000F900F900F9080918002882311F40C947D
:108340005D4B1F928F9387EF95E09F938F930E94D1
:1083500038920F900F900F900F900C945D4B60919E
:108360007E0270917F0280E090E00E9460918C011B
:108370006EE074E00E948191409066025090670226
:108380006090680270906902892B19F4689457F81C
:1083900009C061E174E0C8010E948191892B99F4C0
:1083A000E89457F840926602509267026092680221
:1083B0007092690244E050E06EE170E086E692E07F
:1083C0000E94719313C057FE03C08EE094E002C078
:1083D00081E194E09F938F938DE793E09F938F9338
:1083E0000E9438920F900F900F900F908091800212
:1083F000882311F40C945D4B1F928F9384EF95E0CA
:108400009F938F930E9438920F900F900F900F9030
:108410000C945D4B60917E0270917F0280E090E051
:108420000E9460915C0168EA75E00E948191892B4D
:1084300011F489E108C06CEA75E0C5010E948191E0
:10844000892B49F480E18093C4001092C50082E03A
:108450008093C00055C060EB75E0C5010E9481911A
:10846000892B11F488E0EFCF65EB75E0C5010E9420
:108470008191892B39F06AEB75E0C5010E948191E9
:10848000892B11F483E0DFCF8091C400893141F45E
:1084900088E793E09F938F930E9438920F900F90FC
:1084A0008091C400803141F483E793E09F938F93E0
:1084B0000E9438920F900F908091C400883041F450
:1084C0008DE693E09F938F930E9438920F900F90C8
:1084D0008091C400833041F487E693E09F938F93AB
:1084E0000E9438920F900F908091C400883041F420
:1084F00081E693E09F938F930E9438920F900F90A4
:1085000080918002882311F40C945D4B1F928F930D
:1085100081EF95E09F938F930E9438920F900F9078
:108520000F900F900C945D4B60917E0270917F02D2
:1085300080E090E00E94609167E975E00E9481917F
:10854000892B11F481E001C080E00E94AE28809167
:108550008002882311F40C945D4B1F928F938EEE52
:1085600095E09F938F930E9438920F900F900F90F9
:108570000F900C945D4B0E94D4268091800288233A
:1085800011F40C945D4B1F928F938BEE95E09F93AB
:108590008F930E9438920F900F900F900F900C9431
:1085A0005D4B0E94D02680918002882311F40C94A8
:1085B0005D4B1F928F9388EE95E09F938F930E945F
:1085C00038920F900F900F900F900C945D4B60912C
:1085D0007E0270917F0280E090E00E9460910E9494
:1085E0004E90803170F4809386130E94586941E068
:1085F00050E06DE170E086E893E10E9471930C9485
:108600005D4B809186131F928F9387E593E09F9334
:108610008F930E9438920F900F900F900F900C94B0
:108620005D4B60917E0270917F0280E090E00E943D
:1086300060910E944E9095EF980F903170F4809366
:1086400065020E94326841E050E06CE170E085E62E
:1086500092E00E9471930C945D4B809165021F9291
:108660008F938EE493E09F938F930E9438920F90A4
:108670000F900F900F900C945D4B60917E02709163
:108680007F0280E090E00E946091009789F04AE0CC
:1086900050E0BC0189E79CE10E9491914AE050E0E2
:1086A00064E070E089E79CE10E9471930C945D4B5B
:1086B00089E79CE19F938F938FEB95E09F938F9336
:1086C0000E9426920F900F900F900F900C945D4B8C
:1086D00060917E0270917F0280E090E00E94609144
:1086E0005C0164E673E00E948191892BD9F4219AA0
:1086F0008091660290916702A0916802B091690230
:1087000080618093660290936702A0936802B093A1
:10871000690244E050E06EE170E086E692E00E947B
:108720007193CBC769EE74E0C5010E948191892BDA
:10873000D9F4229A8091660290916702A091680212
:10874000B091690280628093660290936702A09361
:108750006802B093690244E050E06EE170E086E6A2
:1087600092E00E947193A9C766E473E0C5010E947C
:108770008191892BD9F4239A8091660290916702A6
:10878000A0916802B0916902806480936602909320
:108790006702A0936802B093690244E050E06EE182
:1087A00070E086E692E00E94719387C76CE874E0FF
:1087B000C5010E948191892BD9F4239A8091660288
:1087C00090916702A0916802B091690280688093DD
:1087D000660290936702A0936802B093690244E036
:1087E00050E06EE170E086E692E00E94719365C70A
:1087F0006EE373E0C5010E948191892B71F581E0E0
:108800008093CA3082E99CE19093CC308093CB3046
:108810001092CE301092CD30809166029091670216
:10882000A0916802B0916902916080936602909372
:108830006702A0936802B093690244E050E06EE1E1
:1088400070E086E692E00E9471934AEC50E362E1A8
:1088500082E492E00E94146F30C76DE673E0C501B8
:108860000E948191892B11F5E2ECFCE111921192A9
:108870002CE1E23EF207D1F7809166029091670207
:10888000A0916802B0916902926080936602909311
:108890006702A0936802B093690244E050E06EE181
:1088A00070E086E692E00E94719307C761E174E090
:1088B000C5010E94819140916602509167026091CA
:1088C000680270916902892BC1F44F705C7F4093FC
:1088D00066025093670260936802709369022B9A54
:1088E00044E050E06EE170E086E692E00E94719311
:1088F00080916F350E944768E0C644FF03C08EE058
:1089000094E002C081E194E09F938F9383E493E02D
:108910009F938F930E943892809166020F900F90E0
:108920000F900F9085FF03C08EE094E002C081E1BC
:1089300094E09F938F9388E393E09F938F930E949B
:108940003892809166020F900F900F900F9086FFE3
:1089500003C08EE094E002C081E194E09F938F9386
:108960008DE293E09F938F930E94389280916602EC
:108970000F900F900F900F9087FF03C08EE094E050
:1089800002C081E194E09F938F9382E293E09F93F2
:108990008F930E9438928091660290916702A09115
:1089A0006802B09169020F900F900F900F9090FFA6
:1089B00003C08EE094E002C081E194E09F938F9326
:1089C00087E193E09F938F930E9438928091660293
:1089D00090916702A0916802B09169020F900F9088
:1089E0000F900F9091FF03C08EE094E002C081E1F0
:1089F00094E09F938F938CE093E09F938F930E94DA
:108A000038928091660290916702A0916802B091BD
:108A100069020F900F900F900F9091FF4EC687EC58
:108A200095E00E945C9272ECA72E7CE1B72E0BE0E1
:108A300010E0EFEC8E2EE5E09E2EF5018081918115
:108A4000F2E0AF0EB11C9F938F931F930F939F92F1
:108A50008F920E9426920F5F1F4F0F900F900F90E2
:108A60000F900F900F900B31110539F726C684EE49
:108A700095E09F938F930E943892809180020F908F
:108A80000F90882361F01F928F9381EE95E09F9362
:108A90008F930E9438920F900F900F900F90F89440
:108AA00028E088E190E00FB6F894A89580936000E4
:108AB0000FBE20936000FFCF0E945F60FEC56091F3
:108AC0007E0270917F0280E090E00E9460918C01B4
:108AD0006EE074E00E948191892BE9F40E9438676E
:108AE0008091660290916702A0916802B09169023C
:108AF0008D7F81608093660290936702A0936802E5
:108B0000B093690244E050E06EE170E086E692E0E6
:108B10000E947193D2C561E174E0C8010E94819105
:108B2000892BE1F40E946F66809166029091670242
:108B3000A0916802B09169028C7F80936602909345
:108B40006702A0936802B093690244E050E06EE1CE
:108B500070E086E692E00E947193AFC56AED75E021
:108B6000C8010E948191892BE9F40E946F6680916F
:108B7000660290916702A0916802B09169028E7FAF
:108B800082608093660290936702A0936802B0931C
:108B9000690244E050E06EE170E086E692E00E94F7
:108BA00071938BC58091660281FF0FC08AED95E0BD
:108BB0009F938F9388E093E09F938F930E943892C6
:108BC0000F900F900F900F9078C580FF03C08EE03C
:108BD00094E002C081E194E09F938F9384E093E05E
:108BE0009F938F930E9438920F900F900F900F9049
:108BF00064C58091C8308F938091C7308F938091E6
:108C0000C6308F938091C5308F938091C4308F93FD
:108C10008091C3308F938091C2308F938091C13007
:108C20008F938091C0308F938091BF308F938091CC
:108C3000BE308F938091BD308F938091BC308F93E5
:108C40008091BB308F938091BA308F938091B930EF
:108C50008F9385EB95E09F938F930E9438920E94AB
:108C6000D211809180020FB6F894DEBF0FBECDBF47
:108C7000882309F422C51F928F9382EB95E09F937E
:108C80008F930E9438920F900F900F900F9015C500
:108C9000F89481E090E029E0FC0120935700C8950A
:108CA000E02C80E090E0FC0120935700C895F02C68
:108CB0007894F89483E090E0FC0120935700C895E5
:108CC000002D82E090E0FC0120935700C895102D04
:108CD00078948091A2288F938091A1288F9380917E
:108CE000A0288F9380919F288F9328EA35E03F93A7
:108CF0002F930E9438921F92EF921F92FF921F9221
:108D00000F931F921F9381E895E09F938F930E948A
:108D100038920E946E27809166001F928F9385E79C
:108D200095E09F938F930E9438920E94D211809178
:108D300080020FB6F894DEBF0FBECDBF882309F4C2
:108D4000BCC41F928F9382E795E09F938F930E94FC
:108D500038920F900F900F900F90AFC460E070E0CA
:108D600080E090E00E94DB1160E070E081E090E044
:108D70000E94DB1180918002882309F49EC41F9217
:108D80008F938FE695E09F938F930E9438920F9078
:108D90000F900F900F9091C40E9490250E94D211C5
:108DA00080918002882309F488C41F928F938CE6F7
:108DB00095E09F938F930E9438920F900F900F90A1
:108DC0000F907BC460917E0270917F0280E090E002
:108DD0000E94609161E975E00E948191892B31F5D3
:108DE000F8948BE79AE00E94EB6F5C01009769F0C2
:108DF000C5010F960E94556CB50188E092E00E9473
:108E00009870C5010E944C70F0CF8BE79AE00E94E9
:108E10003F70892B29F08BE79AE00E94FF6FF5CF16
:108E20008BE79AE00E94E76F789434C08BE79AE072
:108E30000E94EB6F5C010FED15E0A114B10451F13C
:108E4000F50186811F928F9380851F928F93858174
:108E50001F928F9381851F928F9387811F928F938B
:108E600084811F928F9383811F928F9382811F929F
:108E70008F9382851F928F931F930F930E94269248
:108E8000C5010E944C705C010FB6F894DEBF0FBEA6
:108E9000CDBFD3CF80918002882309F40EC41F92E6
:108EA0008F9389E695E09F938F930E9438920F905D
:108EB0000F900F900F9001C40E94FC34FEC360918C
:108EC0007E0270917F0280E090E00E9460918C01B0
:108ED0006EE176E00E948191892BD1F48091660247
:108EE00090916702A0916802B0916902977F809388
:108EF000660290936702A0936802B093690244E00F
:108F000050E06EE170E086E692E00E947193D5C376
:108F10006DE975E0C8010E948191892BD1F480919F
:108F2000660290916702A0916802B0916902986010
:108F30008093660290936702A0936802B0936902DF
:108F400044E050E06EE170E086E692E00E947193AA
:108F5000B4C30E94410EB1C360917E0270917F0242
:108F600080E090E00E946091FC0120812332B1F406
:108F70004AE050E060E070E001960E94028E1B0122
:108F800060917E0270917F0280E090E00E9460918B
:108F9000F4E02F1631040CF094C002C0212C312CC7
:108FA000009709F48EC01982BE016F5F7F4F0E9447
:108FB000592E29013A014B01B82FA92F8AE0829D31
:108FC000F001839DF00D1124EE56F34E20812A838B
:108FD00031813B8382818C8393819D8324812E8385
:108FE00035813F8386818887978199879201A30184
:108FF000B4018B2F9A2FAA80BB80CC80DD80EE80BD
:10900000FF80088519850E94858909F45DC08981E2
:10901000882351F18CF02A81422A3B81532A8C818A
:10902000682A9D81792A2E81822A3F81932A888508
:10903000B82B9985A92B18C04094509460947094D3
:1090400080949094B095A0952A8142223B8153222E
:109050008C8168229D8179222E8182223F819322F8
:109060008885B8239985A9234082518262827382C0
:1090700084829582B683A78348E250E062E270E082
:1090800082E99CE10E94719381E695E09F938F9322
:109090000E9438928AE0829DF001839DF00D112498
:1090A000EE56F34E20813181428153816481758176
:1090B000868197810E94F52A0E94D2110F900F900D
:1090C00003C082E00E94FB2F85E595E09F938F937C
:1090D0000E9438922FEF3FEF4FEF5FEF6FEF7FEF80
:1090E0008FEF9FEF0E94F52A0E94D211809180029B
:1090F0000F900F90882309F4E0C21F928F9382E5AE
:1091000095E09F938F930E9438920F900F900F904D
:109110000F90D3C260917E0270917F0280E090E058
:109120000E946091FC0120812332A1F44AE050E0CA
:1091300060E070E001960E94028E8B0160917E02D9
:1091400070917F0280E090E00E94609104301105F0
:10915000ECF402C000E010E00097C1F04AE050E0FB
:1091600060E070E00E94368F2AE0209FF001219F8E
:10917000F00D1124EE56F34E7187608748E250E0FF
:1091800062E270E082E99CE10E94719381E00E94BA
:10919000FB2F80918002882309F48FC21F928F9346
:1091A0008FE495E09F938F930E9438920F900F90D9
:1091B0000F900F9082C20E94DA7080918002882303
:1091C00009F47BC21F928F938CE495E09F938F9359
:1091D0000E9438920F900F900F900F906EC20E94D5
:1091E000BF3080918002882309F467C21F928F9359
:1091F00089E495E09F938F930E9438920F900F908F
:109200000F900F905AC280E090E00E948A278091D0
:109210008002882309F451C21F928F9386E495E05F
:109220009F938F930E9438920F900F900F900F9002
:1092300044C28091AF2C81FF2DC00E941425892B40
:1092400049F58091A6288F938091A5288F938091CE
:10925000A4288F938091A3288F938BE395E09F930D
:109260008F930E943892809187358F9380918635B5
:109270008F93809185358F93809184358F938EE283
:1092800095E09F938F930E9438920FB6F894DEBFBB
:109290000FBECDBF0E94D2118091AF2C9091B02C07
:1092A00090FF63C081E090E00E948C243B014C0160
:1092B00080E090E00E948C241B012C010E94EA2394
:1092C0009F928F927F926F928DE195E09F938F9303
:1092D0000E9438925F924F923F922F928DE095E0DC
:1092E0009F938F930E943892222D332D442D552D1C
:1092F000662D772D882D992D0E948D229F938F9317
:109300007F936F9382E095E09F938F930E943892B2
:10931000222D332D442D552D662D772D882D992DF9
:109320000E94EE229F938F937F936F9384EF94E03C
:109330009F938F930E943892222D332D442D552DCB
:10934000662D772D882D992D0E944F239F938F9303
:109350007F936F9381EE94E09F938F930E94389256
:109360000FB6F894DEBF0FBECDBF0E94D211809120
:109370008002882309F4A1C11F928F938EED94E09F
:109380009F938F930E9438920F900F900F900F90A1
:1093900094C18091AF2C82FF2BC021E048E061E0B6
:1093A00083E00E9483198091961D8F938091951D73
:1093B0008F938091941D8F938091931D8F938091B3
:1093C000921D8F938091911D8F938091901D8F930B
:1093D00080918F1D8F9387EC94E09F938F930E94D1
:1093E00038920E94D2110FB6F894DEBF0FBECDBFE7
:1093F0008091AF2C9091B02C91FF41C00E94DA1D5A
:10940000B62EA72E982E892E20E030E048EC52E4AC
:10941000D501F4016B2F7A2F8F2F9E2F0E94E68C9F
:1094200020E836EE45EC57E40E94658A21E03EEDE7
:1094300042E45EE30E94498D9B01AC0160E070E074
:1094400080E89FE30E949A892BE43AE34DEB57E3CF
:109450000E94658A9F938F937F936F938F929F92C1
:10946000AF92BF928EEA94E09F938F930E943892BE
:109470000E94D2110FB6F894DEBF0FBECDBF80910F
:109480008002882309F419C11F928F938BEA94E01C
:109490009F938F930E9438920F900F900F900F9090
:1094A0000CC160917E0270917F0280E090E00E948A
:1094B000609163E276E00E948191892B99F460913A
:1094C0007E0270917F0280E090E00E9460910097A0
:1094D00009F4F3C00E944E9090915201982B909302
:1094E0005201EBC0809152018F701F928F9387EFD2
:1094F00092E09F938F930E9438920E94D2110F9016
:109500000F900F900F90D9C060917E0270917F02F2
:1095100080E090E00E946091009711F14AE050E0F5
:1095200060E070E00E94028E603198F46093640203
:109530001F926F938EE994E09F938F930E943892CD
:1095400041E050E06BE170E084E692E00E947193AC
:1095500011C0809164021F928F9385E994E006C048
:10956000809164021F928F938CE894E09F938F9375
:109570000E9438920F900F900F900F900E94D2117E
:1095800080918002882309F498C01F928F9389E804
:1095900094E09F938F930E9438920F900F900F90BA
:1095A0000F908BC060917E0270917F0280E090E00E
:1095B0000E9460918C016EE074E00E948191892B81
:1095C000E1F40E9462658091660290916702A09129
:1095D0006802B0916902906180936602909367027D
:1095E000A0936802B093690244E050E06EE170E03D
:1095F00086E692E00E94719360C061E174E0C80168
:109600000E948191892B81F5F8940E94706588E110
:109610000FB6F89480936000109260000FBE84B77C
:10962000877F84BF80916000886180936000109282
:10963000600078948091660290916702A091680220
:10964000B09169029F7E8093660290936702A09317
:109650006802B093690244E050E06EE170E086E693
:1096600092E00E94719329C068E276E0C8010E94EE
:1096700081914091660250916702609168027091F9
:109680006902892B21F454FF18C0F894FFCF54FFCE
:1096900003C08EE094E002C081E194E09F938F9339
:1096A00083EF92E09F938F930E9438920F900F90D8
:1096B0000F900F9002C00E94B425EA85FB851182AD
:1096C000108283E02B960FB6F894DEBF0FBECDBF9D
:1096D000DF91CF911F910F91FF90EF90DF90CF908E
:1096E000BF90AF909F908F907F906F905F904F90C2
:1096F0003F902F900895CF93DF93EC01888199815B
:10970000009741F08B3C914109F48CC0198218827A
:1097100083E093C00E944F368091660280FD05C0B1
:1097200081FF01C01D9B0E946F66809170008C7F3D
:10973000809370008091B60080628093B600109292
:10974000B20082E08093B1008091B6008770E1F7AB
:10975000809170008160809370006FE57EE080E012
:1097600090E00E943F650E94D02680E00E94AE28D3
:109770008DEA91E19F938F930E9438920E94631625
:109780008091AF2C0F900F9086FD0E940B6080910E
:10979000AF2C9091B02C90FD0E94A6238091AF2C0D
:1097A00087FF06C021E04CE061E080ED0E94AE60E2
:1097B000809186130E945869809165020E943268E8
:1097C0000E942F6880936B0A809165020E94326824
:1097D000809186131F928F9380916B0A1F928F93B3
:1097E0008DE296E09F938F930E94269210926D0ACD
:1097F00010926C0A0F900F900F900F900F900F9097
:1098000086E592E0909382358093813583E290E003
:1098100090938213809381138BEC91E199838883D9
:1098200081E00BC06332E1F74EED50E360E070E0A1
:109830008CE69AE00E94C637E3CFDF91CF9108957E
:109840000F931F93CF93DF93EC018A018881998155
:10985000009711F1803E914121F01982188283E036
:1098600020C06231E9F4A80162E170E08CE69AE080
:109870000E94C63784E08093663510926835109256
:10988000673510936A350093693546E655E362E122
:1098900082E492E00E94146F80EE91E199838883C4
:1098A00081E0DF91CF911F910F910895843691054A
:1098B00014F19F938F9383E896E09F938F930E9478
:1098C00026928091B9309091BA30A091BB30B0917E
:1098D000BC300196A11DB11D8093B9309093BA3070
:1098E000A093BB30B093BC300F900F900F900F90AF
:1098F00081E090E0089580E090E008952F923F92FB
:109900004F925F926F927F928F929F92AF92BF928F
:10991000CF92DF92EF92FF920F931F93CF93DF933B
:10992000CDB7DEB7C859D1090FB6F894DEBF0FBE68
:10993000CDBFC057DF4F99838883C059D0408A017B
:10994000633871F480E79AE0C856DF4F6883C859DE
:10995000D0400E943B72C856DF4F6881C859D04042
:10996000C057DF4FA881B981C059D0402D913C919B
:109970002837B1E13B0711F40C94BA5940F4211592
:10998000310581F02C3A3F4009F4FFC3F3C32A3874
:1099900041E1340709F4CDC32139314111F40C946C
:1099A000C259E8C345E159E061E870E080E79AE018
:1099B0000E9421728CEA9FE0B3C3E3E0F0E0EC0F79
:1099C000FD1FE20FF31F1082C9010E94564C892B24
:1099D00089F720E030E040E050E0C357DF4F688176
:1099E000CD58D040627070E080E090E0A0E00E942E
:1099F0008E8909F07CC6C557DF4F2881CB58D040EF
:109A0000287030E040E050E060E070E080E090E0FE
:109A1000A0E00E948E89A1F127E04AE250E06BE2CB
:109A200070E089E290E00E94915C88E795E30E94F3
:109A30005D5EBC01882777FD8095982F0E94048B7E
:109A400020E030E048EC52E40E94658A9F938F93B7
:109A50007F936F9387EB96E09F938F931F9287E797
:109A60008F93CE018E0D9F1D03969F938F930E941F
:109A70008992E80EF91E0FB6F894DEBF0FBECDBF77
:109A8000C557DF4F2881CB58D040207130E040E0EF
:109A900050E060E070E080E090E0A0E00E948E89FD
:109AA000F1F126E04AE250E06BE270E089E290E0FA
:109AB0000E94915C81E090E00E9460118093851388
:109AC0008BEE9CE10E945D5EBC01882777FD80954E
:109AD000982F0E94048B20E030E048EC52E40E9472
:109AE000658A9F938F937F936F9381EC96E09F930A
:109AF0008F931F9287E78F93C7010296E1E0F0E012
:109B0000EC0FFD1F8E0F9F1F9F938F930E948992D2
:109B1000E80EF91E0FB6F894DEBF0FBECDBF272D9D
:109B200030E040E050E060E070E080E090E0A0E0F5
:109B30000E948E8901F10E941C119F938F937F9345
:109B40006F938CEC96E09F938F931F9287E78F9390
:109B5000C701029641E050E04C0F5D1F840F951F36
:109B60009F938F930E948992E80EF91E0FB6F89486
:109B7000DEBF0FBECDBFC557DF4F2881CB58D040C9
:109B8000207430E040E050E060E070E080E090E081
:109B9000A0E00E948E8931F18091B4308F93809142
:109BA000B3308F938091B2308F938091B1308F9387
:109BB0008AED96E09F938F931F9287E78F93C7015B
:109BC0000296A1E0B0E0AC0FBD1F8A0F9B1F9F93D0
:109BD0008F930E948992E80EF91E0FB6F894DEBFAB
:109BE0000FBECDBFC557DF4F2881CB58D04020785E
:109BF00030E040E050E060E070E080E090E0A0E025
:109C00000E948E8941F1F89480915E3590915F3584
:109C1000A0916035B09161357894BF93AF939F93D5
:109C20008F9388EE96E09F938F931F9287E78F9391
:109C3000C701029621E030E02C0F3D1F820F931FD9
:109C40009F938F930E948992E80EF91E0FB6F894A5
:109C5000DEBF0FBECDBF20E0C457DF4F3881CC58E8
:109C6000D040317040E050E060E070E080E090E093
:109C7000A0E00E948E8909F04CC520E0C457DF4F58
:109C80003881CC58D040327040E050E060E070E065
:109C900080E090E0A0E00E948E8909F0ADC520E050
:109CA000C457DF4F3881CC58D040347040E050E08A
:109CB00060E070E080E090E0A0E00E948E8909F012
:109CC000CCC520E0C457DF4F3881CC58D040387025
:109CD00040E050E060E070E080E090E0A0E00E94B2
:109CE0008E8909F0E9C520E0C457DF4F3881CC5890
:109CF000D040307140E050E060E070E080E090E003
:109D0000A0E00E948E8909F04AC620E0C457DF4FC8
:109D10003881CC58D040307240E050E060E070E0D4
:109D200080E090E0A0E00E948E8909F068C620E003
:109D300030E040E050E0C357DF4F6881CD58D0405D
:109D4000647070E080E090E0A0E00E948E8909F0ED
:109D500084C620E0CB56DF4F3881C559D04040E063
:109D600050E060E070E080E090E0A0E00E948E892A
:109D700009F0E0C620E0CA56DF4F3881C659D0400E
:109D800040E050E060E070E080E090E0A0E00E9401
:109D90008E8909F0FDC6502F5170D52E20E030E09D
:109DA000452F50E060E070E080E090E0A0E00E948D
:109DB0008E8909F01BC720E030E0402F427050E050
:109DC00060E070E080E090E0A0E00E948E8909F001
:109DD00040C720E030E0C657DF4F4881CA58D04026
:109DE00050E060E070E080E090E0A0E00E948E89AA
:109DF00009F062C720E030E0402F487050E060E09A
:109E000070E080E090E0A0E00E948E8909F07EC7BB
:109E100020E030E0402F407150E060E070E080E0F2
:109E200090E0A0E00E948E8909F0A0C720E030E019
:109E3000402F407250E060E070E080E090E0A0E0F1
:109E40000E948E8909F0C2C720E030E0402F4074A4
:109E500050E060E070E080E090E0A0E00E948E8939
:109E600009F0E4C7F02FF078AF2E20E030E04F2F5C
:109E700050E060E070E080E090E0A0E00E948E8919
:109E800011F00C944757212F2170B22E20E030E0C2
:109E900040E05B2D60E070E080E090E0A0E00E9498
:109EA0008E8911F00C94545720E030E04A2D50E098
:109EB00060E070E080E090E0A0E00E948E8911F008
:109EC0000C94625720E030E040E05B2D60E070E0F1
:109ED00080E090E0A0E00E948E8911F00C949757EA
:109EE00020E030E040E0512F527060E070E080E010
:109EF00090E0A0E00E948E8911F00C94CC5720E0F5
:109F000030E040E0512F547060E070E080E090E07D
:109F1000A0E00E948E8911F00C94FF5720E030E001
:109F200040E0512F507160E070E080E090E0A0E0F0
:109F30000E948E8911F00C94325820E030E040E00D
:109F4000512F507260E070E080E090E0A0E00E944D
:109F50008E8911F00C94715820E030E040E0512FD0
:109F6000507460E070E080E090E0A0E00E948E8994
:109F700011F00C94B05820E030E040E0512F5870C0
:109F800060E070E080E090E0A0E00E948E8911F037
:109F90000C94EF5820E030E040E05C2D60E070E091
:109FA00080E090E0A0E00E948E8911F00C9420598E
:109FB00020E030E04D2D50E060E070E080E090E087
:109FC000A0E00E948E8911F00C945C59C557DF4FB8
:109FD0002881CB58D040C457DF4F3881CC58D0406F
:109FE000A801C357DF4F6881CD58D040CE56DF4F10
:109FF0007881C259D040CD56DF4F8881C359D040B7
:10A00000CC56DF4F9881C459D040A0E00E948E8981
:10A0100011F00C946759809164028061898380916A
:10A02000640A8A83FE01EE0DFF1D1382809189135D
:10A0300090918A13A0918B13B0918C1387010D5FBF
:10A040001F4F80FF0CC01F930F9388E798E09F93EA
:10A050008F930E9426920F900F900F900F90B8014F
:10A06000CE0101960E9428748091660282FF0AC088
:10A070002EE531E3A801BE016F5F7F4F8EE692E0CF
:10A080000E947B5F8091891390918A13A0918B131A
:10A09000B0918C1382FD73980E94386780E79AE034
:10A0A0000E943D728091660290916702A0916802C1
:10A0B000B091690290FD02C00C949E593FEFE31AE3
:10A0C000F30A0E942F68D82E89E10E9447684091C8
:10A0D000660250916702609168027091690250FDBA
:10A0E00002C00C949A5973988091640A8F5F809390
:10A0F000640A8A83B7016F5F7F4FCE0101960E9489
:10A10000287480E79AE00E943D7240E050E065E8E4
:10A110008091CB149091CC140E94146F88E791E148
:10A12000C057DF4FA881B981C059D0408D939C930F
:10A130001EC088E59AE00E94A56D892BC1F00E949F
:10A1400038678091660287FD2B9840E450E060E01C
:10A1500070E088E59AE00E94876D81E991E1C0573F
:10A16000DF4FE881F981C059D0409183808381E03D
:10A170000C94D559C057DF4FA881B981C059D04040
:10A180001D921C9283E00C94D559623181F7C090E6
:10A190006602D0906702E0906802F0906902D1FCFC
:10A1A00009CCF8018081813091F50180F281E02DA8
:10A1B0002081C557DF4F2883CB58D0403181C45709
:10A1C000DF4F3883CC58D040028113814481C3577C
:10A1D000DF4F4883CD58D0405581CE56DF4F58834E
:10A1E000C259D0408681CD56DF4F8883C359D040B5
:10A1F0009781CC56DF4F9883C459D0402084318456
:10A20000C257DF4F19821882CE58D0406AC08230C0
:10A21000E9F4A381B481C257DF4FB983A883CE5834
:10A22000D040212C312CB1E0C557DF4FB883CB583B
:10A23000D040C457DF4F1882CC58D04000E010E81F
:10A24000C357DF4F1882CD58D0403CC08330F9F05F
:10A25000843009F0AFCB212C312CC257DF4F19824B
:10A260001882CE58D040E5E0C557DF4FE883CB5881
:10A27000D040C457DF4F1882CC58D04000E010E0E7
:10A28000F2E0C357DF4FF883CD58D0401BC0212CDC
:10A29000312CC257DF4F19821882CE58D04025E0AA
:10A2A000C557DF4F2883CB58D040C457DF4F1882A3
:10A2B000CC58D04000E010E031E0C357DF4F388386
:10A2C000CD58D040CE56DF4F1882C259D040CD561F
:10A2D000DF4F1882C359D040CC56DF4F1882C45983
:10A2E000D0408090B1309090B230A090B330B09018
:10A2F000B43040908D0250908E0260908F0270902A
:10A3000090022DEC3CEC4CE45EE3C301B2010E94F0
:10A310009B899B01AC01C501B4010E94278C87FD7C
:10A320000BC0E894E0F8C0926602D0926702E09217
:10A330006802F09269024AC0A3019201C501B4010A
:10A340000E94618A87FF42C08091BD309091BE30EB
:10A35000A091BF30B091C0300196A11DB11D809376
:10A36000BD309093BE30A093BF30B093C030E0FCBE
:10A3700021CB6894E0F8C0926602D0926702E09226
:10A380006802F092690245E4C557DF4F4883CB5815
:10A39000D04050E2C457DF4F5883CC58D04000E043
:10A3A00010E084E0C357DF4F8883CD58D040CE56AD
:10A3B000DF4F1882C259D040CD56DF4F1882C359A3
:10A3C000D040CC56DF4F1882C459D040902F9470A3
:10A3D000C657DF4F9883CA58D04020E030E0492F5D
:10A3E00050E060E070E080E090E0A0E00E948E89A4
:10A3F00009F08C9AC557DF4FA881CB58D040A07286
:10A400007A2E2A2F30E040E050E060E070E080E0FB
:10A4100090E0A0E00E948E8911F00E941C11C457A8
:10A42000DF4FB881CC58D040B074CB56DF4FB883E3
:10A43000C559D04020E03B2F40E050E060E070E0A4
:10A4400080E090E0A0E00E948E8911F00E94142527
:10A45000C457DF4FE881CC58D040E078CA56DF4F70
:10A46000E883C659D04020E03E2F40E050E060E055
:10A4700070E080E090E0A0E00E948E8951F00E94A0
:10A48000B71060936B3570936C3580936D359093F6
:10A490006E35C557DF4F2881CB58D040217030E052
:10A4A00040E050E060E070E080E090E0A0E00E94DA
:10A4B0008E89F1F089E79CE19F938F9387E996E07D
:10A4C0009F938F931F9287E78F93CE0103969F935D
:10A4D0008F930E9489926C010E94564C0FB6F8949B
:10A4E000DEBF0FBECDBF892B09F064CA760102C062
:10A4F000E12CF12CC557DF4F2881CB58D04022707A
:10A5000030E040E050E060E070E080E090E0A0E00B
:10A510000E948E89D1F1C70102966FE976E041E091
:10A5200050E04C0F5D1F840F951F0E948A9153E0ED
:10A53000E50EF11C48E7A42E45E3B42E56E7C52EE0
:10A5400053E0D52E67E7962ED5018D915D011F92C0
:10A550008F93DF92CF921F929F92C7010296E1E004
:10A56000F0E0EC0FFD1F8E0F9F1F9F938F930E94B3
:10A570008992E80EF91E0FB6F894DEBF0FBECDBF6C
:10A5800030E8A31635E3B306F9F6C557DF4F288147
:10A59000CB58D040247030E040E050E060E070E004
:10A5A00080E090E0A0E00E948E8909F447C0C701D6
:10A5B000029663EA76E041E050E04C0F5D1F840FA5
:10A5C000951F0E948A9154E0E50EF11C4E018AE726
:10A5D000880E911C80E1D4011D928A95E9F728E04C
:10A5E000A40168E980EB0E94C7175401B8E0AB0EE4
:10A5F000B11C26E7C22E23E0D22E37E7632EF401EA
:10A6000081914F011F928F93DF92CF921F926F9291
:10A61000C701029621E030E02C0F3D1F820F931FEF
:10A620009F938F930E948992E80EF91E0FB6F894BB
:10A63000DEBF0FBECDBF8A149B0409F7512F50789F
:10A64000C52E20E030E040E060E070E080E090E087
:10A65000A0E00E948E89E1F4809187139091881385
:10A660009F938F9388EA96E09F938F931F9287E73B
:10A670008F93CE018E0D9F1D03969F938F930E9403
:10A680008992E80EF91E0FB6F894DEBF0FBECDBF5B
:10A6900020E030E040E050E0C357DF4F6881CD5804
:10A6A000D040617070E080E090E0A0E00E948E8970
:10A6B00009F48FC9E3E0F0E0EC0FFD1FEE0DFF1D84
:10A6C00080E28083E1EEF0E3808197012F5F3F4FCE
:10A6D0007901882309F471C98081A1E0B0E0AC0F51
:10A6E000BD1FAE0DBF1D12968C933196EDCFCE01DE
:10A6F0008E0D9F1D6FEA76E003960E948A9197E087
:10A70000E90EF11CC7010E94564C892B09F052C971
:10A7100072C92114310409F4B0CAF89440905E352E
:10A7200050905F356090603570906135789480917D
:10A73000E31C9091E41CA091E51CB091E61CA301E0
:10A740009201281B390B4A0B5B0BCA01B9010E940D
:10A75000028B4B015C01B10180E090E00E94028B12
:10A760009B01AC01C501B4010E94658AB82ED92EA7
:10A770009F938F937F936F9383EF96E09F938F9335
:10A780001F9287E78F939E012E0D3F1D2D5F3F4F38
:10A790003F932F93C856DF4F6883C859D040C9569E
:10A7A000DF4F7883C759D0400E948992E80EF91E86
:10A7B000C856DF4F6881C859D040C956DF4F7881ED
:10A7C000C759D040862F972FAB2DBD2D8093703564
:10A7D00090937135A0937235B09373354092E31C1A
:10A7E0005092E41C6092E51C7092E61C0FB6F8943F
:10A7F000DEBF0FBECDBF41CA2114310409F44FCAD8
:10A80000F8948091BA1C9091BB1CA091BC1CB09193
:10A81000BD1C78949F938F9380916D028F9380914C
:10A820006C028F9380E097E09F938F931F9287E74E
:10A830008F93C7010296A1E0B0E0AC0FBD1F8A0F55
:10A840009B1F9F938F930E948992E80EF91E0FB66B
:10A85000F894DEBF0FBECDBF22CAF8948091623556
:10A8600090916335A0916435B09165357894BF932C
:10A87000AF939F938F9380E197E09F938F931F9265
:10A8800087E78F93C701029621E030E02C0F3D1F30
:10A89000820F931F9F938F930E948992E80EF91E57
:10A8A000C7010E94564C0FB6F894DEBF0FBECDBF55
:10A8B000892B09F07FC805CA2114310409F413CA91
:10A8C000F894409062355090633560906435709094
:10A8D000653578948091E71C9091E81CA091E91C63
:10A8E000B091EA1CA3019201281B390B4A0B5B0BA8
:10A8F000CA01B9010E94028B4B015C01B10180E0E9
:10A9000090E00E94028B9B01AC01C501B4010E9442
:10A91000658AB82ED92E9F938F937F936F938BE187
:10A9200097E09F938F931F9287E78F939E012E0D41
:10A930003F1D2D5F3F4F3F932F93C856DF4F6883D6
:10A94000C859D040C956DF4F7883C759D0400E94BC
:10A950008992E80EF91EC856DF4F6881C859D04069
:10A96000C956DF4F7881C759D040862F972FAB2D1E
:10A97000BD2D8093743590937535A0937635B09343
:10A9800077354092E71C5092E81C6092E91C709267
:10A99000EA1C0FB6F894DEBF0FBECDBFA4C92328B2
:10A9A00009F4B3C9F8948091BE1C9091BF1CA0918A
:10A9B000C01CB091C11C78949F938F9380916B02BF
:10A9C0008F9380916A028F9388E297E09F938F9391
:10A9D0001F9287E78F93C7010296A1E0B0E0AC0F0A
:10A9E000BD1F8A0F9B1F9F938F930E948992E80E31
:10A9F000F91E0FB6F894DEBF0FBECDBF86C9809199
:10AA0000B5309091B630A091B730B091B830BF93C7
:10AA1000AF939F938F9388E397E09F938F931F92B9
:10AA200087E78F93C701029621E030E02C0F3D1F8E
:10AA3000820F931F9F938F930E948992E80EF91EB5
:10AA4000C7010E94564C0FB6F894DEBF0FBECDBFB3
:10AA5000892B11F00C94DA4C6AC98091C0308F9325
:10AA60008091BF308F938091BE308F938091BD30A5
:10AA70008F938091BC308F938091BB308F93809166
:10AA8000BA308F938091B9308F9383E497E09F938E
:10AA90008F931F9297E7D92EDF92C7010296A1E00C
:10AAA000B0E0AC0FBD1F8A0F9B1F9F938F930E9436
:10AAB0008992E80EF91EC7010E94564C0FB6F89411
:10AAC000DEBF0FBECDBF892B11F00C94DA4C809104
:10AAD000AF2C9091B02C90FF3CC98091C4308F93E3
:10AAE0008091C3308F938091C2308F938091C13019
:10AAF0008F9387E697E09F938F931F92DF92C70112
:10AB0000029621E030E02C0F3D1F820F931F9F9390
:10AB10008F930E948992E80EF91EC7010E94564C3D
:10AB20000FB6F894DEBF0FBECDBF892B11F00C9489
:10AB3000DA4C0FC98091A6288F938091A5288F9316
:10AB40008091A4288F938091A3288F9389E797E021
:10AB50009F938F931F9287E78F93C7010296A1E07F
:10AB6000B0E0AC0FBD1F8A0F9B1F9F938F930E9475
:10AB70008992E80EF91EC7010E94564C0FB6F89450
:10AB8000DEBF0FBECDBF892B11F00C94DA4CF2C89A
:10AB900080916E358F9380916D358F9380916C3558
:10ABA0008F9380916B358F9384E897E09F938F9379
:10ABB0001F9287E78F93C701029621E030E02C0FA8
:10ABC0003D1F820F931F9F938F930E948992E80EDF
:10ABD000F91EC7010E94564C0FB6F894DEBF0FBE97
:10ABE000CDBF892B11F00C94DA4CD5C881E00E94BE
:10ABF0006810209185023091860240918702509121
:10AC000088020E94E68C9F938F937F936F9381E9D4
:10AC100097E09F938F931F9287E78F93C7010296C8
:10AC2000A1E0B0E0AC0FBD1F8A0F9B1F9F938F93D5
:10AC30000E948992E80EF91EC7010E94564C0FB679
:10AC4000F894DEBF0FBECDBF892B11F00C94DA4C07
:10AC5000B2C882E00E946810209181023091820285
:10AC600040918302509184020E94E68C9F938F93BF
:10AC70007F936F938EE997E09F938F931F9287E75F
:10AC80008F93C701029621E030E02C0F3D1F820F09
:10AC9000931F9F938F930E948992E80EF91EC7011C
:10ACA0000E94564C0FB6F894DEBF0FBECDBF892B65
:10ACB00011F00C94DA4C8DC883E00E9468109F93C9
:10ACC0008F937F936F938BEA97E09F938F931F925D
:10ACD00087E78F93C7010296A1E0B0E0AC0FBD1FDC
:10ACE0008A0F9B1F9F938F930E948992E80EF91EF3
:10ACF0008C98C7010E94564C0FB6F894DEBF0FBE69
:10AD0000CDBF892B11F00C94DA4C74C88091AF2C14
:10AD100087FF7EC821E042E161E080ED0E94AE60E5
:10AD20009F938F937F936F9388EB97E09F938F937D
:10AD30001F9287E78F93C701029621E030E02C0F26
:10AD40003D1F820F931F9F938F930E948992E80E5D
:10AD5000F91EC7010E94564C0FB6F894DEBF0FBE15
:10AD6000CDBF892B11F00C94DA4C52C88091AF2CD6
:10AD700087FF5CC821E042E162E080ED0E94AE60A6
:10AD80009F938F937F936F9386EC97E09F938F931E
:10AD90001F9287E78F93C7010296A1E0B0E0AC0F46
:10ADA000BD1F8A0F9B1F9F938F930E948992E80E6D
:10ADB000F91EC7010E94564C0FB6F894DEBF0FBEB5
:10ADC000CDBF892B11F00C94DA4C30C88091AF2C98
:10ADD00087FF3AC821E042E163E080ED0E94AE6067
:10ADE0009F938F937F936F9384ED97E09F938F93BF
:10ADF0001F9287E78F93C701029621E030E02C0F66
:10AE00003D1F820F931F9F938F930E948992E80E9C
:10AE1000F91EC7010E94564C0FB6F894DEBF0FBE54
:10AE2000CDBF892B11F00C94DA4C0EC88091AF2C59
:10AE300087FF18C821E042E164E080ED0E94AE6027
:10AE40009F938F937F936F9382EE97E09F938F935F
:10AE50001F9287E78F93C7010296A1E0B0E0AC0F85
:10AE6000BD1F8A0F9B1F9F938F930E948992E80EAC
:10AE7000F91EC7010E94564C0FB6F894DEBF0FBEF4
:10AE8000CDBF892B11F00C94DA4C0C94324F809189
:10AE9000AF2C82FD02C00C94434F46E061E083E09A
:10AEA0000E9483190C94434F8091AF2C82FD02C005
:10AEB0000C94544F21E046E061E083E00E94831946
:10AEC0000C94544F8091AF2C82FD02C00C94624FC1
:10AED0008091921D8F938091911D8F938091901DF1
:10AEE0008F9380918F1D8F9380EF97E09F938F9327
:10AEF0001F9287E78F93C701029641E050E04C0F05
:10AF00005D1F840F951F9F938F930E948992E80E77
:10AF1000F91EC7010E94564C0FB6F894DEBF0FBE53
:10AF2000CDBF892B11F00C94DA4C0C94624F8091B8
:10AF3000AF2C82FD02C00C94704F8091961D8F93B0
:10AF40008091951D8F938091941D8F938091931D77
:10AF50008F9388EF97E09F938F931F9287E78F934C
:10AF6000C7010296E1E0F0E0EC0FFD1F8E0F9F1F7E
:10AF70009F938F930E948992E80EF91EC7010E9449
:10AF8000564C0FB6F894DEBF0FBECDBF892B11F023
:10AF90000C94DA4C0C94704F8091AF2C9091B02CA3
:10AFA00090FD02C00C947F4F80E090E00E948C24C2
:10AFB0009F938F937F936F9383E098E09F938F93FA
:10AFC0001F9287E78F93C701029641E050E04C0F34
:10AFD0005D1F840F951F9F938F930E948992E80EA7
:10AFE000F91EC7010E94564C0FB6F894DEBF0FBE83
:10AFF000CDBF892B11F00C94DA4C0C947F4F8091CB
:10B00000AF2C9091B02C90FD02C00C948E4F81E03B
:10B0100090E00E948C249F938F937F936F9383E1A2
:10B0200098E09F938F931F9287E78F93C7010296B3
:10B03000E1E0F0E0EC0FFD1F8E0F9F1F9F938F93B9
:10B040000E948992E80EF91EC7010E94564C0FB665
:10B05000F894DEBF0FBECDBF892B11F00C94DA4CF3
:10B060000C948E4F8091AF2C9091B02C90FD02C02B
:10B070000C949D4F81E090E00E948C244B015C0178
:10B0800080E090E00E948C249B01AC01C501B401DA
:10B090000E948D229F938F937F936F9384E298E019
:10B0A0009F938F931F9287E78F93C701029641E08A
:10B0B00050E04C0F5D1F840F951F9F938F930E944C
:10B0C0008992E80EF91EC7010E94564C0FB6F894FB
:10B0D000DEBF0FBECDBF892B11F00C94DA4C0C945F
:10B0E0009D4F8091AF2C9091B02C90FD02C00C949C
:10B0F000AC4F81E090E00E948C244B015C0180E029
:10B1000090E00E948C249B01AC01C501B4010E9417
:10B11000EE229F938F937F936F938FE298E09F939C
:10B120008F931F9287E78F93C7010296E1E0F0E0CB
:10B13000EC0FFD1F8E0F9F1F9F938F930E9489928C
:10B14000E80EF91EC7010E94564C0FB6F894DEBFF8
:10B150000FBECDBF892B11F00C94DA4C0C94AC4F80
:10B160008091AF2C9091B02C90FD02C00C94BB4FFD
:10B1700081E090E00E948C244B015C0180E090E033
:10B180000E948C249B01AC01C501B4010E944F2395
:10B190009F938F937F936F938DE398E09F938F930B
:10B1A0001F9287E78F93C701029641E050E04C0F52
:10B1B0005D1F840F951F9F938F930E948992E80EC5
:10B1C000F91EC7010E94564C0FB6F894DEBF0FBEA1
:10B1D000CDBF892B11F00C94DA4C0C94BB4F8091AD
:10B1E000AF2C9091B02C91FD02C00C94CA4F0E94DC
:10B1F000DA1D9F938F937F936F9380E598E09F93E1
:10B200008F931F9287E78F93C7010296E1E0F0E0EA
:10B21000EC0FFD1F8E0F9F1F9F938F930E948992AB
:10B22000E80EF91EC7010E94564C0FB6F894DEBF17
:10B230000FBECDBF892B11F00C94DA4C0C94CA4F81
:10B24000C257DF4FA881B981CE58D04016968C9155
:10B2500016971F928F9315968C9115971F928F9327
:10B2600013968C9113971F928F9312968C911F9225
:10B270008F9381E698E09F938F931F9287E78F9338
:10B28000C7010296E1E0F0E0EC0FFD1F8E0F9F1F5B
:10B290009F938F930E948992E80EF91EC7010E9426
:10B2A000564C0FB6F894DEBF0FBECDBF892B11F000
:10B2B0000C94DA4C0C94D84F779A80918913909122
:10B2C0008A13A0918B13B0918C1392FD749A809184
:10B2D000891390918A13A0918B13B0918C1382FDE6
:10B2E0000CC08091660280FD08C081FD02C00C94F4
:10B2F0000B501D9902C00C940B5040E050E060E0F0
:10B3000070E0CE0101960E94B60E2091981D30E0AB
:10B3100080917F13909180132817390710F40C94B3
:10B320000B5040E050E062E180E192E00E94146F37
:10B330000C940B508D2D0E944768739A809187134F
:10B3400090918813892B11F00E946F668091640A96
:10B350008F5F8093640A8091891390918A13A091E2
:10B360008B13B0918C1382FD02C00C94DA4C739A4B
:10B370000C94DA4C653811F00C94B750E12CF12C98
:10B380000C94675088E59AE00E94A56D892B11F412
:10B390000C94B7500E946F668091660287FD02C0D0
:10B3A0000C94DA4C2B9A0C94DA4CC856DF4F0FB63B
:10B3B000F894DEBF0FBECDBFDF91CF911F910F91EB
:10B3C000FF90EF90DF90CF90BF90AF909F908F90C5
:10B3D0007F906F905F904F903F902F9008950C94C6
:10B3E000D4714F925F926F927F929F92AF92BF9271
:10B3F000CF92DF92EF92FF920F931F93CF93DF9341
:10B40000CDB7DEB760970FB6F894DEBF0FBECDBFE5
:10B410005B010E942F68E82FF0E0EE0FFF1FE4555C
:10B42000F34E80819181019691838083809189136D
:10B4300090918A13A0918B13B0918C1381FD749815
:10B4400040906602509067026090680270906902B6
:10B450000E9486736C01FC018081982F92959F70E9
:10B46000913099F48F7051F48091901C9091911CBF
:10B4700001969093911C8093901C3CC1B50186E984
:10B4800097E30E943F73892B51F080918E1C90911D
:10B490008F1C019690938F1C80938E1C2BC1D3011F
:10B4A000C2011EE0B695A795979587951A95D1F795
:10B4B000F82FF1709F2E8BE79AE00E94EB6F7C01D2
:10B4C000009709F44BC0B501C70102960E943F7373
:10B4D000892B09F43FC0870129E73EE040E054E6AC
:10B4E00060E070E0C7010F960E941D6CF60191812B
:10B4F000F7018481981321C082858F5F82878091B4
:10B500008C1C90918D1C019690938D1C80938C1CAB
:10B5100084E00E947474F701208530E02817390711
:10B5200008F07CC184E00E947474F7018087F60102
:10B5300080818F70F7018187DDC0F701128684E07A
:10B540000E947474F7018087F60180818F70F70183
:10B55000818765C1C7010E944C70B1CF88E092E03D
:10B560000E9473707C01009709F4C4C0B501C70143
:10B5700002960E943873F60181818150F70184831D
:10B5800080E091E0A0E0B0E083879487A587B6874C
:10B59000128684E00E947474F7018087F60180812E
:10B5A0008F70F7018187B7018BE79AE00E942670C0
:10B5B000870129E73EE040E054E660E070E0C70123
:10B5C0000F960E941D6C11E0F6018181F7018483C2
:10B5D000F60180818F70F701878384E00E94747484
:10B5E000F701858383E00E947474F7018683878165
:10B5F0008F3009F010E0F6014180F7018481481A8C
:10B60000512C612C712C76E0440C551C661C771C67
:10B610007A95D1F72385348545855685A0ECB0E031
:10B620000E94C287BB27A92F982F872F480E591E2B
:10B630006A1E7B1E4386548665867686A501B70101
:10B64000C6010E94B60E2091981D30E080917F13B4
:10B65000909180132817390738F040E050E062E1FC
:10B6600080E192E00E94146F80917F13909180138B
:10B67000029708F44BC08091AF2C86FF2AC00E942D
:10B68000FD5FC60105960E94C95FF60181811F9288
:10B690008F93F70186811F928F9385811F928F93DD
:10B6A00089E898E09F938F931F9280E18F93CE015A
:10B6B00001965C01BF928F930E94899282E00E9462
:10B6C000E35FC5010E94C95F0FB6F894DEBF0FBEED
:10B6D000CDBF8091660290916702A0916802B091FF
:10B6E000690297FD50C080917F139091801302975B
:10B6F00008F47EC08091891390918A13A0918B13D6
:10B70000B0918C1381FF8DC0749A8BC080916602BA
:10B7100090916702A0916802B091690296FFABCF49
:10B72000992009F4A8CFF6012081322F3F70832F92
:10B7300090E00297F4F08FEF830F207F822B8083BD
:10B7400080E79AE00E94EF5980918A1C90918B1CAF
:10B75000019690938B1C80938A1C80918913909101
:10B760008A13A0918B13B0918C1396FF84CF73989A
:10B7700082CF8091901C9091911C01969093911C86
:10B780008093901C78CF89E79CE12091791C22233B
:10B7900009F4A9CF9F938F938CE998E09F938F939F
:10B7A000CE0101965C01BF928F930E94C6923C012C
:10B7B000B501C60102960E94AB910F900F900F90B9
:10B7C0000F900F900F90009709F48DCF93012F5F8A
:10B7D0003F4F280F391FA9012F5F3F4FFA0180818A
:10B7E0008032C9F362E18AE192E00E94146F7BCF5C
:10B7F000112309F47FCF82E08093CA301092CC30BD
:10B800001092CB30F092CE30E092CD304AEC50E343
:10B8100062E182E492E00E94146F6CCF912C10E000
:10B82000D3CE60960FB6F894DEBF0FBECDBFDF91CA
:10B83000CF911F910F91FF90EF90DF90CF90BF902D
:10B84000AF909F907F906F905F904F90089581157B
:10B85000910511F00197F1F70895E0918B35F09182
:10B860008C35908180918A3589230895E0918835BF
:10B87000F0918935808190918A35892B8083E09180
:10B880008D35F0918E35808190918A35892B80831A
:10B8900008951F93CF93DF93E0918835F091893518
:10B8A000908180918A35809589238083E0918D35C0
:10B8B000F0918E35808190918A35892B80838FEB32
:10B8C00093E00E94275C1FB7F894E0918D35F091CA
:10B8D0008E35908180918A3580958923808383E895
:10B8E00090E00E94275CE0918B35F0918C35D081FF
:10B8F000C0918A351FBF78948BE393E00E94275C48
:10B90000E0918B35F0918C35908180918A35982328
:10B9100019F08D2F8C2301C081E0DF91CF911F9111
:10B92000089550938E3540938D357093893560938B
:10B93000883590938C3580938B3581E001C0880FDA
:10B940002A95EAF780938A350C94495CCF93DF936C
:10B95000C82FDFB7F894E0918D35F0918E35808156
:10B9600090918A35892B808383E090E00E94275C48
:10B97000CC2351F0E0918D35F0918E3580819091FE
:10B980008A3590959823908387E190E00E94275C08
:10B99000E0918B35F0918C35808190918A358923A7
:10B9A00009F4C0E089E590E00E94275CE0918D35C4
:10B9B000F0918E35808190918A359095982390836F
:10B9C000DFBF8BE390E00E94275C8C2FDF91CF914B
:10B9D0000895CF93DF93C82FD8E08C2F81700E94F9
:10B9E000A65CC6958111C068D150B9F78C2FDF9144
:10B9F000CF9108958FEF0C94E95CDF92EF92FF9264
:10BA00000F931F93CF93DF93E82EEB010E94495CC5
:10BA100081112FC080EF0E94E95CF12C10E488EFC7
:10BA2000D82ED10E81E00E94A65C082F81E00E94F2
:10BA3000A65C882319F0002361F01DC0011109C024
:10BA40001E1528F0888180FF04C0E11611F0F12E48
:10BA500001E0802F0E94A65C988196950111906864
:10BA6000988311501D11DECF21961111D8CF8F2D43
:10BA700003C08FEF01C08EEFDF91CF911F910F9127
:10BA8000FF90EF90DF900895FF920F931F93CF9355
:10BA9000DF93F82EEB010E94495C209769F085E561
:10BAA0000E94E95C8E01085F1F4F89910E94E95C4A
:10BAB000C017D107D1F703C08CEC0E94E95C8F2D31
:10BAC000DF91CF911F910F91FF900C94E95C0F9340
:10BAD0001F93CF93DF93DB01EC9111969C9111970B
:10BAE000F0E0F92B803181F4BF016E7FE3E0660F57
:10BAF000771FEA95E1F716969C911697ECE0F0E037
:10BB0000E91BF109E60FF71FF7FF07C091E0EA0113
:10BB10009883F195E195F10902C0EA011882883213
:10BB200079F414968C91982F9076903649F086FF90
:10BB300002C0EE7F05C085FF02C0EC7F01C0E87F38
:10BB4000CF0144E0969587954A95E1F7D9018C930A
:10BB5000EF70E801E88380E0DF91CF911F910F91B2
:10BB600008950F931F93CF93DF93EC018B01B801DE
:10BB700088810E94FD5C888381508D3F30F4F801FC
:10BB80008081883211F0803191F7DF91CF911F9140
:10BB90000F910895CF93DF93EC010E94495CBE01A1
:10BBA00084EB0E94445D81E00E94A65CC82F0E9445
:10BBB000495C81E0C11101C080E0DF91CF9108951F
:10BBC0001F93CF93DF931F921F92CDB7DEB7182F2D
:10BBD00069837A830E94495C0E942D5C69817A8125
:10BBE000882341F084E40E94445D113029F00E94D2
:10BBF000365C02C082E001C080E00F900F90DF91C0
:10BC0000CF911F9108954F925F926F927F928F9282
:10BC10009F92AF92BF92CF92DF92EF92FF920F93DB
:10BC20001F93CF93DF93CDB7DEB729970FB6F89464
:10BC3000DEBF0FBECDBF6C015B014A0189010E94CE
:10BC4000495CB6018EEB0E94445DCE0101967C01F9
:10BC50003E019AE0690E711C27010E94FA5CF7010F
:10BC600081937F01E615F705C1F769E070E0C20135
:10BC70000E941C78811109C09401A501B201F6014E
:10BC800080810E94675D80E001C083E029960FB645
:10BC9000F894DEBF0FBECDBFDF91CF911F910F9102
:10BCA000FF90EF90DF90CF90BF90AF909F908F90DC
:10BCB0007F906F905F904F900895EF92FF920F9357
:10BCC0001F93CF93DF93CDB7DEB72B970FB6F894C2
:10BCD000DEBF0FBECDBFF82EE92E682F792F88E08A
:10BCE0008F0D0E94E05D882319F084E391E243C048
:10BCF00066E471E48FE090E00E94C85E8E01075F09
:10BD00001F4F9801AE01465F5F4FBE01655F7F4FD9
:10BD10008F2D9E2D0E94035E8111E7CF88E0E1EE1A
:10BD2000F2E0DE01119601900D928A95E1F74985C6
:10BD300021E732E0429FC001439F900D112464E649
:10BD400070E00E9449878A8594E6899F600D711D85
:10BD50001124FE0131968191481303C06F5F7F4F1C
:10BD600003C0E017F107B9F78B85882319F07195A7
:10BD700061957109CB012B960FB6F894DEBF0FBE0B
:10BD8000CDBFDF91CF911F910F91FF90EF9008955C
:10BD9000DC01CB0181159105A105B10529F0815088
:10BDA0009040A040B040D9F708959B01AC0110929B
:10BDB000B90060E072E18AE790E00E945D8720515F
:10BDC0003109410951095695479537952795209393
:10BDD000B800089594EA9093BC0040EA56E861E008
:10BDE00070E09091BC0097FD0BC041505109610972
:10BDF0007109411551056105710599F781E00895B3
:10BE00009091B900987F983011F09031B9F78093F4
:10BE1000BB0084E88093BC0080EA96E8A1E0B0E033
:10BE20002091BC0027FD08C00197A109B109009726
:10BE3000A105B105A9F7E2CF8091B900887F8831CB
:10BE400011F08034D9F680E0089524EA34E844E91A
:10BE50002093BC009091BC0097FFFCCF9091B9005B
:10BE6000987F983011F0903199F78093BB00309310
:10BE7000BC009091BC0097FFFCCF9091B900987FD7
:10BE8000903211F0983539F44093BC009091BC0089
:10BE900094FDFCCFDDCF08950C94EA5E84E9809395
:10BEA000BC008091BC0084FDFCCF08958093BB0052
:10BEB00084E88093BC008091BC0087FFFCCF909108
:10BEC000B900987F81E0983209F480E0089584EC0D
:10BED0008093BC008091BC0087FFFCCF8091BB00A9
:10BEE000089584E88093BC008091BC0087FFFCCF5C
:10BEF0008091BB000895E0E1DC01FD91CD01F0935C
:10BF00003F01E150C9F780913C018F7D80933C0156
:10BF100080913C01877F80933C01FB0180E19191FE
:10BF200090933E018150D9F780913C0180688093C5
:10BF30003C0180913D0180FFFCCF4051510980912F
:10BF40003C01806280933C0180913C01877F80931B
:10BF50003C01141615069CF4FB0180E1919190932D
:10BF60003E018150D9F780913C01806880933C016B
:10BF700080913D0180FFFCCF40515109EACFF9018A
:10BF800080E190913E0191938150D9F781E090E05A
:10BF900008950F931F93CF93DF93EC018CE70E94DA
:10BFA000255F8CE70E94565F8E01005F1F4F8991CD
:10BFB0000E94565FC017D107D1F7DF91CF911F9133
:10BFC0000F910C944E5F813019F440E050E002C0B4
:10BFD00040EC50E060E070E08CE790E00C94AF172C
:10BFE000813019F44EE050E002C048E050E060E0DB
:10BFF00070E08CE790E00C94AF1741E050E060E017
:10C0000070E08CE790E00E94AF176AE67AE080E08B
:10C0100090E00C94C85E48E350E060E070E08CE78C
:10C0200090E00E94AF1749E350E060E070E08CE7D9
:10C0300090E00E94AF1744E150E060E070E08CE7D0
:10C0400090E00E94AF1748E750E060E070E08CE7B6
:10C0500090E00E94AF174EE550E060E070E08CE7A2
:10C0600090E00E94AF174DE650E060E070E08CE792
:10C0700090E00E94AF176CE17AE186E090E00E94C8
:10C08000C85E4CE050E060E070E08CE790E00E9419
:10C09000AF1741E050E060E070E08CE790E00E9474
:10C0A000AF1746E050E060E070E08CE790E00E945F
:10C0B000AF176AE67AE080E090E00C94C85ECF9318
:10C0C000DF93CDB7DEB7A2970FB6F894DEBF0FBEF1
:10C0D000CDBF81E1EBE2F9E0DE01529601900D92D5
:10C0E0008A95E1F781E1ECE3F9E0DE011196019038
:10C0F0000D928A95E1F70E940B60CE0142960E9454
:10C10000C95F82E00E94E35F6AE67AE080E090E047
:10C110000E94C85ECE0101960E94C95F60E17EEA7E
:10C1200088E290E00E94C85E80E00E94F05F60E1DB
:10C130007EEA88E290E00E94C85E4EE050E060E057
:10C1400070E08CE790E00E94AF17A2960FB6F894CB
:10C15000DEBF0FBECDBFDF91CF910895CF92DF92AA
:10C16000EF92FF920F931F93CF93DF9300D0CDB741
:10C17000DEB7F82E042F122F213031F0223031F0AB
:10C18000243031F0283031F090E005C091E003C058
:10C1900092E001C093E00C3059F00E3011F494603D
:10C1A00007C0003111F4986003C0023109F49C60AB
:10C1B000613059F0623011F4906207C0633011F4BD
:10C1C000906403C0643009F490669068692F70E051
:10C1D00023E030E0AE014F5F5F4F8F2D90E00E9473
:10C1E000C71769E07AE180E090E00E94C85E8F2D79
:10C1F0008160F82E0E94EA5E0E94675F89830E9438
:10C20000675F8A83023119F40E94675F8B830E9403
:10C21000675F87FDF1CF0E94715F0E944E5F69E00A
:10C220007AE180E090E00E94C85E8F2D0E94EA5E75
:10C230000E94675F89830E94675F8A83023119F4D5
:10C240000E94715F8B830E94715F0E944E5F3981F3
:10C250002A81023149F5832F90E0A0E0B0E04B81C4
:10C260007727662731FF0EC030E0322F2227620F7A
:10C27000731F811D911D640F711D811D911D8C6F98
:10C280009F6F0BC030E0322F2227620F731F811D7A
:10C29000911D640F711D811D911D0E94048B20E86A
:10C2A0003FEF4FEF57E420C0632F70E0762F6627F3
:10C2B000620F711D882777FD8095982F0E94048B4F
:10C2C0000C3029F420E030EE4FEF54E40DC00E3076
:10C2D00029F420E038EF4FEF55E406C0003131F487
:10C2E00020E03EEF4FEF56E40E94658A2FE632E1F0
:10C2F00043E050E40E94E68C6B017C01612F70E00A
:10C3000080E090E00E94048B9B01AC01C701B60164
:10C310000E94658A0F900F900F90DF91CF911F912F
:10C320000F91FF90EF90DF90CF900895CF93E6E4C8
:10C33000F1E0208190818081C081C295C695C6952B
:10C34000C370207CC20F969596959073C90F829505
:10C350008C70C80F1F92CF9327EE32E13F932F933B
:10C360000E9438920F900F900F900F908C2FCF91CA
:10C3700008951F93CF93DF9346E06CE080E00E9426
:10C38000F86480E00E944D650E94DB6304B600FE05
:10C3900008C086ED92E19F938F930E9438920F9090
:10C3A0000F9004B601FE08C085EC92E19F938F9335
:10C3B0000E9438920F900F9004B602FE08C084EBE2
:10C3C00092E19F938F930E9438920F900F9004B642
:10C3D00003FE08C083EA92E19F938F930E943892F4
:10C3E0000F900F9004B604FE08C086E992E19F9377
:10C3F0008F930E9438920F900F90E0EFF9E322E4C0
:10C4000032E4318320833A968DB79EB70A97E817B6
:10C41000F907B8F38DE499E09F938F938BE792E14E
:10C420009F938F930E9438920E946E6F0E94A16E1C
:10C4300060E070E085EB92E00E94416F0E94116C19
:10C44000E0919109F091920919950E94966190E00E
:10C450000E9479650E94507382E0809396378093A2
:10C4600097370E94D36346E957E3BC018DEC9BEA02
:10C470000E944C680E944D630E9432680E94D763FC
:10C480000E9458690E948D74E091070AF091080A91
:10C490001995E091DF09F091E0091995E091D10932
:10C4A000F091D20919950E945A69182FC091130A68
:10C4B000D091140AFE0119950F900F900F900F90D4
:10C4C000892B49F0FE011995BC0180E890E00E949B
:10C4D0003587EB0102C0C0E8D0E00E942F681F92B0
:10C4E0001F93DF93CF931F928F938091060A8F93B0
:10C4F0008091050A8F938091DE098F938091DD09E9
:10C500008F9389E492E19F938F930E9438928CE3FA
:10C5100092E19F938F930E9438928BE292E19F93D6
:10C520008F930E94389260E070E087ED92E00E9465
:10C53000416F89E199E00E949C6B83E292E19F93B5
:10C540008F930E9438928DB79EB742960FB6F8949B
:10C550009EBF0FBE8DBFDF91CF911F91089580E8E0
:10C5600080936100109261000E94B96180E0282EE2
:10C5700082E1382ECFEED1E10EED11E190EDE92E02
:10C5800091E1F92E2CE3822E912CA12CB12C33EBCE
:10C59000C32E31E1D32E04B600FE08C0A1E1B2E102
:10C5A000BF93AF930E9438920F900F9004B601FE94
:10C5B00006C03F922F920E9438920F900F9004B6BF
:10C5C00002FE06C0DF93CF930E9438920F900F9027
:10C5D00004B603FE06C01F930F930E9438920F907B
:10C5E0000F9004B604FE06C0FF92EF920E943892AC
:10C5F0000F900F9014BE0E94B16E0E946E65409025
:10C6000094355090953560909635709097350E948E
:10C610000564461657066806790609F4BCCF0E94E1
:10C620000564609394357093953580939635909317
:10C630009735A50194010E945D87672B682B692BB4
:10C6400011F40E94DA708091943590919535A09103
:10C650009635B09197359370AA27BB270397A1050C
:10C66000B10509F098CFE0EFF9E380819181823440
:10C67000924469F0E05FF943FF93EF93DF92CF922A
:10C680000E9438920F900F900F900F9084CF3A969F
:10C69000E53FB1E8FB0748F37ECF1F93CF93DF93CD
:10C6A000CDB7DEB7A0970FB6F894DEBF0FBECDBFF3
:10C6B00083E690E00E946B93182F282F35EF380FF8
:10C6C000303108F0982F9095291709F461C086EF52
:10C6D00092E19F938F930E943892EBE3F3E10F90E6
:10C6E0000F90DE01119684918D93319683E1E334AE
:10C6F000F807C9F7F89448E050E06FE770E0CE0122
:10C7000001960E947193EDE2F3E1DE0111968491AE
:10C710008D93319683E1EB33F807C9F74EE050E093
:10C7200061E770E0CE0101960E947193E3E2F3E1CC
:10C73000DE01119684918D93319683E1ED32F807F5
:10C74000C9F74AE050E067E670E0CE0101960E942A
:10C7500071936DEC7BEA81E690E00E94899360E042
:10C7600070E08FE590E00E94899360E08EE590E0B4
:10C770000E947B9360E070E085E690E00E948993E0
:10C780001AE16AE175EE83E690E00E94899378945D
:10C79000812FA0960FB6F894DEBF0FBECDBFDF91FC
:10C7A000CF911F9108958FE590E00C946B938EE5E7
:10C7B00090E00C946393F8941092B60016BC83EF4B
:10C7C00087BD82E084BD94E095BD95B395BB809311
:10C7D0006E00789408950F931F9360918F1370915A
:10C7E0009013809191139091921300918F13109157
:10C7F0009013209191133091921360177107820763
:10C80000930759F71F910F9108950F931F9360910C
:10C81000A0357091A1358091A2359091A3350091FA
:10C82000A0351091A1352091A2353091A335601724
:10C8300071078207930759F71F910F9108951F926F
:10C840000F920FB60F9211240BB60F922F933F93B6
:10C850004F935F936F937F938F939F93AF93BF9308
:10C86000EF93FF9380918F1390919013A091911368
:10C87000B09192130196A11DB11D80938F139093D7
:10C880009013A0939113B093921380918E138F5FA6
:10C8900080938E1387FF15C010928E138091A03560
:10C8A0009091A135A091A235B091A3350196A11D1B
:10C8B000B11D8093A0359093A135A093A235B0937C
:10C8C000A33580913F378823E1F080918D138F5FEE
:10C8D00080938D1387FF15C010928D13809198352A
:10C8E00090919935A0919A35B0919B350196A11DF3
:10C8F000B11D8093983590939935A0939A35B09354
:10C900009B350E94B06D892B11F00E94D16CFF9174
:10C91000EF91BF91AF919F918F917F916F915F91B7
:10C920004F913F912F910F900BBE0F900FBE0F9024
:10C930001F9018951F920F920FB60F9211240BB6ED
:10C940000F922F933F934F935F936F937F938F93A8
:10C950009F93AF93BF93EF93FF938091C600E091B5
:10C96000A635F091A735309709F01995FF91EF9111
:10C97000BF91AF919F918F917F916F915F914F91F7
:10C980003F912F910F900BBE0F900FBE0F901F90F5
:10C9900018951F920F920FB60F9211240BB60F929B
:10C9A0002F933F934F935F936F937F938F939F93B7
:10C9B000AF93BF93EF93FF938091CE00E091A435A6
:10C9C000F091A535309709F01995FF91EF91BF913E
:10C9D000AF919F918F917F916F915F914F913F9117
:10C9E0002F910F900BBE0F900FBE0F901F901895B8
:10C9F00081110EC01092C5006093C40088E9809335
:10CA0000C1004093C2001092A7351092A635089538
:10CA1000813069F41092CD006093CC0088E9809356
:10CA2000C9004093CA001092A5351092A43508950C
:10CA3000811107C08091C00085FFFCCF6093C600C4
:10CA40000895813031F48091C80085FFFCCF609358
:10CA5000CE000895CF93C82F8A3031F46DE08091D5
:10CA600093130E94186502C08D3029F06C2F8091BD
:10CA700093130E94186580E090E0CF910895811192
:10CA800005C07093A7356093A6350895813021F4D1
:10CA90007093A5356093A43508958093931383E92B
:10CAA00092E09093EB398093EA39089584B7877FB9
:10CAB00084BF88E10FB6F894809360001092600004
:10CAC0000FBE08952FE088E190E00FB6F894A89586
:10CAD000809360000FBE209360000895A89508958C
:10CAE00088E10FB6F89480936000109260000FBE4A
:10CAF00008950C94F78D0C94F38D8091AD3590E0F2
:10CB000008958091390181FF09C0809139018D7F9D
:10CB1000809339018DE090E00197F1F723E040E048
:10CB20006FE182E491E00E94BA6A83E090E00197AD
:10CB3000F1F708959091390191FD0AC0282F8031B5
:10CB400008F02FE040E06FE085E491E00C94BA6AD1
:10CB500008958091390181FD0EC040E06FE181E4CC
:10CB600091E00E94B06A282F2F7E81E090E0213072
:10CB700021F080E0089580E090E0089580913901EF
:10CB800081FD10C040E06FE181E491E00E94B06A55
:10CB90008F3131F0982F9F7E915081E0923018F4C0
:10CBA00080E0089581E008958091390181FD04C0FD
:10CBB0000E94BE658823C1F3089510923F3780918B
:10CBC000390181FD8BC00E94D4658091390181FDBE
:10CBD00085C00E948165809139018260809339010E
:10CBE000809177378823D9F18091940090919500B6
:10CBF000409188375091893784179507A0F4809128
:10CC0000543790915537A0915637B09157378C577C
:10CC1000914EAF4FBF4F8093543790935537A093A9
:10CC20005637B09357372091940030919500241BCC
:10CC3000350B8091543790915537A0915637B0916C
:10CC40005737820F931FA11DB11D809354379093C6
:10CC50005537A0935637B093573710927737809156
:10CC600079378823D9F18091940090919500409173
:10CC70008C3750918D3784179507A0F480915C37DD
:10CC800090915D37A0915E37B0915F378C57914E90
:10CC9000AF4FBF4F80935C3790935D37A0935E3763
:10CCA000B0935F372091940030919500241B350B91
:10CCB00080915C3790915D37A0915E37B0915F377E
:10CCC000820F931FA11DB11D80935C3790935D3738
:10CCD000A0935E37B0935F371092793708958091B3
:10CCE0003F37882321F00E94BE650E94DD6580E009
:10CCF00090E00895AB0122E0260F27FF0CC0809141
:10CD00003D3790913E37019690933E3780933D3763
:10CD10008FEF9FEF0895BC0184E993E10E94719128
:10CD200080E090E0089540E06FE181E491E00C94B0
:10CD3000B06A282F40E06FEF86E591E00E94BA6A62
:10CD40000895CF93DF93C82F88EF8C0F823038F08F
:10CD50008C2F8F7E863019F0C93109F04CC080913C
:10CD6000390181FD4BC00E94D4650E949366D82F83
:10CD7000C81709F43DC0C83029F4809139010E94D8
:10CD8000816527C0C93119F4863181F404C0C631E8
:10CD900069F4893159F429E040E06FE182E491E0DF
:10CDA0000E94BA6AE3E0F0E03197F1F72C2F40E0FF
:10CDB0006FE182E491E00E94BA6AD83031F48FEFDB
:10CDC0000E949966E9E6F1E002C0E3E0F0E0319705
:10CDD000F1F70E9493668C1759F0C63029F4813020
:10CDE00039F083E490E00CC0C631D9F78131C9F73E
:10CDF00080E490E005C082E490E002C084E490E02A
:10CE0000DF91CF9108958091940090919500909337
:10CE10008D3780938C3721E02093793720933F37EB
:10CE20008091390181FF1FC08091940090919500FD
:10CE300090938937809388372093773720933A37B8
:10CE40002FB7789480913901809139018D7F80933B
:10CE5000390180E197E230913A37332319F0019795
:10CE60000097C9F72FBF86E10E94A1660C94D46594
:10CE700080913F37811102C00E94036781E090E0FA
:10CE800008950F931F93CF93DF931F92CDB7DEB713
:10CE900080913F37882361F08091390181FF02C082
:10CEA00080E07CC00E94BE658823D1F310E003C0FF
:10CEB0000E94386711E080919400909195009093C2
:10CEC00087378093863701E00093763780E8809338
:10CED000550186E00E94A1660093AE358FB7898325
:10CEE0007894109247018091AE358111FCCF8981F1
:10CEF0008FBF9091470181E09E3008F080E0082FBD
:10CF0000019586E10E94A1661092550180917637C5
:10CF10008823D9F12091940030919500E0918637D3
:10CF2000F09187372E173F07A0F44091503750916A
:10CF3000513760915237709153374C57514E6F4F64
:10CF40007F4F4093503750935137609352377093CF
:10CF5000533720919400309195002E1B3F0B409148
:10CF60005037509151376091523770915337420F7B
:10CF7000531F611D711D409350375093513760937B
:10CF80005237709353371092763711110E946F66A3
:10CF90000295069506950370802F817090E00F90A2
:10CFA000DF91CF911F910F9108958FEF80934E01E4
:10CFB00021E044E060EF8CE691E00E94BA6A25E04F
:10CFC00041E06EE08CE691E00E94BA6A80E88093CE
:10CFD0006F018091460180936D0121E045E060E2A0
:10CFE00084E491E00C94BA6A8DEF93E00197F1F735
:10CFF0000E94AF6A1092B435109236361092B8364D
:10D000001092B3351092B235E9E3F1E080818E7F62
:10D01000808380818D7F808381EE91E00197F1F79D
:10D0200080818160808323E040E06FE182E491E0D1
:10D030000E94BA6A8DEF93E00197F1F780915D014C
:10D0400080915E010E94D56760E070E081EA92E025
:10D050000E94416F0E94036781E090E008958091F3
:10D0600015140895CF93DF931F92CDB7DEB7898350
:10D070000E94D465898180931514282F40E06FE1C8
:10D0800088E491E00F90DF91CF910C94BA6A0E94EE
:10D09000326886E00C94A166EF92FF920F931F9383
:10D0A000CF93DF931F921F92CDB7DEB78C017A0129
:10D0B0007F936F931F938F9327E639E03F932F93CE
:10D0C00069837A830E942692009362011093630120
:10D0D0006981609360017A81709361010F900F9074
:10D0E0000F900F900F900F90E114F104C9F0F70129
:10D0F000808180936B01818180936A01828180931A
:10D1000069018381809368018481809367018581AF
:10D110008093660186818093650187818093640195
:10D120000F900F90DF91CF911F910F91FF90EF9093
:10D13000089581EA92E00E94626F81E08093AD35AC
:10D140008091AF359091B03501969093B035809332
:10D15000AF3581E090E008951F93CF93DF93209146
:10D16000B33512E8129F90011124D901AC54BA4C86
:10D170004C91442309F450C047FD08C0433030F0BF
:10D1800050E0EA0122976C177D0710F41C9244C00E
:10D19000B9016B547A4C0E9471918091B335189FFC
:10D1A000F0011124EC54FA4CDF01A058BF4F9C91C0
:10D1B0009093A83510828F5F833018F48093B33535
:10D1C00002C01092B335E091B33582E8E89FF001D8
:10D1D0001124EC54FA4C8081882319F00E9499683C
:10D1E00002C01092AD35809147018093A93590918E
:10D1F000AC35992311F0891710F48093AC35609108
:10D20000A93570E084E00E9469746091A83570E0EF
:10D2100083E00E94697402C0C0E0D0E0CE01DF91DB
:10D22000CF911F9108950F931F93CF93DF931F9278
:10D23000CDB7DEB78C01FC0180819181009709F1A7
:10D240008334954029F0F8011182108283E02AC0CE
:10D250006238E1F40E9415748FB78983F8940E94B4
:10D26000867360E870E00E94AC6829812FBF1816B1
:10D27000190674F40E948173E0910D0AF0910E0A70
:10D28000199583E495E0F8019183808381E00AC0D9
:10D290008091AA359091AB3501969093AB358093F0
:10D2A000AA35EFCF0F90DF91CF911F910F91089585
:10D2B0000C949A658091390181FD06C040E06FE0D1
:10D2C00085E491E00C94B06A80E10895CF92DF92FA
:10D2D000FF921F93CF93DF931F92CDB7DEB7F82E47
:10D2E0008091390181FD07C00E94D46580913F374C
:10D2F00081111FC05DC08091940090919500909322
:10D3000089378093883781E08093773780933A37E5
:10D31000809139018D7F8093390120E137E280913E
:10D320003A37882309F32150310921153105B9F71E
:10D33000DBCF809179378823D9F120919400309107
:10D34000950080918C3790918D3728173907A0F47C
:10D3500040915C3750915D3760915E3770915F37D7
:10D360004C57514E6F4F7F4F40935C3750935D3712
:10D3700060935E3770935F372091940030919500F1
:10D38000281B390B40915C3750915D3760915E37B7
:10D3900070915F37420F531F611D711D40935C37C1
:10D3A00050935D3760935E3770935F371092793793
:10D3B00089E10E94A16686E00E947474892B51F075
:10D3C0000E945A69C82E86E00E94747481500E949F
:10D3D0009A6502C0C12CD12C809194009091950047
:10D3E00090938B3780938A3781E0809378378FB71B
:10D3F0008983F8948091390182608093390180910A
:10D4000039018D7F8093390162E06F0D84E993E1EA
:10D410000E94FF6A89818FBF20913B3730913C3752
:10D420002F5F3F4F30933C3720933B370E94D465AA
:10D4300045E060EE82E491E00E94B06A182F86E039
:10D440000E947474892B19F08C2D0E949A6580912A
:10D4500078378823D9F12091940030919500E0919C
:10D460008A37F0918B372E173F07A0F44091583739
:10D470005091593760915A3770915B374C57514EE4
:10D480006F4F7F4F409358375093593760935A37B7
:10D4900070935B3720919400309195002E1B3F0BC9
:10D4A000409158375091593760915A3770915B3796
:10D4B000420F531F611D711D4093583750935937C8
:10D4C00060935A3770935B371092783780913F376B
:10D4D000882371F0209194003091950030938D371E
:10D4E00020938C3781E0809379370E94036702C0D4
:10D4F0000E94DD65123028F48CE00E94747410E004
:10D500000BC0133031F0153031F0173029F411E031
:10D5100003C012E001C013E0812F90E00F90DF9173
:10D52000CF911F91FF90DF90CF900895CF93DF931D
:10D53000EB010E947A66009729F4CE010E94666989
:10D54000009751F020913D3730913E372F5F3F4F8C
:10D5500030933E3720933D37DF91CF910895089562
:10D56000FC018081862390E002C0959587954A95BD
:10D57000E2F70895CF93DF931F92CDB7DEB73FB7A1
:10D580003983F894FC015081362F30955323042EB3
:10D5900001C0220F0A94EAF72623522B5083898177
:10D5A0008FBF0F90DF91CF91089540917B012DEFB8
:10D5B000240FFC012D3738F01082E058FF4F108205
:10D5C0003196108208954193A0E8B1E050E8540FDD
:10D5D0009D012F5F3F4F6C916193521711F0D9015C
:10D5E000F7CF4150E42FF0E0E058FE4F2181FC01DD
:10D5F000E058FF4F2083319621E020830895609307
:10D600008001E1E8F1E061589F012F5F3F4FDC01AD
:10D610004D91CD014083621711F0F901F5CF0895C6
:10D620001F920F920FB60F9211240BB60F922F93E9
:10D630003F934F935F936F937F938F939F93AF939A
:10D64000BF93EF93FF93809147018093A935809119
:10D65000B23522E8829FC00111248C549A4C0E945A
:10D66000D56A8091B2358F5F833018F48093B235DC
:10D6700002C01092B2350E949968FF91EF91BF915C
:10D68000AF919F918F917F916F915F914F913F915A
:10D690002F910F900BBE0F900FBE0F901F901895FB
:10D6A0001F920F920FB60F9211240F900FBE0F9082
:10D6B0001F9018951F920F920FB60F9211240F9082
:10D6C0000FBE0F901F9018951F920F920FB60F92DA
:10D6D00011240F900FBE0F901F9018951F920F925C
:10D6E0000FB60F92112410923A370F900FBE0F9081
:10D6F0001F9018951F920F920FB60F92112410923F
:10D70000B1350F900FBE0F901F9018951F920F927A
:10D710000FB60F9211240F900FBE0F901F90189507
:10D720001F920F920FB60F9211241092AE350F90E8
:10D730000FBE0F901F901895CF93DF93EC01899146
:10D740009991009729F060E070E00E94416FF7CF57
:10D75000DF91CF910895EF92FF920F931F93CF9394
:10D76000DF938C017A01FC0180819181009741F067
:10D770008A34910511F1F8011182108283E04AC0C8
:10D7800087E194E10E94EB6FEC01209761F04E81FC
:10D790005F8168857985CE0102960E94876D099028
:10D7A000D881C02DF2CF81E0809316148AE490E0F6
:10D7B000F8019183808381E02DC06838E1F787E12B
:10D7C00094E10E94EB6FEC01209781F3CE01029669
:10D7D000E816F906D9F4BE0187E194E10E940B70C6
:10D7E000E090CB14F090CC148E859F859093CC1450
:10D7F0008093CB14E889F989309719F08A899B893D
:10D800001995F092CC14E092CB14D0CF0990D88126
:10D81000C02DDACFDF91CF911F910F91FF90EF9044
:10D8200008951092161487E194E10E94E76F60E07A
:10D8300070E08BEA92E00C94416FEF92FF920F93AD
:10D840001F93CF93DF93EC01E090CB14F090CC14B6
:10D85000FF86EE86398B288B1B8B0A8B80911614E2
:10D86000882379F08BEA92E09093CC148093CB14C8
:10D87000CE0102960E94876DF092CC14E092CB14F8
:10D8800004C04E835F8368877987BE0187E194E196
:10D890000E940B70BE0187E194E1DF91CF911F914F
:10D8A0000F91FF90EF900C942670CF93DF93EC01D3
:10D8B00080911614882329F0CE0102960E94BB6D38
:10D8C00004C01B861A861D861C86BE0187E194E172
:10D8D000DF91CF910C940B708F929F92AF92BF9279
:10D8E000CF92DF92EF92FF920F931F9380911D14BE
:10D8F00090911E14892B49F41092191410921A1445
:10D9000010921B1410921C1441C00E94EB63E09112
:10D910001D14F0911E140481158126813781C08069
:10D92000D180E280F3800C0D1D1D2E1D3F1D061BB6
:10D93000170B280B390B0084F185E02D3097C1F0CF
:10D9400084809580A680B780C080D180E280F380FB
:10D950008C0C9D1CAE1CBF1C861A970AA80AB90A1B
:10D9600080169106A206B30630F795018401E3CF35
:10D97000DC01CB01800F911FA21FB31F80931914EC
:10D9800090931A14A0931B14B0931C141F910F9121
:10D99000FF90EF90DF90CF90BF90AF909F908F90CF
:10D9A000089585EB92E00C94626FEF92FF920F93D3
:10D9B0001F93CF93DF938C01FC01808191810097AD
:10D9C00099F089359105D9F0F8011182108283E030
:10D9D00068C0828593858417950709F049C0008443
:10D9E000F185E02D3097A9F710921E1410921D14A6
:10D9F00089E590E0F8019183808381E052C0673827
:10DA000091F16238A9F7C0911D14D0911E14E12C38
:10DA1000F12C209769F3CE010E94C16F892BF1F0A0
:10DA2000AE0168E88A859B850E94146F892BA1F45A
:10DA30001B861A8688859985E114F10421F0F70187
:10DA40009187808704C090931E1480931D141986BB
:10DA500018860E946C6CD7CF0E94D16C7E0108841E
:10DA6000D985C02DD6CFE0911D14F0911E14BACFE8
:10DA7000F0931E14E0931D14A085B185109709F44E
:10DA8000B7CF1A968D919C911B978417950711F02B
:10DA9000FD01F2CF18968D919C91199791878087FF
:10DAA000EBCFDF91CF911F910F91FF90EF900895F1
:10DAB000CF93DF93EC010E94D16C8A859B853091D6
:10DAC0001D1420911E14892B91F0E32FF22F309713
:10DAD00071F0EC17FD0739F48091CB149091CC14C0
:10DAE0009387828710C00084F185E02DF0CF80916C
:10DAF000CB149091CC149B878A8738872987D09341
:10DB00001E14C0931D14DF91CF910C946C6CCF93B5
:10DB1000DF93EC010E948F6FCE01DF91CF910C94C7
:10DB2000586DCF93DF93EC010E949F6FCE01DF9180
:10DB3000CF910C94586DCF93DF93EC010E94B56F99
:10DB4000CE01DF91CF910C94586D21E030E0FC01C3
:10DB500082859385892B11F020E030E0C90108957A
:10DB600081E090E020911D1430911E14232B11F4BC
:10DB700080E090E00895CF93DF93EC01E0911D14D5
:10DB8000F0911E148E179F0769F4888599859093EC
:10DB90001E1480931D140DC0808591858C179D07E0
:10DBA00021F0FC013097C1F706C0888599859187DF
:10DBB00080870E946C6C198618861B861A86DF91F6
:10DBC000CF9108951F93CF93DF93EC01162FEC8133
:10DBD000FD813097D1F09093CC148093CB1482E0E8
:10DBE0008887CE0106961995992787FD909502970B
:10DBF000029710F0133839F4BE01CE01DF91CF91B6
:10DC00001F910C940F6E81E08887DF91CF911F9157
:10DC10000895FC01208520FD0C94E26D0895CF92BB
:10DC2000DF92EF92FF920F931F93CF93DF93EC015C
:10DC30006B01E090CB14F090CC140091CD141091B6
:10DC4000CE14F801EC17FD0739F0309709F44AC0FB
:10DC50000190F081E02DF6CF209709F443C088852C
:10DC6000882309F118860115110561F0C017D10745
:10DC700029F0AE0167E8C8010E94096EF801008131
:10DC80001181F1CFEC81FD81309769F0CC15DD0574
:10DC900051F0D093CC14C093CB1440E050E063E833
:10DCA000CE0106961995E091CD14F091CE14CE17C1
:10DCB000DF0769F4888199819093CE148093CD1405
:10DCC0000DC0808191818C179D0721F0FC01309758
:10DCD000C1F704C08881998191838083F092CC142C
:10DCE000E092CB14DF91CF911F910F91FF90EF90B5
:10DCF000DF90CF9008951F93CF93DF931092271456
:10DD0000C091CD14D091CE1411E0209779F089857F
:10DD1000882341F01887198640E050E062E8CE0180
:10DD20000E94E26D0990D881C02DEFCFDF91CF9195
:10DD30001F9108958091CA1491E0980F9093CA148E
:10DD400008958AE88093CA141092C8141092C914D6
:10DD50001092CE141092CD141092CC141092CB14B9
:10DD600008958091271481110E947B6E7091C914CF
:10DD7000772309F451C0E091C8142E2F30E085E0DC
:10DD8000E89FF0011124E85DFB4E6081609326144A
:10DD900041815281509325144093241483819481AE
:10DDA00090932314809322142F5F3F4F2F713327BA
:10DDB0002093C81471507093C914009731F5809165
:10DDC000CD149091CE1490932114809320148091BF
:10DDD000201490912114892BF9F08091271481113E
:10DDE0000E947B6E4091241450912514609126145A
:10DDF00080912014909121140E94096EE0912014CA
:10DE0000F091211480819181DECF613819F421E0F5
:10DE1000FC0120870E94096E809127142091C9146B
:10DE200090E0820F911D08952091C9142032B9F01D
:10DE3000E091C814E20FEF71E0931F1435E0E39F07
:10DE4000F0011124E85DFB4E60835283418394838B
:10DE500083832F5F2093C91480E090E0089581E0D0
:10DE600090E00895CF93DF93C091CB14D091CC1460
:10DE70000E94096ED093CC14C093CB14DF91CF9144
:10DE80000895AB013091CD142091CE14E32FF22FE1
:10DE9000E817F907B1F0309721F00190F081E02DFB
:10DEA000F7CF009771F0FC01308321839093CE145B
:10DEB0008093CD1421E020871782168261E80C94AC
:10DEC000326F0895009749F0FC01208521502230DF
:10DED00020F421E021872093271408950C94AC7836
:10DEE0008091CF149091D0140097C1F01092D0146B
:10DEF0001092CF14DC0114966D917C9115971296B7
:10DF0000ED91FC9113971995E091CF14F091D014F5
:10DF1000309721F0808191810C94C6780895CF9339
:10DF2000DF93EC014C835D836E837F830E94EB6300
:10DF3000688379838A839B83DF91CF9108950F93C0
:10DF40001F93FC014081518162817381048115819D
:10DF500026813781400F511F621F731F40835183F9
:10DF6000628373831F910F910895CF93DF93EC0128
:10DF70000E94EB63688379838A839B83DF91CF91CF
:10DF800008950F931F93CF93DF93EC010E94EB63EF
:10DF9000088119812A813B81601B710B820B930BD5
:10DFA0006F5F7F4F8F4F9F4F41E050E00C811D818D
:10DFB0002E813F81061717072807390710F040E028
:10DFC00050E0CA01DF91CF911F910F910895FC019C
:10DFD000118210820895FC01808191810895DC01F5
:10DFE000ED91FC91309731F080819181009729F07B
:10DFF000FC01FACF80E090E00895CF010895DC01A4
:10E00000ED91FC911197309721F0208131812D9372
:10E010003C93CF010895DC01ED91FC913097A9F07C
:10E02000A0E0B0E020813181E617F70741F41097B6
:10E0300009F4DC012D933C9311821082089521157F
:10E04000310519F0DF01F901EDCF08950F931F930A
:10E05000CF93DF938C01EB010E940B701982188221
:10E06000C8010E94EF6F009711F4F80101C0FC0194
:10E07000D183C083DF91CF911F910F910895DC016F
:10E08000ED91FC9180E090E0309729F001960190AD
:10E09000F081E02DF9CF0895009721F0FC018081F7
:10E0A0009181089580E090E00895CF93DF93EC0193
:10E0B0004A815B8160E070E08C819D810E947A9151
:10E0C0002A813B8188819981289FA001299F500D39
:10E0D000389F500D112460E070E08E819F81DF91A8
:10E0E000CF910C947A91FC018281938120E030E001
:10E0F00028173907D1F0A481B581A20FB31F4C9125
:10E10000411110C081E08C9380819181289FA001F2
:10E11000299F500D389F500D112486819781840FBF
:10E12000951F08952F5F3F4FE3CF80E090E0089563
:10E13000FC01268137814281538180E090E0841781
:10E140009507C9F02617370781F4A481B581A80F78
:10E15000B91F2C91121614F421502C930480F581D0
:10E16000E02DE80FF91F80810895A081B1812A0F69
:10E170003B1F0196E4CF8FEF0895FC0186819781C4
:10E1800068177907A0F0A081B18142815381A49FD3
:10E190009001A59F300DB49F300D1124280F391F19
:10E1A00081E090E06217730720F080E0089580E03E
:10E1B00090E008952F923F924F925F926F927F92DC
:10E1C0008F929F92AF92BF92CF92DF92EF92FF9287
:10E1D0000F931F93CF93DF93CDB7DEB768970FB63A
:10E1E000F894DEBF0FBECDBFECE6F7E320813181AE
:10E1F00042815381E8E6F7E35080418032802380FA
:10E20000ECE5F7E39080818072806380E8E5F7E3D6
:10E210008081898391819A83A281AB83B381BC83FE
:10E22000E4E5F7E380818D8391819E83A281AF83B2
:10E23000B381B887E0E5F7E38081898791819A8788
:10E24000A281AB87B381BC87ECE4F7E380818D8743
:10E2500091819E87A281AF87B381B88BE8E4F7E311
:10E260008081898B91819A8BB280A380E4E4F7E36B
:10E27000F080E180D280C380E0E4F7E3A081AF8B3F
:10E28000B181B88F128103812B8B3C8B4D8B5E8BC0
:10E290000E9405645E895F934D894F933C893F934B
:10E2A0002B892F932F923F924F925F926F927F9282
:10E2B0008F929F922C812F932B812F932A812F93C2
:10E2C00029812F9328852F932F812F932E812F9390
:10E2D0002D812F932C852F932B852F932A852F9378
:10E2E00029852F9328892F932F852F932E852F9360
:10E2F0002D852F93AF92BF922A892F9329892F932F
:10E30000CF92DF92EF92FF920F931F93288D2F935E
:10E310002F892F939F938F937F936F93809197373C
:10E320001F928F93809196371F928F9383E493E18E
:10E330009F938F930E9438920FB6F894DEBF0FBE62
:10E34000CDBF68960FB6F894DEBF0FBECDBFDF918C
:10E35000CF911F910F91FF90EF90DF90CF90BF90E2
:10E36000AF909F908F907F906F905F904F903F9075
:10E370002F900895EF92FF920F931F93CF93DF9307
:10E38000EC018B017A010E944E72F886EF8260ECFC
:10E3900079E0C801DF91CF911F910F91FF90EF902D
:10E3A0000C9472720C9456720C940A73DC011796DA
:10E3B000ED91FC9118970190F081E02D309709F0D4
:10E3C00019940895DC011796ED91FC91189702803D
:10E3D000F381E02D309709F019940895DC01199626
:10E3E000ED91FC911A970280F381E02D309709F0AE
:10E3F000199408950F931F93CF93DF931F921F9249
:10E40000CDB7DEB78C0188E10E948774BC01CE01D4
:10E4100001960E943873D8011996ED91FC911A97D4
:10E420000190F081E02D309729F0BE016F5F7F4FA2
:10E43000C80119950F900F90DF91CF911F910F9107
:10E440000895EF92FF920F931F93CF93DF93EC0108
:10E450008B017A0142EC59E00E94BA71FA86E98692
:10E4600066EC79E0C801DF91CF911F910F91FF9089
:10E47000EF900C9472720C94D271CF93DF93EC01F5
:10E4800066E977E388E10E947D74CE01DF91CF9148
:10E490000C94D47181ED94E10C94E76FFC017383CB
:10E4A0006283BC0181ED94E10C942670BC0181ED86
:10E4B00094E10C940B70CF93DF93EC0181ED94E128
:10E4C0000E94EB6F009749F0FC01228133812C17E9
:10E4D0003D0729F00E944C70F5CF80E090E0DF917D
:10E4E000CF9108950F931F93CF93DF938B010E94D9
:10E4F0005B72EC01009731F01D830C83C8010E9410
:10E5000089828E83DF91CF911F910F910895CF92D1
:10E51000DF92EF92FF920F931F93CF93DF937C01D3
:10E520008B016A0183ED94E10E94EB6FEC0100978F
:10E5300051F0EC81FD81309711F0C8011995CE01A1
:10E540000E944C70F3CFA601B801C701DF91CF91B3
:10E550001F910F91FF90EF90DF90CF900C94E2719C
:10E560000F931F93CF93DF931F921F92CDB7DEB708
:10E570000E945B828C0183ED94E10E94EB6F009717
:10E5800079F0DC011296ED91FC911397309729F008
:10E5900089839A8319959A8189810E944C70EFCF63
:10E5A0000115110549F0C8010F900F90DF91CF912F
:10E5B0001F910F910C94D6710F900F90DF91CF9116
:10E5C0001F910F910895CF92DF92EF92FF920F93D8
:10E5D0001F930E948D740E9415740E94E4800E9413
:10E5E0005982C12C88E0D82E87E0E82EF12C00E07B
:10E5F0001EE120E030E040E052E060E070E082E0C8
:10E6000090E00E9416821F910F91FF90EF90DF9093
:10E61000CF900895CF93DF93EC010E946E82009714
:10E6200061F00E949F73E091E109F091E209BE015F
:10E6300087E892E7199581E090E0DF91CF91089506
:10E64000E091090AF0910A0A1994E091D309F09136
:10E65000D4091994E0910F0AF091100A1994E091ED
:10E66000110AF091120A199480E090E0089508953B
:10E67000FB0120813181FC0131832083089542E038
:10E6800050E00E94649121E030E0892B11F020E0FD
:10E6900030E0C9010895BC0186E997E30C94387312
:10E6A000E0919109F09192091995E091070AF09192
:10E6B000080A1995E091DF09F091E0091995E091B8
:10E6C000D109F091D209199440918C1550918D1572
:10E6D0004817590798F020918A1530918B15280F0B
:10E6E000391F30938B1520938A15481B590B509373
:10E6F0008D1540938C1581E090E0089580E090E0C6
:10E70000089590938D1580938C15089580918A15A6
:10E7100090918B15895F9A4E08958091891590E0AC
:10E7200089529B4E089581E090E02091D51430915C
:10E73000D6142750354111F480E090E008950E94EE
:10E740009373892B61F06091D5147091D614409128
:10E750008C1550918D1587E095E10C947191209165
:10E760008A1530918B1521153105B9F080918C15E2
:10E7700090918D15C096E7E0F5E1AF01475D5441FA
:10E780004817590734F4DF01A20FB31F4C9141938E
:10E79000F4CF10928B1510928A15089580918C15E4
:10E7A00090918D15089520E380918915281B809103
:10E7B0008C1590918D15820F911D08951F93CF9305
:10E7C000DF93EC0110918915812F90E08C179D0744
:10E7D0006CF00E94D3738C0F9D1F8138910530F42B
:10E7E0001C1B1093891581E090E002C080E090E04E
:10E7F000DF91CF911F910895CF93DF93E0EAF7E384
:10E800001192119287E3E03DF807D1F7C8E9D7E309
:10E810006BEE79E0CE010E943873229687E3C03A0E
:10E82000D807B1F7DF91CF91089510928B15109210
:10E830008A1510928D1510928C1580E3809389159E
:10E8400087E095E19093D6148093D5140C94FC73D3
:10E85000EF92FF920F931F93CF93DF931F921F921C
:10E86000CDB7DEB78C0169837A830E941574698104
:10E87000E62E7A81F72E81E8E816F10418F080E898
:10E88000E82EF12CA701B8018091D5149091D614EF
:10E890000E947191F0928D15E0928C15C7010F9036
:10E8A0000F90DF91CF911F910F91FF90EF900895FE
:10E8B00020E3FC01A0EAB7E301900D922A95E1F76D
:10E8C00088E0FB01A8E9B7E301900D928A95E1F792
:10E8D0000895E82FF0E0EE0FFF1FE056F84C71832B
:10E8E000608381E090E00895E82FF0E0EE0FFF1FD5
:10E8F000E056F84C80819181089590E0880F991F2F
:10E900008859984C0E94387381E090E0089590E017
:10E91000880F991F8859984C08958FEB92E00E94B8
:10E9200055708FEC92E00E94557087EC92E00C9449
:10E9300055700F931F93CF93DF93EC01BC018FECC5
:10E9400092E00E94BD70892BA9F00990D881C02D5A
:10E95000FE0161917191CF010E942874BE016E5435
:10E960007F4FCE018E579F4FDF91CF911F910F9117
:10E970000C945874BE0187EC92E00E94BD70892B04
:10E98000D1F00E941574688179818A819B810E94EF
:10E9900028748CA990E00E94DE730CA910E00E94FC
:10E9A0008D73BE016C5F7F4FA801DF91CF911F91E6
:10E9B0000F910C947191DF91CF911F910F91089558
:10E9C00081E09CE10E94A56D892B21F081E09CE112
:10E9D0000C949B6D0895E091ED1BF091EE1B309728
:10E9E00009F0199480E00895EF92FF920F931F931E
:10E9F000CF93DF937C01EA01FC0180819181009734
:10EA000041F08A33934081F1F7011182108283E053
:10EA1000F4C080E024E0829FF0011124E151F44E23
:10EA2000118210828F5F8430A8F38093EC1B809159
:10EA3000CB149091CC149093001C8093FF1B0E94E8
:10EA40009A6E8093D03740E450E060E070E081E05F
:10EA50009CE10E94876D0E948A798AE393E0F70126
:10EA60009183808381E0C9C06230D9F48091D1372D
:10EA70009091D237892B89F38091E237863029F43F
:10EA80008091FA3781FD0E94E07481E00E94D07984
:10EA90008091D1379091D237892BF9F20E94497633
:10EAA000DCCF633060F5611114C02097B1F2D093D0
:10EAB000CF38C093CE3883E00E94D0798091D1378F
:10EAC0009091D237892B11F00E94EB740E94E07470
:10EAD000C4CF613011F6209709F4BFCFD093CB3863
:10EAE000C093CA3885E00E94D0798091D137909147
:10EAF000D237892B09F4B1CF0E94EB74AECF6738BF
:10EB0000E9F51092EB1B0FEE1BE18091EB1B8430BB
:10EB1000B8F4F801828193818C179D0749F48081B4
:10EB200091810E94B679F8011182108213821282BB
:10EB30000C5F1F4F8091EB1B8F5F8093EB1BE5CF2A
:10EB4000E9EEF8E3838194818C179D0719F4148210
:10EB500013821082B09629E3E936F20799F7E6E6C8
:10EB6000F9E3818592858C179D0711F41582148233
:10EB70003D9689E3E83EF807A1F76FCF683809F0C2
:10EB80006CCFC150DC4109F068CF81E09CE10E946C
:10EB9000A56D892B09F461CF1092EB1BE091EB1B63
:10EBA000E43008F05ACF20E2E29FF0011124E05354
:10EBB000F74C818D8823D9F081E09CE10E949B6D08
:10EBC0008091EB1BE0E28E9FC00111248053974C93
:10EBD0009093CF388093CE3882E00E94D079809194
:10EBE000D1379091D237892B11F00E94EB7480912C
:10EBF000EB1B8F5F8093EB1BD1CFDF91CF911F91E8
:10EC00000F91FF90EF900895CF93DF93A091CE38AE
:10EC1000B091CF38109719F0ED016C9605C0C091F6
:10EC2000CA38D091CB3829968091C93886FF22C046
:10EC30001092EA1B40E0EFEEFBE14430B8F4208193
:10EC4000318114968D919C9115972817390759F4A5
:10EC500082819381009739F04093EA1B99838883DE
:10EC60001B821A8205C034964F5FE7CF4093EA1BA0
:10EC70000E94E07488819981009741F04A815B810C
:10EC80006091D037DF91CF910C94326FDF91CF91AB
:10EC900008950F931F93CF93DF938091E2378630CF
:10ECA00009F07AC08091D1379091D237803F910599
:10ECB00008F472C08897EC01D695C7959E01220F83
:10ECC000331F8E012817390710F40F5F1F4FCE0135
:10ECD00088969093D2378093D1379093DB37809387
:10ECE000DC371092FE371092FD370E9484798095B0
:10ECF00090959093FE378093FD371092E4371092F1
:10ED0000E3370E947379809590959093E4378093D0
:10ED1000E3370E94EB74C80188969093D2378093B2
:10ED2000D1379093DB378093DC378091CC3890914A
:10ED3000CD38BC016C0F7D1FA8010E947191BE01EE
:10ED400081EF97E30E9422798091D5378093F13744
:10ED50008091D6378093F2378091D7378093F337FD
:10ED60008091D8378093F4371092FE371092FD3798
:10ED70000E948479809590959093FE378093FD371B
:10ED80001092E4371092E3370E9473798095909542
:10ED90009093E4378093E337DF91CF911F910F91E8
:10EDA0000C94EB74E091A109F091A209199480E010
:10EDB00090E00895AF92BF92CF92DF92EF92FF92D0
:10EDC0000F931F93CF93DF93CDB7DEB7E1970FB6C5
:10EDD000F894DEBF0FBECDBF7C015B01CE01019672
:10EDE0006C0181E3F60111928A95E9F781E089834C
:10EDF0008CE00E9474748C831D821F8280910D1C94
:10EE000091E0980F90930D1C898713E018878DEC83
:10EE10009BEA9B878A8789E10E9487746BEE79E081
:10EE20000E943F73892B31F082E08E838FEF8C87B5
:10EE30008D8709C089E10E948774BC01CE010C96C0
:10EE40000E9438731E838DEC9BEA9D8B8C8B66E948
:10EE500077E3CE0146960E9438730E9486739FA77F
:10EE60008EA70E94CE7399AB88ABC6010E94D58253
:10EE70008C011127C8010E94DE73892B31F10E9499
:10EE80008D73A801BC01C6010E94F8820091970908
:10EE9000109198090E94D3736C010E948D73B60182
:10EEA000F8011995E114F10481F0009739F0019708
:10EEB00061F441E050E064E070E004C041E050E003
:10EEC00060E070E0C501F7011995E1960FB6F8947E
:10EED000DEBF0FBECDBFDF91CF911F910F91FF908D
:10EEE000EF90DF90CF90BF90AF9008950F931F9356
:10EEF000CF93DF931F921F92CDB7DEB78C014115E0
:10EF0000510591F0FA018281938169837A830E948D
:10EF1000997469817A81C8010F900F90DF91CF9128
:10EF20001F910F910C94DA760F900F90DF91CF9193
:10EF30001F910F9108950F931F93CF93DF93CDB738
:10EF4000DEB7E1970FB6F894DEBF0FBECDBF0E94CB
:10EF5000CE738C010E948673AE014F5F5F4FB80184
:10EF60000E94F283892B09F447C088A999A99801C6
:10EF7000281B390BC9010E946473892BE9F12E818A
:10EF800021110CC0BE016A5E7F4F88E10E947D7432
:10EF9000E091E309F091E40919952EC08A859B85DB
:10EFA0008D3C3BEA930711F0019631F5223019F0C0
:10EFB00088E090E002C082E090E001979C012F5F22
:10EFC0003F4F12161306F4F6E1E0F0E0EC0FFD1FE0
:10EFD000E80FF91F23852F3F81F3BE01645F7F4F48
:10EFE00089E10E947D7489E10E94877466E977E374
:10EFF0000E943F73892B31F6E1960FB6F894DEBF7D
:10F000000FBECDBFDF91CF911F910F9108950E9448
:10F010007B6580930D1CE091A109F091A2091994E0
:10F02000892B29F0E091A109F091A20904C0E09197
:10F03000A309F091A4091994FC01680F791F80E0DD
:10F0400048E1E617F70781F0219198E0322F382741
:10F05000532F517030FD84278695513009F4806814
:10F060002695915099F7EDCF08951F920F920FB604
:10F070000F9211240BB60F922F933F934F935F93F0
:10F080006F937F938F939F93AF93BF93EF93FF9370
:10F09000809194009091950090938337809382376C
:10F0A00081E08093743780917100807D809371003E
:10F0B0000E94706F809174378823D9F180919400F9
:10F0C000909195004091823750918337841795072E
:10F0D000A0F48091483790914937A0914A37B09178
:10F0E0004B378C57914EAF4FBF4F8093483790931B
:10F0F0004937A0934A37B0934B3720919400309111
:10F100009500241B350B8091483790914937A09189
:10F110004A37B0914B37820F931FA11DB11D8093C9
:10F12000483790934937A0934A37B0934B371092A2
:10F130007437FF91EF91BF91AF919F918F917F9124
:10F140006F915F914F913F912F910F900BBE0F9058
:10F150000FBE0F901F9018959FB7F894E1E7F0E06D
:10F160008081807D808388B38F6288BB10929000FD
:10F17000E1E9F0E010821092920010929500109256
:10F1800094008081856080839FBF08952FB7F89495
:10F19000909399008093980088B38F6288BBE1E7D1
:10F1A000F0E08081826080832FBF0895FB01415091
:10F1B0005109460F571FE417F50778F4208130E016
:10F1C000322F22276181260F311D820F931F821754
:10F1D000930708F401963296EECFE417F50751F441
:10F1E000208130E0322F2227820F931F821793074E
:10F1F00008F401960895CF93DF93C091DC37D0E0F7
:10F2000064972091DB3730E0322F2227C20FD31FC3
:10F2100048E050E065EE77E39E01280F311DC901FB
:10F220000E94D678AE016DEE77E30E94D678009703
:10F2300021F098278927982702C08FEF9FEFDF9151
:10F24000CF910895FC015381560F5093D837872FE3
:10F2500099274281480F4093D737A181A093D63791
:10F26000E081E093D537242F30E02817390748F4A0
:10F2700081E08A0F8093D637811103C0EF5FE0935E
:10F28000D537852F90E077278617970788F44F5F4B
:10F290004093D73741110CC08091D6378F5F809350
:10F2A000D637811105C08091D5378F5F8093D537D0
:10F2B00008952091CE383091CF38BC01C90108960D
:10F2C0000E942279E091CE38F091CF388091D537E5
:10F2D00080878091D63781878091D73782878091C8
:10F2E000D8378387089544E150E069ED77E380E003
:10F2F00090E00E94D678009721F0982789279827D8
:10F3000008958FEF9FEF089586E00C94FB7881E1DC
:10F310000C94FB7880E0E82FF0E0EE0FFF1FE05B3D
:10F32000F64C118210828F5F8430A8F380E090E267
:10F33000899FF0011124E053F74C118E8F5F8430C8
:10F34000B0F380E094E09093131C8093121C80E053
:10F350009DE0989FF0011124EA59F64C1582148221
:10F360008F5F8A30B0F38093111C089540E04430E1
:10F37000A0F4E42FF0E051E0540FEE0FFF1FE05B2C
:10F38000F64C208131812817390729F44093111C4C
:10F39000118210820895452FEACF4093111C0895E1
:10F3A000AF92BF92CF92DF92EF92FF920F931F9393
:10F3B000CF93DF93C091CE38D091CF38843009F409
:10F3C000DCC121E038E33093CD382093CC38309342
:10F3D000D4372093D337833059F4898D8F7083309D
:10F3E00009F06BC088899989892B09F0DCC67FC038
:10F3F000823009F080C08091171C8F5F8093171CAA
:10F40000811113C08091161C8F5F8093161C81118F
:10F410000CC08091151C8F5F8093151C811105C055
:10F420008091141C8F5F8093141C1092D23710921D
:10F43000D1371092653910926439298D822F8D7FD2
:10F44000853041F48A8D8F5F8A8F843109F0ABC695
:10F45000198EA9C6222309F4A6C688899989892B01
:10F4600009F441C08A8D9FEF980F9A8F81119BC636
:10F470008B8D883031F09FEF920F923048F48530B9
:10F4800039F4198E80E88093C9380E94047645C506
:10F49000853038F493E0082E01C0990F0A94EAF7FA
:10F4A00001C090E39A8F8F5F8B8F822F8F70833094
:10F4B000A1F048F4813009F44EC3823009F073C6DC
:10F4C0001092FA374BC3863009F4C6C4883009F469
:10F4D000C3C4843009F067C6BFC484E08093C938D0
:10F4E0000E9404764CC52F70233009F05CC688E07A
:10F4F0008093C93807C5853019F5E091CA38F09175
:10F50000CB3884819581892B09F44DC61092CF3870
:10F510001092CE3885EF97E39093CD388093CC3816
:10F520009093D4378093D337109265391092643911
:10F530001092D2371092D13788E08093C9381BC11E
:10F540008091D937853409F02EC60091DB3710E061
:10F55000102F00278091DC37080F111D8091D137C3
:10F560009091D2378017910708F41DC61093D237B7
:10F570000093D1378091DF378F7309F014C68091E3
:10F58000E037811110C68091603990916139C09146
:10F59000150AD091160A8C179D0759F440916239CB
:10F5A000509163392091170A3091180A4217530776
:10F5B000A1F02091E9373091EA372817390709F08F
:10F5C000F2C52091EB373091EC3780916239909100
:10F5D00063392817390709F0E6C50E947379019647
:10F5E00009F0E1C58091E237863009F429C1813103
:10F5F000E9F1813009F0D7C58091ED37883009F005
:10F60000D2C51092ED378091EF379091F037873F58
:10F610003FEF930710F0099601C008969093F037DA
:10F620008093EF378091E5379091E637A091E737E7
:10F63000B091E8378093E9379093EA37A093EB379E
:10F64000B093EC378091603990916139A091623923
:10F65000B09163398093E5379093E637A093E7370D
:10F66000B093E83780E48093E1377AC50C511109F3
:10F670001093D2370093D13785EF97E39093CD382D
:10F680008093CC388091F3379091F437892B29F00F
:10F690000E948779019609F086C52091EF37309155
:10F6A000F0372115310509F47EC586E699E390937C
:10F6B000CB388093CA38A090ED37B090EE374091A8
:10F6C000170A5091180A6091190A70911A0AA091AC
:10F6D0001B0AB0911C0A0091E5371091E637E090C3
:10F6E000E737F090E837E091CA38F091CB3889E3FA
:10F6F000E83EF80708F057C584819581009721F10D
:10F700002817390709F586819781009719F0A816FF
:10F71000B906D1F4808191818C179D0729F4C280AC
:10F72000D380C416D506B1F08617970729F4C28096
:10F73000D380CA16DB0671F00817190729F48281F5
:10F740009381E816F90631F03D96F093CB38E093BB
:10F75000CA38C9CF1092CF381092CE3882E0809349
:10F76000C93885EF97E39093D4378093D3371092BD
:10F770006539109264390E940476809164399091C1
:10F780006539009709F40FC59C01245E3F4F309303
:10F79000D2372093D1373093DB372093DC37E09199
:10F7A000CA38F091CB3820852093E13721E12093AE
:10F7B000E23708969827892798279093F237809305
:10F7C000F1371092F4371092F3378481958190933A
:10F7D000EE378093ED37868197819093F037809351
:10F7E000EF378091603990916139A0916239B09181
:10F7F00063398093E5379093E637A093E737B0936A
:10F80000E83780819181A281B3818093E937909319
:10F81000EA37A093EB37B093EC3781E098E390930D
:10F82000CD388093CC380E94877980959095009749
:10F8300011F48FEF9FEF9093F4378093F33790C4D8
:10F840000E948479019609F0AEC48091EF379091BF
:10F85000F037009709F4A7C42091ED373091EE37C7
:10F860002115310509F49FC44091E5375091E637E1
:10F870006091E7377091E837E9EEF8E3C0EDD8E33F
:10F88000F080FF20A9F0AC81BD818A179B0781F42D
:10F89000AE81BF812A173B0759F4A881B9814A1765
:10F8A0005B0731F4AA81BB816A177B0709F46EC13B
:10F8B000A096B096A9E3C035DA0711F72091FA3780
:10F8C0002F732230D9F490930F1C80930E1C40E0CC
:10F8D000443090F4E42FF0E0EE0FFF1FE05BF64CB5
:10F8E000208131814F5F8217930791F71092111C8D
:10F8F00020E0C0E0D0E07EC04093111C8091FA3738
:10F9000082FD51C484E18093FA3788E290E09093BD
:10F91000D2378093D13780E58093F9378091F437DF
:10F920009091F8379093F4373091F3379091F737FF
:10F930009093F3373093F7372091F2379091F63761
:10F940009093F2372093F6379091F1379093111CF2
:10F950004091F5374093F1379093F5378F5F80935F
:10F96000F83781110FC081E0830F8093F737811141
:10F9700009C081E0820F8093F637811103C09F5F39
:10F980009093F5378091ED379091EE3790930F1C5F
:10F9900080930E1C2091EF373091F0373093EE3783
:10F9A0002093ED379093F0378093EF378091E537D0
:10F9B0009091E637A091E737B091E8378093E93727
:10F9C0009093EA37A093EB37B093EC37809160398E
:10F9D00090916139A0916239B09163398093E53794
:10F9E0009093E637A093E737B093E8379EC337305C
:10F9F00089F02F5F2430C0F430E2239FC00111242E
:10FA0000FC01E053F74C318D3111F1CF2093111CE3
:10FA1000EF010CC0209721F0428D3A8D341748F742
:10FA2000EC01C053D74CE5CF2093111C209709F46B
:10FA3000BAC3D093CF38C093CE3883E08A8F888FF3
:10FA40001E8A84E08F8B1B8E8091EF379091F03768
:10FA50009D838C838091ED379091EE379F838E83C9
:10FA60008091E5379091E637A091E737B091E8377C
:10FA700088839983AA83BB8381E0898F8091141C3A
:10FA80008C878091151C8D878091161C8E878091A4
:10FA9000171C8F8781E090E0998B888B8091F437D9
:10FAA0008B878091F3378A878091F237898780919D
:10FAB000F137888781E090E00E9459798091F93789
:10FAC000282F207F30E0213531050CF444C0829589
:10FAD0008F7090E00597880F991F880F991F3091BC
:10FAE000101C20E0E22FF0E0E817F90784F5E75258
:10FAF000F84C30A5311105C02093111C1092101C38
:10FB00002AC0313011F42F5FEDCF3230D9F441A546
:10FB10004430C1F42093111C3093101C82A590E056
:10FB2000982F882723A5822B90930F1C80930E1C5F
:10FB3000893C910510F088EC90E09B8B8A8B9D8B23
:10FB40008C8B09C041A5442311F0240FCBCF209307
:10FB5000111C3093101C80E18093FA378091FA37A2
:10FB600082608093FA3782E08093013884E080934A
:10FB700002381092033888EC809304388CE290E0CD
:10FB80009093D2378093D13780E67DC2D093CF381F
:10FB9000C093CE381092C9389091FA3792FF03C0C3
:10FBA000198E80E219C28091F93782958F70880F83
:10FBB000880F8093111C081B11090451110910931F
:10FBC000D2370093D1378F2D8F70823029F4892F4F
:10FBD0008F73823139F41FC0813021F4892F8F73E4
:10FBE0008230C9F0012B19F4892F8370A1F0209184
:10FBF000F137888528133DC22091F2378985281373
:10FC000038C22091F3378A85281333C22091F43704
:10FC10008B8528132EC294FF4AC0688979896115A3
:10FC2000710509F444C0CE010C960E9422793091EE
:10FC3000F5378091D53738133AC02091F637809147
:10FC4000D637281334C09091F7378091D73798135F
:10FC50002EC08091F8374091D837841328C03C8754
:10FC60002D879E878F878B8D81111AC02E89888D55
:10FC70009A8D891B922F969596959695891B280F9C
:10FC80002E8B87FD81959F89392F36953695931B4D
:10FC9000980F9F8B822F869586958695890F888FE2
:10FCA00081E08093C938888D8A8F198A188A498D96
:10FCB000842F8F7090E0FC013197E830F10508F057
:10FCC00072C2E656FF4F0C949E878091C93880FF20
:10FCD00014C083E0898F80E48093C938198A188A18
:10FCE0008091D1379091D237009709F407C122E46F
:10FCF0002093C9380E94597901C18091FA378F73D6
:10FD0000823009F050C227CF8091C93880FF6FC080
:10FD10008091FA378F73823109F069C08091F93789
:10FD2000282F207F30E0213531050CF444C0829526
:10FD30008F7090E00597880F991F880F991F309159
:10FD4000101C20E0E22FF0E0E817F90784F5E752F5
:10FD5000F84C30A5311105C02093111C1092101CD5
:10FD60002AC0313011F42F5FEDCF3230D9F441A5E4
:10FD70004430C1F42093111C3093101C82A590E0F4
:10FD8000982F882723A5822B90930F1C80930E1CFD
:10FD9000893C910510F088EC90E09B8B8A8B9D8BC1
:10FDA0008C8B09C041A5442311F0240FCBCF2093A5
:10FDB000111C3093101C83E0898F8091F137888764
:10FDC0008091F23789878091F3378A878091F43761
:10FDD0008B8781E090E00E94597982E48093C93852
:10FDE000198A188A1092D2371092D13787C080E2D0
:10FDF0008093C9380E940476E091CE38F091CF38D4
:10FE0000118E7CCD8091FA3780FF28C044FD26C03A
:10FE100088899989892B09F0C6C18091D137909141
:10FE2000D23701960E9459792091C938822F80617A
:10FE30008093C9388091D1379091D237892B19F0AE
:10FE400022612093C9380E94047681E090E0998B6A
:10FE5000888B88E0898F1B8E81E10CC185FF1CC0D7
:10FE60008091FF3790E0982F882720910038822BCF
:10FE70002091CC383091CD38280F391F3093CD38B0
:10FE80002093CC382091D1373091D237281B390BB1
:10FE90003093D2372093D1378091D1379091D23798
:10FEA000009749F044FD07C02091C9382260209393
:10FEB000C9380E9459798091FB3790E0982F8827A4
:10FEC0002091FC37820F911D90930F1C80930E1C84
:10FED0002C893D892817390710F0892B21F430939C
:10FEE0000F1C20930E1C80910E1C90910F1C9B8B5D
:10FEF0008A8B8091C938837009F455C11092653995
:10FF0000109264390E9404768091C93885FF07C039
:10FF10001092653910926439198E84E1ABC084FF68
:10FF20000AC0109265391092643981E090E0998B93
:10FF3000888B84E08FCF2091643930916539211509
:10FF40003105E1F080FF02C0198A188A88899989F1
:10FF5000009781F48A899B898217930720F49093F4
:10FF60006539809364398091643990916539998BB2
:10FF7000888B04C090936539809364391B8E80917F
:10FF8000D3379091D4379093CD388093CC388091EB
:10FF9000643990916539892B59F08889998900973E
:10FFA00039F088969093D2378093D13788E10BC08F
:10FFB0008091C93881FFF7C088E290E09093D237F2
:10FFC0008093D13780E18093FA375CC08091C93843
:10FFD00080FFE9C0198E80E18093C9380E940476C1
:10FFE000E2C08091D1379091D237009711F00E94F2
:10FFF00059799091FA378091C93890FF0BC080FFF2
:020000021000EC
:1000000006C087E0898F1A8E198A188A19C086E07F
:10001000898F16C080FF1EC085E0898F198A188AD3
:10002000C2C08091D1379091D237009711F00E94D1
:1000300059798091FA3780FF0DC087E0898F1A8E39
:1000400081E090E00E94597980E18093C9380E9454
:1000500004760FC08091D1379091D237892B49F423
:10006000A2C08091C93880FF9EC087E0898F1A8E18
:100070009AC080E18093FA3788E290E09093D2377B
:100080008093D13780E58093F93788858093F53761
:1000900089858093F6378A858093F7378B8580939F
:1000A000F8378C858093F1378D858093F2378E8574
:1000B0008093F3378F858093F43786E08093E2371F
:1000C0008C819D819093EE378093ED378E819F8157
:1000D0009093F0378093EF37809160399091613938
:1000E000A0916239B09163398093E5379093E637F8
:1000F000A093E737B093E83788819981AA81BB81C3
:100100008093E9379093EA37A093EB37B093EC37BD
:10011000898D84FF05C01092FC371092FB3705C013
:100120001092FB3788EC8093FC3780E48093E137B2
:100130008091D1379091D2379093DB378093DC3721
:10014000109200381092FF371092FE371092FD3750
:100150000E948479809590959093FE378093FD3727
:1001600085E48093D9371092DA371092E0371092F5
:10017000DF378091181C9091191C01969093191CDF
:100180008093181C9093DD378093DE371092E4370C
:100190001092E3370E947379809590959093E4379D
:1001A0008093E33704C01092D2371092D137109267
:1001B000C938DF91CF911F910F91FF90EF90DF90A1
:1001C000CF90BF90AF9008958CE19CE10C94E76FC5
:1001D00090931B1C80931A1C08958CE19CE10C9455
:1001E000EB6FEF92FF920F931F93CF93DF938C01EE
:1001F000EB017A018CE19CE10E94EB6F0097D9F052
:10020000DC0112962D913C9113972C173D0781F438
:100210001696ED91FC911797309769F09701AE0112
:10022000B801DF91CF911F910F91FF90EF9019943A
:100230000E944C70E3CFDF91CF911F910F91FF90FF
:10024000EF90089508950F931F93CF93DF93CDE51B
:10025000DCE1488159816A817B8100E010E02DE476
:1002600031E88DE39CE10E941D6C0E947B65BC011E
:1002700080E090E0288139814A815B810E945D871E
:10028000AB01BC0122E731E889E29CE10E941D6CD0
:10029000DF91CF911F910F91089580915D1C9091F6
:1002A0005E1CA0915F1CB091601C4091591C509144
:1002B0005A1C60915B1C70915C1C880F991FAA1FCF
:1002C000BB1F481759076A077B0710F4DB01CA01F7
:1002D00080935D1C90935E1CA0935F1CB093601C88
:1002E0000C942381CF93DF930E9415740E94867330
:1002F000EC01198218820E94ED80288139810097D3
:1003000019F1FC0140854423F9F0FC01428153813D
:10031000F901EE0FFF1FEE0FFF1FEC0FFD1F5383C0
:100320004283FC01448155812F5F3F4FF901EE0F5D
:10033000FF1FEE0FFF1FEC0FFD1F5183408339831A
:1003400028830E944C70D9CFC901880F991F880F4C
:10035000991F02960E94817388819981892B31F0BF
:100360008EE19CE1DF91CF910C943D72DF91CF91B2
:100370000895AF92BF92CF92DF92EF92FF920F93C8
:100380001F93CF93DF931F921F92CDB7DEB75B0110
:100390000E9486738C01FC01E080F180FA82E98280
:1003A0000E94CE739701220F331F220F331F2E5F3F
:1003B0003F4F82179307A8F00E5F1F4FC12CD12C1F
:1003C000CE14DF0471F0F8014281538160817181A4
:1003D000C5010E94F1800C5F1F4FFFEFCF1ADF0AAB
:1003E000EFCF0F900F90DF91CF911F910F91FF9062
:1003F000EF90DF90CF90BF90AF9008950F930130B2
:1004000099F48091511C9091521CA091531CB09171
:10041000541C80935D1C90935E1CA0935F1CB09352
:10042000601C0F910C9423810F9108954F925F925D
:100430006F927F928F929F92AF92BF92CF92DF92F4
:10044000EF92FF920F931F934A015B01280139013C
:100450004DE15AE0BC018EE19CE10E942172809244
:10046000511C9092521CA092531CB092541C40926A
:10047000551C5092561C6092571C7092581CC0928A
:10048000591CD0925A1CE0925B1CF0925C1C8EEFBF
:1004900091E81F910F91FF90EF90DF90CF90BF9068
:1004A000AF909F908F907F906F905F904F900C9443
:1004B000E8800C944A72CF93DF93E091210AF09187
:1004C000220A1995EC01009729F06A817B8181E06D
:1004D0000E946974CE01DF91CF9108950F931F930D
:1004E000CF93DF93EC01E091230AF091240A199550
:1004F0008C016A817B8181E00E94697481E090E0D7
:10050000012B11F480E090E0DF91CF911F910F91CA
:100510000895E091250AF091260A1994CF93DF936C
:10052000FC01DB0185E0EB0119928A95E9F78581F1
:10053000837011F082E08C938781837021F082E0D8
:1005400012968C9312978581837081F087818370D6
:1005500069F023893489818592852817390731F418
:1005600081E0848312961C92129701C014828581C7
:100570008370823021F0833021F080E003C082E07C
:1005800001C088E011968C93119787818370823027
:1005900021F0833021F080E003C082E001C088E0D8
:1005A00013968C93DF91CF910895CF93DF9300D072
:1005B0001F921F92CDB7DEB7BE016F5F7F4F0E94C3
:1005C0008E82898190E003962A81820F911D2B8172
:1005D000820F911D2C81820F911D2D81820F911D03
:1005E0000F900F900F900F900F90DF91CF91089583
:1005F0004F925F926F927F928F929F92AF92BF9233
:10060000CF92DF92EF92FF920F931F93CF93DF93DE
:1006100000D01F921F92CDB7DEB78C017B012A015B
:10062000BE016F5F7F4F0E948E82F981EA817B81DC
:100630006C818F2F90E003962E2F30E0820F931F56
:10064000870F911D462F50E0840F951FAD818A0FB3
:10065000911D481659060CF4ADC0D80111968C9125
:10066000119780FB662460F8712C83E0660C771C80
:100670008A95E1F712968C91129780FB882480F876
:10068000912C94E0880C991C9A95E1F786288C911E
:100690008770882A13968C91139780FBAA24A0F860
:1006A000B12C85E0AA0CBB1C8A95E1F78A28149628
:1006B0008C9180FBCC24C0F8D12C96E0CC0CDD1CB6
:1006C0009A95E1F78C28D7018C92D80115969C91C8
:1006D0009370B4E09B9F60011124D80116968C9111
:1006E0008370B0E18B9FC0011124C82AD8011796EE
:1006F0008C91B0E48B9FC0011124C82AD7011196B8
:10070000CC92D80118968C91D70112968C93F23026
:1007100079F4D80119968C91D70113968C93D8014E
:100720001A968C91D70114968C9395E0C92E02C02D
:1007300083E0C82EF0E080E090E0200F311FDF2E34
:10074000DC0C0197FE1759F0D901A80FB91F1B96B1
:10075000BC90D701AD0DB11DBC92FF5FF0CFAD2DA8
:10076000723089F497012D0D311DF8018389F9014B
:10077000808381E08D0D9701280F311DAE5FF80158
:100780008489F901808370E080E090E0040F151FF8
:100790000197272F2A0F30E0761751F0F801E80F64
:1007A000F91F4589F701E20FF31F40837F5FF0CF08
:1007B000C90102C080E090E00F900F900F900F9061
:1007C0000F90DF91CF911F910F91FF90EF90DF90ED
:1007D000CF90BF90AF909F908F907F906F905F90E1
:1007E0004F900895AF92BF92CF92DF92EF92FF9217
:1007F0000F931F93CF93DF937C016B01EA0163306A
:1008000071050CF4B0C0FC01808186FBAA24A0F81D
:100810009181292F269526952370B92EB294B694EE
:10082000B69453E0B522382F3770388383FB3327D3
:1008300030F9398384FB332730F93A8385FB8827E5
:1008400080F98B83AC822D83892F829583708E8370
:10085000BF8282818887222371F13381848190E075
:10086000982F8827830F911D9A87898787010B5FAF
:100870001F4F223071F46BEE79E0CE010B960E948F
:100880003873F70186818B8785818C870E5F1F4FB8
:100890001DC02330D9F487E090E0F801E80FF91F7C
:1008A0002081FE01E81BF90B228B0197B0F787012D
:1008B000035F1F4F0BC087010D5F1F4F6BEE79E089
:1008C000CE010B960E9438731A861986BB20B1F1AF
:1008D000A1100DC0F8012081818190E0982F882718
:1008E000820F911D9C8B8B8B0E5F1F4F04C08985DF
:1008F0009A859C8B8B8BF2E0BF120EC06BEE79E079
:10090000CE0145960E943873F80181818D8B8081DC
:100910008E8B0E5F1F4F1AC0F3E0BF1217C087E027
:1009200090E0F801E80FF91F2081FE01E81BF90BA8
:10093000248F0197B0F7085F1F4F08C06BEE79E076
:10094000CE0145960E9438731C8A1B8A98012E1985
:100950003F09C601821B930B98AB8FA71EA70DA75B
:10096000C216D3061CF480E090E001C0C901DF91FB
:10097000CF911F910F91FF90EF90DF90CF90BF909C
:10098000AF90089520E030E00296FC01329740815C
:10099000442331F0FC0131974081240F311DF4CF05
:1009A000C9010895FC01208130E0322F2227818186
:1009B000282B02C0220F331F6A95E2F7832F992755
:1009C000FA01E95DF54F208130E08223932328E08E
:1009D00030E0241B350B02C0969587952A95E2F7E7
:1009E00008956F927F928F929F92AF92BF92CF9213
:1009F000DF92EF92FF920F931F93CF93DF938C01BF
:100A0000EB016A0179012830310524F4A901B6010E
:100A1000CE014AC0590123E0B594A7942A95E1F785
:100A20004115510521F04801612C712C03C0D801FA
:100A3000FB0120C048E050E0B601CE01860D971DB5
:100A40000E94D284F40181934F01FFEF6F1A7F0A55
:100A50006A147B047CF3C501B7FE02C080E090E01D
:100A6000A701477055274115510511F1080F191FAE
:100A7000B60118C0CF018C1B9D0B8A159B051CF479
:100A800081918D93F7CFC501B7FE02C080E090E061
:100A9000A701477055274115510551F0080F191F3F
:100AA00060E070E08C0F9D1F0E94D284F80180836B
:100AB000DF91CF911F910F91FF90EF90DF90CF903A
:100AC000BF90AF909F908F907F906F9008958F927E
:100AD0009F92AF92BF92CF92DF92EF92FF920F93CD
:100AE0001F93CF93DF931F921F92CDB7DEB70E9463
:100AF00086738C0182E090E00E946473892B19F464
:100B000080E090E05DC0F801818190E0982F882717
:100B10002081820F911D0E945B727C01009781F3FE
:100B20000E9486734C01F7012681822F8695869557
:100B3000869590E0422F477021E030E011F420E0EC
:100B400030E0820F931F0E946473892BC9F2F70172
:100B500004811581C12CD12CF8018081882379F181
:100B6000F801A180B12CB60133E0759567953A95EF
:100B7000E1F7A60147705527680D791D883168F0A7
:100B80009501CE0101960E94F184BE016F5F7F4FF7
:100B9000F80180810E947D740DC01A82198295012E
:100BA000CE0101960E94F18469817A81F8018081E9
:100BB0000E946974CA0CDB1C0E5F1F4FCDCFC701AA
:100BC0000F900F90DF91CF911F910F91FF90EF90B9
:100BD000DF90CF90BF90AF909F908F900895DC01F1
:100BE00050E0E0E1F0E0E61BF70BE21BF30B02C084
:100BF000440F551FEA95E2F78C91852B8C93119643
:100C00008C911197842B11968C9308956F927F92FB
:100C10008F929F92AF92BF92CF92DF92EF92FF920C
:100C20000F931F93CF93DF938C016B01EA0179013E
:100C3000283031051CF44881C8015CC0390153E0FB
:100C4000759467945A95E1F76115710521F04E018D
:100C5000A12CB12C03C0D801FE0127C0F4014191A1
:100C60004F0128E030E0B601C8018A0D9B1D0E94AB
:100C7000EF85FFEFAF1ABF0AA614B7047CF3C301D8
:100C800077FE02C080E090E097012770332721159E
:100C9000310509F43FC0C80FD91F488150E0B601A3
:100CA000621B730B685F7F4F1CC0CF018C1B9D0BB9
:100CB000861597051CF481918D93F7CFC30177FEBC
:100CC00002C080E090E0970127703327211531059D
:100CD00009F1C80FD91F488150E068E070E0621B3D
:100CE000730B02C0559547956A95E2F760E070E096
:100CF000800F911FDF91CF911F910F91FF90EF9087
:100D0000DF90CF90BF90AF909F908F907F906F902B
:100D10000C94EF85DF91CF911F910F91FF90EF9091
:100D2000DF90CF90BF90AF909F908F907F906F900B
:100D300008956F927F928F929F92AF92BF92CF92BF
:100D4000DF92EF92FF920F931F93CF93DF931F9247
:100D50001F92CDB7DEB78C01FC018681E82EE694A8
:100D6000E694E694F12C282F277081E090E011F4AE
:100D700080E090E0E80EF91EC70102960E94DE7343
:100D8000009709F445C00E948D73F8012281FC018F
:100D90002083F8012381FC0121830E948D73029638
:100DA0005C01A70160E070E00E947A91F801048183
:100DB0001581E12CF12CF8018081882339F1F801AB
:100DC0008180912C670163E0D594C7946A95E1F71F
:100DD0003701F7E06F227724CA0CDB1C883128F03A
:100DE0000E9487749401AC0108C00E9474749A83B5
:100DF00089839401AE014F5F5F4FB301C6010E942A
:100E00000686E80CF91C0E5F1F4FD5CF81E090E0FD
:100E10000F900F90DF91CF911F910F91FF90EF9066
:100E2000DF90CF90BF90AF909F908F907F906F900A
:100E30000895DB018F939F930E94C287BF91AF916A
:100E4000A29F800D911DA39F900DB29F900D112424
:100E50000895991B79E004C0991F961708F0961B16
:100E6000881F7A95C9F780950895AA1BBB1B51E18D
:100E700007C0AA1FBB1FA617B70710F0A61BB70B0A
:100E8000881F991F5A95A9F780959095BC01CD01AF
:100E9000089597FB072E16F4009407D077FD09D02C
:100EA0000E94358707FC05D03EF4909581959F4FB1
:100EB0000895709561957F4F0895A1E21A2EAA1B9F
:100EC000BB1BFD010DC0AA1FBB1FEE1FFF1FA217FA
:100ED000B307E407F50720F0A21BB30BE40BF50BF7
:100EE000661F771F881F991F1A9469F76095709580
:100EF000809590959B01AC01BD01CF010895052E11
:100F000097FB1EF400940E94968757FD07D00E941D
:100F10005D8707FC03D04EF40C949687509540955E
:100F2000309521953F4F4F4F5F4F08959095809595
:100F3000709561957F4F8F4F9F4F0895EE0FFF1F64
:100F40000590F491E02D19940E94AC87332312F49C
:100F50008A1B9B0B0C94BD87A29FB001B39FC0015D
:100F6000A39F700D811D1124911DB29F700D811DD5
:100F70001124911D08950E94AC87B7FF0895821B2C
:100F8000930B08950E94AC87A59F900DB49F900D80
:100F9000A49F800D911D11240895B7FF0C94C28762
:100FA0000E94C287821B930B0895DF93CF931F93F8
:100FB0000F939A9DF02D219FF00D8B9DF00D8A9D32
:100FC000E02DF10D039FF00D029FE00DF11D4E9DF0
:100FD000E00DF11D5E9DF00D4F9DF00D7F936F9321
:100FE000BF92AF925F934F93D5010E94AC878B0164
:100FF000AC01D7010E94AC87EB01E80FF91FD601C5
:101000000E9425882F913F91D6010E94AC87C60F80
:10101000D71FE81FF91FAF91BF910E9425882F911C
:101020003F910E94AC87C60FD71FE81FF91FD6015A
:101030000E94AC87E60FF71F9801BE01CF01112473
:101040000F911F91CF91DF9108950E94AC87460FB9
:10105000571FC81FD91F08F431960895E894DF93ED
:10106000CF93FC01DB010E94AC877F936F93E90172
:101070009A01AC01BF93AF933F932F93DF010E947E
:10108000AC8726F46C1B7D0B820B930B9E01EB014E
:10109000FC010E942588AF91BF912F913F910E9442
:1010A0002588BE01CF01F9012F913F91CF91DF91AA
:1010B0000895689401C0E894F92FF12B12F00C9474
:1010C0008D88A0E0B0E0E7E6F8E80C94FF88092EF0
:1010D000059422F40E94E988112392F4F0E80F2687
:1010E000FFEFE094F09400951095B094C094D094E4
:1010F000A194BF0ACF0ADF0AEF0AFF0A0F0B1F0BEA
:101100000E94988807FC0E94E988CDB7DEB7ECE022
:101110000C941B89689401C0E8948F929F92CF939E
:10112000DF930E949888DF91CF919F908F900895D0
:1011300088249924F401E401B0E49F93AA279A1526
:101140008B049C04ED05FE05CF05D007A10798F49C
:10115000AD2FDC2FCF2FFE2FE92D982C892E982F25
:10116000872F762F652F542F432F322F2227B850E9
:1011700031F7BF9127C01B2EBF91BB27220F331F12
:10118000441F551F661F771F881F991F881C991CB5
:10119000EE1FFF1FCC1FDD1FAA1FBB1F8A149B045D
:1011A000EC05FD05CE05DF05A007B10748F08A185C
:1011B0009B08EC09FD09CE09DF09A00BB10B2160EA
:1011C0001A94E1F62EF49401AF01BE01CD01000C9A
:1011D00008956095709580959095309540955095BF
:1011E00021953F4F4F4F5F4F6F4F7F4F8F4F9F4F17
:1011F00008952F923F924F925F926F927F928F92BB
:101200009F92AF92BF92CF92DF92EF92FF920F9395
:101210001F93CF93DF93CDB7DEB7CA1BDB0B0FB69F
:10122000F894DEBF0FBECDBF19942A88398848884C
:101230005F846E847D848C849B84AA84B984C884F2
:10124000DF80EE80FD800C811B81AA81B981CE0FE9
:10125000D11D0FB6F894DEBF0FBECDBFED010895CE
:101260000F93083090F0982F872F762F652F542FEB
:10127000432F322F22270850F4CF220F331F441F51
:10128000551F661F771F881F991F0A95B2F70F9188
:10129000089597FB10F8169400080F93083098F003
:1012A0000850232F342F452F562F672F782F892F43
:1012B000902DF4CF059497958795779567955795D9
:1012C0004795379527950A95AAF70F9108952A0D06
:1012D0003B1D4C1D5D1D6E1D7F1D801F911F0895C0
:1012E0000024A7FD00942A0F301D401D501D601DD5
:1012F000701D801D901D08952A193B094C095D0938
:101300006E097F09800B910B08952A153B054C054A
:101310005D056E057F058007910708950024A7FDF0
:1013200000942A17300540055005600570058005BA
:10133000900508955058BB27AA270ED04EC23FD221
:1013400030F044D220F031F49F3F11F41EF4FFC17D
:101350000EF4E095E7FBF5C1E92F50D280F3BA1700
:10136000620773078407950718F071F49EF568C249
:101370000EF4E0950B2EBA2FA02D0B01B9019001B0
:101380000C01CA01A0011124FF27591B99F0593FF4
:1013900050F4503E68F11A16F040A22F232F342F3C
:1013A0004427585FF3CF469537952795A795F0408A
:1013B0005395C9F77EF41F16BA0B620B730B840B9F
:1013C000BAF09150A1F0FF0FBB1F661F771F881F57
:1013D000C2F70EC0BA0F621F731F841F48F48795AF
:1013E00077956795B795F7959E3F08F0B3CF93959E
:1013F000880F08F09927EE0F979587950895DFD10C
:1014000058F080E891E009F49EEFE0D128F040E840
:1014100051E059F45EEF09C09AC112C2E92FE07899
:10142000EDD168F3092E052AC1F3261737074807BF
:10143000590738F00E2E07F8E02569F0E025E06442
:101440000AC0EF6307F8009407FADB01B9019D01B8
:10145000DC01CA01AD01EF9347D0BFD10AD05F9143
:10146000552331F02BED3FE049E450FD49EC63CFCB
:101470000895DF93DD27B92FBF7740E85FE31616A5
:10148000170648075B0710F4D92FE5D19F938F9378
:101490007F936F934AD3E4E4F1E06CD19ED12F9116
:1014A0003F914F915F919ED2DD2349F09058A2EA7F
:1014B0002AED3FE049EC5FE3D0785D274DDFDF9117
:1014C0008CC11BD108F481E008950CD086C17ED177
:1014D00040F075D130F021F45F3F19F032C1511165
:1014E000B0C135C18BD198F39923C9F35523B1F31A
:1014F000951B550BBB27AA2762177307840738F083
:101500009F5F5F4F220F331F441FAA1FA9F333D0E1
:101510000E2E3AF0E0E830D091505040E695001C95
:10152000CAF729D0FE2F27D0660F771F881FBB1F51
:10153000261737074807AB07B0E809F0BB0B802D2B
:10154000BF01FF2793585F4F2AF09E3F510568F077
:10155000F8C077C15F3FECF3983EDCF38695779552
:101560006795B795F7959F5FC9F7880F911D969579
:10157000879597F90895E1E0660F771F881FBB1FD5
:10158000621773078407BA0720F0621B730B840B82
:10159000BA0BEE1F88F7E095089519F40EF0D1C04C
:1015A0004FC1D5C033D1C8F39638C0F707F80F92B2
:1015B000E8942BE33AEA48EB5FE716D20F920F92DA
:1015C0000F924DB75EB70F92CED1E1E7F1E0D2D0E6
:1015D0004F915F91EF91FF91E595EE1FFF1F49F04D
:1015E000FE57E0684427EE0F441FFA95E1F7419556
:1015F000550B3AD10F9007FE2EC1089597FB0EF4BC
:10160000A9D03EC0E89409C097FB3EF49095809520
:10161000709561957F4F8F4F9F4F9923A9F0F92FB8
:1016200096E9BB279395F695879577956795B79536
:10163000F111F8CFFAF4BB0F11F460FF1BC06F5F1C
:101640007F4F8F4F9F4F16C0882311F096E911C02E
:10165000772321F09EE8872F762F05C0662371F04F
:1016600096E8862F70E060E02AF09A95660F771F63
:10167000881FDAF7880F9695879597F90895E8946B
:10168000F92F96EBFF2381F0121613061406440B74
:101690009395F69587957795679557954040FF23E5
:1016A000B9F71BC099270895882351F49850D2F7B1
:1016B000872B762F652F542F432F322F20E0B1F345
:1016C000121613061406440B88233AF09A95440F19
:1016D000551F661F771F881FCAF755234AF4440F0A
:1016E000551F11F460FF04C06F5F7F4F8F4F9F4FF6
:1016F000880F9695879597F90895990F0008550FCB
:10170000AA0BE0E8FEEF16161706E807F907C0F087
:1017100012161306E407F50798F0621B730B840B8F
:10172000950B39F40A2661F0232B242B252B21F469
:1017300008950A2609F4A140A6958FEF811D811D09
:10174000089597F99F6780E870E060E008959FEF43
:1017500080EC089590958095709560955095409592
:10176000309521953F4F4F4F5F4F6F4F7F4F8F4FBA
:101770009F4F0895DF93CF931F930F93FF92EF92A4
:10178000DF927B018C01689405C0DA2EEF012AD12B
:10179000FE01E894A5912591359145915591AEF3BF
:1017A000EF01DADDFE019701A801DA9479F7DF9005
:1017B000EF90FF900F911F91CF91DF91089500243A
:1017C0000A941616170618060906089500240A94A6
:1017D00012161306140605060895092E0394000C2C
:1017E00011F4882352F0BB0F40F4BF2B11F460FFBB
:1017F00004C06F5F7F4F8F4F9F4F089557FD9058E4
:10180000440F551F59F05F3F71F04795880F97FBC4
:10181000991F61F09F3F79F087950895121613067E
:101820001406551FF2CF4695F1DF08C016161706AD
:101830001806991FF1CF86957105610508940895E2
:10184000E894BB2766277727CB0197F9089555DFE2
:1018500008F48FEF08959B01AC0160E070E080E830
:101860009FE333CE6ECF64C1D1DFE8F39923D9F380
:10187000940F511DBBF39150504094F059F08823C0
:1018800032F0660F771F881F91505040C1F79E3F7E
:10189000510544F7880F911D9695879597F90895FE
:1018A0005F3FACF0983E9CF0BB2786957795679597
:1018B000B79508F4B1609395C1F7BB0F58F711F4D1
:1018C00060FFE8CF6F5F7F4F8F4F9F4FE3CFB9CF60
:1018D0000AD029ED3BE54EED5EE378C00EF028C15D
:1018E00036CF68942ECF92DFC8F39923D1F3C6F395
:1018F000DF93CF931F930F93FF92C92FDD27882388
:101900002AF02197660F771F881FDAF720E030E072
:1019100040E85FEB9FE3883920F0803E30F021966D
:101920008F7709DDE9E9F1E003C005DDE6ECF1E0E0
:1019300021DF8B01BE01EC01FB2E6F5771097595FC
:10194000771F880B990B60DE28E132E741E35FE304
:1019500049D0AF2D9801AE01FF900F911F91CF910B
:10196000DF91FADC3ACFFA01DC01AA0FBB1F9B0121
:10197000AC01BF5728F422273327442750781FC0D3
:10198000B75188F4AB2F0024469537952795011C55
:10199000A395D2F3002069F0220F331F441FB395A3
:1019A000DAF30DD0C7CC61307105A0E88A07B946DB
:1019B00030F49B01AC016627772788279078309612
:1019C00021F0208331834283538308950BD005CFC8
:1019D000F6DE28F0FBDE18F0952309F0B2CEB7CE84
:1019E00011242FCF0BDFA0F3959FD1F3950F50E07B
:1019F000551F629FF001729FBB27F00DB11D639FC1
:101A0000AA27F00DB11DAA1F649F6627B00DA11D66
:101A1000661F829F2227B00DA11D621F739FB00D0C
:101A2000A11D621F839FA00D611D221F749F33277C
:101A3000A00D611D231F849F600D211D822F762F15
:101A40006A2F11249F5750408AF0E1F088234AF012
:101A5000EE0FFF1FBB1F661F771F881F915050405E
:101A6000A9F79E3F510570F06CCEEBCE5F3FECF3D3
:101A7000983EDCF3869577956795B795F795E7954A
:101A80009F5FC1F7FE2B880F911D9695879597F95B
:101A90000895FA01EE0FFF1F30962105310599F1E7
:101AA0006115710561F48038BFE39B0749F16894C3
:101AB0009038810561F08038BFEF9B0741F0992392
:101AC00042F5FF3FE1053105210511F1E894089445
:101AD000E795D901AA2329F4AB2FBE2FF85FD0F3E5
:101AE00010C0FF5F70F4A695E0F7F73950F019F0D9
:101AF000FF3A38F49F779F930CD00F9007FC9058D3
:101B000008953EF024CE60E070E080E89FE3089501
:101B10004FE79F775F934F933F932F93E4DE2F918F
:101B20003F914F915F9152DF3DCD9B01AC014ECF74
:101B30009F3F31F0915020F4879577956795B79541
:101B4000880F911D9695879597F908958F929F928A
:101B5000AF92BF92CF92DF92EF92FF92CF93DF933B
:101B6000EC01688179818A819B816115710581050C
:101B7000910521F464E279ED8BE597E02DE133EFF7
:101B800041E050E00E947F8749015A019B01AC016E
:101B9000A7EAB1E40E94C2876B017C01ACEEB4EF0E
:101BA000A50194010E94D087C60ED71EE81EF91E1B
:101BB000F7FE06C081E0C81AD108E10880E8F80AFB
:101BC000C882D982EA82FB82C6019F77DF91CF91DA
:101BD000FF90EF90DF90CF90BF90AF909F908F904D
:101BE00008950C94A68D80E092E00C94A68DA0E060
:101BF000B0E08093000290930102A0930202B093A0
:101C0000030208952F923F925F926F927F928F927C
